:020000040800F2
:1000000000500020F5160008A517000895290008E3
:10001000A5170008A5170008A51700080000000094
:10002000000000000000000000000000A51700080C
:10003000A517000800000000A51700087941000876
:10004000A5170008A5170008A5170008A5170008A0
:10005000A5170008A5170008A5170008A517000890
:10006000A5170008A5170008A5170008A517000880
:10007000A5170008A51700088D400008A51700085F
:10008000A5170008A5170008A5170008A517000860
:10009000A5170008A5170008A5170008A517000850
:1000A000A5170008A5170008A5170008A517000840
:1000B00079110008A5170008A51700080D3A0008D7
:1000C000F53B0008113A0008F13B0008A5170008AD
:1000D000A5170008C1400008FD400008A51700084A
:1000E000A5170008A5170008A517000800000000C4
:1000F0000000000000000000000000000000000000
:0C01000000000000000000005FF808F1A3
:1001100010B5054C237833B9044810B10448AFF347
:1001200000800121217010BDD405002000000000D6
:100130008C01010808B5064B1BB106480649AFF310
:1001400000800648016811B1054A02B1904708BD18
:10015000000000008C010108D8050020D405002013
:100160000000000081F0004102E000BF83F0004386
:1001700030B54FEA41044FEA430594EA050F08BF42
:1001800090EA020F1FBF54EA000C55EA020C7FEA06
:10019000645C7FEA655C00F0E2804FEA5454D4EB83
:1001A0005555B8BF6D420CDD2C4480EA020281EA4D
:1001B000030382EA000083EA010180EA020281EA85
:1001C0000303362D88BF30BD11F0004F4FEA0131D7
:1001D0004FF4801C4CEA113102D0404261EB4101E6
:1001E00013F0004F4FEA03334CEA133302D052426C
:1001F00063EB430394EA050F00F0A780A4F1010428
:10020000D5F1200E0DDB02FA0EFC22FA05F2801861
:1002100041F1000103FA0EF2801843FA05F3594147
:100220000EE0A5F120050EF1200E012A03FA0EFCC6
:1002300028BF4CF0020C43FA05F3C01851EBE371F0
:1002400001F0004507D54FF0000EDCF1000C7EEB0D
:1002500000006EEB0101B1F5801F1BD3B1F5001F4B
:100260000CD349085FEA30004FEA3C0C04F101046A
:100270004FEA445212F5800F80F09A80BCF1004F93
:1002800008BF5FEA500C50F1000041EB045141EA15
:10029000050130BD5FEA4C0C404141EB010111F416
:1002A000801FA4F10104E9D191F0000F04BF0146C1
:1002B0000020B1FA81F308BF2033A3F10B03B3F19F
:1002C00020020CDA0C3208DD02F1140CC2F10C022F
:1002D00001FA0CF021FA02F10CE002F11402D8BF8D
:1002E000C2F1200C01FA02F120FA0CFCDCBF41EA59
:1002F0000C019040E41AA2BF01EB0451294330BD28
:100300006FEA04041F3C1CDA0C340EDC04F1140404
:10031000C4F1200220FA04F001FA02F340EA0300DB
:1003200021FA04F345EA030130BDC4F10C04C4F121
:10033000200220FA02F001FA04F340EA0300294601
:1003400030BD21FA04F0294630BD94F0000F83F44B
:10035000801306BF81F480110134013D4EE77FEA2E
:10036000645C18BF7FEA655C29D094EA050F08BF7A
:1003700090EA020F05D054EA000C04BF194610465B
:1003800030BD91EA030F1EBF0021002030BD5FEA9F
:10039000545C05D14000494128BF41F0004130BDC7
:1003A00014F580043CBF01F5801130BD01F000451B
:1003B00045F0FE4141F470014FF0000030BD7FEA8E
:1003C000645C1ABF194610467FEA655C1CBF0B4689
:1003D000024650EA013406BF52EA033591EA030FA0
:1003E00041F4002130BD00BF90F0000F04BF002198
:1003F000704730B54FF4806404F132044FF00005CB
:100400004FF0000150E700BF90F0000F04BF002143
:10041000704730B54FF4806404F1320410F00045A9
:1004200048BF40424FF000013EE700BF42004FEAA4
:10043000E2014FEA31014FEA02701FBF12F07F4321
:1004400093F07F4F81F06051704792F0000F14BF1E
:1004500093F07F4F704730B54FF4607401F0004562
:1004600021F0004120E700BF50EA010208BF7047B9
:1004700030B54FF000050AE050EA010208BF7047AE
:1004800030B511F0004502D5404261EB41014FF417
:10049000806404F132045FEA915C3FF4DCAE4FF01B
:1004A00003025FEADC0C18BF03325FEADC0C18BF02
:1004B000033202EBDC02C2F1200300FA03FC20FA53
:1004C00002F001FA03FE40EA0E0021FA02F11444A0
:1004D000C1E600BF70B54FF0FF0C4CF4E06C1CEAB5
:1004E00011541DBF1CEA135594EA0C0F95EA0C0F2A
:1004F00000F0DEF82C4481EA030621EA4C5123EA9D
:100500004C5350EA013518BF52EA033541F48011CB
:1005100043F4801338D0A0FB02CE4FF00005E1FB7E
:1005200002E506F00042E0FB03E54FF00006E1FBC8
:1005300003569CF0000F18BF4EF0010EA4F1FF040B
:10054000B6F5007F64F5407404D25FEA4E0E6D414B
:1005500046EB060642EAC62141EA55514FEAC5205C
:1005600040EA5E504FEACE2EB4F1FD0C88BFBCF5D8
:10057000E06F1ED8BEF1004F08BF5FEA500E50F189
:10058000000041EB045170BD06F0004646EA01014F
:1005900040EA020081EA0301B4EB5C04C2BFD4EB81
:1005A0000C0541EA045170BD41F480114FF0000E7A
:1005B000013C00F3AB8014F1360FDEBF002001F0E8
:1005C000004170BDC4F10004203C35DA0C341BDC62
:1005D00004F11404C4F1200500FA05F320FA04F034
:1005E00001FA05F240EA020001F0004221F0004168
:1005F00010EBD37021FA04F642EB06015EEA430EDB
:1006000008BF20EAD37070BDC4F10C04C4F120050A
:1006100000FA04F320FA05F001FA04F240EA0200BD
:1006200001F0004110EBD37041F100015EEA430E8E
:1006300008BF20EAD37070BDC4F1200500FA05F2AE
:100640004EEA020E20FA04F301FA05F243EA02032D
:1006500021FA04F001F0004121FA04F220EA02003C
:1006600000EBD3705EEA430E08BF20EAD37070BD82
:1006700094F0000F0FD101F00046400041EB010162
:1006800011F4801F08BF013CF7D041EA060195F044
:10069000000F18BF704703F00046520043EB0303FE
:1006A00013F4801F08BF013DF7D043EA06037047EB
:1006B00094EA0C0F0CEA135518BF95EA0C0F0CD0F6
:1006C00050EA410618BF52EA4306D1D181EA03013C
:1006D00001F000414FF0000070BD50EA410606BF36
:1006E0001046194652EA430619D094EA0C0F02D17B
:1006F00050EA013613D195EA0C0F05D152EA0336C0
:100700001CBF104619460AD181EA030101F00041DD
:1007100041F0FE4141F470014FF0000070BD41F026
:10072000FE4141F4780170BD70B54FF0FF0C4CF400
:10073000E06C1CEA11541DBF1CEA135594EA0C0F1F
:1007400095EA0C0F00F0A7F8A4EB050481EA030E6C
:1007500052EA03354FEA013100F088804FEA033353
:100760004FF0805545EA131343EA12634FEA022221
:1007700045EA111545EA10654FEA00260EF00041E2
:100780009D4208BF964244F1FD0404F5407402D234
:100790005B084FEA3202B61A65EB03055B084FEAC5
:1007A00032024FF480104FF4002CB6EB020E75EBC2
:1007B000030E22BFB61A754640EA0C005B084FEAEA
:1007C0003202B6EB020E75EB030E22BFB61A754667
:1007D00040EA5C005B084FEA3202B6EB020E75EBB2
:1007E000030E22BFB61A754640EA9C005B084FEA2A
:1007F0003202B6EB020E75EB030E22BFB61A754637
:1008000040EADC0055EA060E18D04FEA051545EA25
:1008100016754FEA06164FEAC30343EA52734FEACE
:10082000C2025FEA1C1CC0D111F4801F0BD141EA47
:1008300000014FF000004FF0004CB6E711F4801FAC
:1008400004BF01430020B4F1FD0C88BFBCF5E06F8C
:100850003FF6AFAEB5EB030C04BFB6EB020C5FEA9C
:10086000500C50F1000041EB045170BD0EF0004EF1
:100870004EEA113114EB5C04C2BFD4EB0C0541EA23
:10088000045170BD41F480114FF0000E013C90E620
:1008900045EA060E8DE60CEA135594EA0C0F08BFE4
:1008A00095EA0C0F3FF43BAF94EA0C0F0AD150EAE3
:1008B00001347FF434AF95EA0C0F7FF425AF104676
:1008C00019462CE795EA0C0F06D152EA03353FF49E
:1008D000FDAE1046194622E750EA410618BF52EA1B
:1008E00043067FF4C5AE50EA41047FF40DAF52EAEF
:1008F00043057FF4EBAE12E74FEA4102B2F1E04369
:1009000024BFB3F5001CDCF1FE5C0DD901F0004CF6
:100910004FEAC0024CEA5070B2F1004F40EB830046
:1009200008BF20F00100704711F0804F21D113F172
:100930003872BCBF01F00040704741F480114FEAAB
:100940005252C2F11802C2F1200C10FA0CF320FA34
:1009500002F018BF40F001004FEAC1234FEAD32351
:1009600003FA0CFC40EA0C0023FA02F34FEA4303BB
:10097000CCE77FEA625307D150EA01331EBF4FF044
:10098000FE4040F44000704701F0004040F0FE405F
:1009900040F40000704700BF80F0004002E000BF5C
:1009A00081F0004142001FBF5FEA410392EA030F5A
:1009B0007FEA226C7FEA236C6AD04FEA1262D2EBA4
:1009C0001363C1BFD218414048404140B8BF5B42A9
:1009D000192B88BF704710F0004F40F4000020F042
:1009E0007F4018BF404211F0004F41F4000121F058
:1009F0007F4118BF494292EA030F3FD0A2F10102A2
:100A000041FA03FC10EB0C00C3F1200301FA03F1DF
:100A100000F0004302D5494260EB4000B0F5000F02
:100A200013D3B0F1807F06D340084FEA310102F1C1
:100A30000102FE2A51D2B1F1004F40EBC25008BF73
:100A400020F0010040EA03007047490040EB00003D
:100A500010F4000FA2F10102EDD1B0FA80FCACF16C
:100A6000080CB2EB0C0200FA0CF0AABF00EBC2506B
:100A700052421843BCBFD0401843704792F0000F59
:100A800081F4000106BF80F400000132013BB5E7AC
:100A90004FEA41037FEA226C18BF7FEA236C21D022
:100AA00092EA030F04D092F0000F08BF0846704787
:100AB00090EA010F1CBF0020704712F07F4F04D155
:100AC000400028BF40F00040704712F100723CBF68
:100AD00000F50000704700F0004343F0FE4040F492
:100AE000000070477FEA226216BF08467FEA236350
:100AF0000146420206BF5FEA412390EA010F40F43B
:100B0000800070474FF0000304E000BF10F0004386
:100B100048BF40425FEA000C08BF704743F096436D
:100B200001464FF000001CE050EA010208BF704788
:100B30004FF000030AE000BF50EA010208BF70470F
:100B400011F0004302D5404261EB41015FEA010C24
:100B500002BF84460146002043F0B64308BFA3F11C
:100B60008053A3F50003BCFA8CF2083AA3EBC253FE
:100B700010DB01FA02FC634400FA02FCC2F120021D
:100B8000BCF1004F20FA02F243EB020008BF20F054
:100B90000100704702F1200201FA02FCC2F12002BA
:100BA00050EA4C0021FA02F243EB020008BF20EAAF
:100BB000DC7070474FF0FF0C1CEAD0521EBF1CEADD
:100BC000D15392EA0C0F93EA0C0F6FD01A4480EACB
:100BD000010C400218BF5FEA41211ED04FF00063B4
:100BE00043EA501043EA5111A0FB01310CF00040E0
:100BF000B1F5000F3EBF490041EAD3715B0040EA06
:100C0000010062F17F02FD2A1DD8B3F1004F40EBD5
:100C1000C25008BF20F00100704790F0000F0CF0A8
:100C2000004C08BF49024CEA502040EA51207F3A6C
:100C3000C2BFD2F1FF0340EAC250704740F4000047
:100C40004FF00003013A5DDC12F1190FDCBF00F038
:100C500000407047C2F10002410021FA02F1C2F1E6
:100C6000200200FA02FC5FEA310040F1000053EA82
:100C70004C0308BF20EADC70704792F0000F00F0D0
:100C8000004C02BF400010F4000F013AF9D040EAD6
:100C90000C0093F0000F01F0004C02BF490011F46A
:100CA000000F013BF9D041EA0C018FE70CEAD15368
:100CB00092EA0C0F18BF93EA0C0F0AD030F0004CE8
:100CC00018BF31F0004CD8D180EA010000F000409C
:100CD000704790F0000F17BF90F0004F084691F05A
:100CE000000F91F0004F14D092EA0C0F01D1420294
:100CF0000FD193EA0C0F03D14B0218BF084608D15D
:100D000080EA010000F0004040F0FE4040F40000A6
:100D1000704740F0FE4040F4400070474FF0FF0C39
:100D20001CEAD0521EBF1CEAD15392EA0C0F93EA80
:100D30000C0F69D0A2EB030280EA010C49024FEAD2
:100D4000402037D04FF0805343EA111143EA10138B
:100D50000CF000408B4238BF5B0042F17D024FF443
:100D6000000C8B4224BF5B1A40EA0C00B3EB510F1E
:100D700024BFA3EB510340EA5C00B3EB910F24BF07
:100D8000A3EB910340EA9C00B3EBD10F24BFA3EB8C
:100D9000D10340EADC001B0118BF5FEA1C1CE0D154
:100DA000FD2A3FF650AF8B4240EBC25008BF20F007
:100DB000010070470CF0004C4CEA50207F32C2BF5B
:100DC000D2F1FF0340EAC250704740F400004FF0F8
:100DD0000003013A37E792F0000F00F0004C02BF29
:100DE000400010F4000F013AF9D040EA0C0093F0F3
:100DF000000F01F0004C02BF490011F4000F013B4D
:100E0000F9D041EA0C0195E70CEAD15392EA0C0FB4
:100E100008D142027FF47DAF93EA0C0F7FF470AFEC
:100E2000084676E793EA0C0F04D14B023FF44CAF2F
:100E300008466EE730F0004C18BF31F0004CCAD1C4
:100E400030F000427FF45CAF31F000437FF43CAF00
:100E50005FE700BF4FF0FF3C06E000BF4FF0010C22
:100E600002E000BF4FF0010C4DF804CD4FEA400204
:100E70004FEA41037FEA226C18BF7FEA236C11D04E
:100E800001B052EA530C18BF90EA010F58BFB2EB01
:100E9000030088BFC81738BF6FEAE17018BF40F081
:100EA000010070477FEA226C02D15FEA402C05D135
:100EB0007FEA236CE4D15FEA412CE1D05DF8040BBA
:100EC000704700BF844608466146FFE70FB5FFF74D
:100ED000C9FF002848BF10F1000F0FBD4DF808ED05
:100EE000FFF7F4FF0CBF012000205DF808FB00BFF6
:100EF0004DF808EDFFF7EAFF34BF012000205DF850
:100F000008FB00BF4DF808EDFFF7E0FF94BF01209C
:100F100000205DF808FB00BF4DF808EDFFF7D2FF99
:100F200094BF012000205DF808FB00BF4DF808EDDC
:100F3000FFF7C8FF34BF012000205DF808FB00BFA9
:100F40004FEA4002B2F1FE4F0FD34FF09E03B3EBD6
:100F500012620DD94FEA002343F0004310F0004F16
:100F600023FA02F018BF404270474FF0000070476C
:100F700012F1610F01D1420205D110F0004008BF0B
:100F80006FF0004070474FF00000704742000ED2F3
:100F9000B2F1FE4F0BD34FF09E03B3EB126209D4B4
:100FA0004FEA002343F0004323FA02F070474FF06A
:100FB0000000704712F1610F01D1420202D14FF0DF
:100FC000FF3070474FF00000704700BF034BDA88D6
:100FD0000280198941805B8983807047F005002079
:100FE000054B1A88510001805A88510041809B8826
:100FF0005A008280704700BFF00500207047000053
:10100000074B084A0360426007480B60074A4FF0ED
:101010007E534860CB604FF4BC711180704700BFB5
:10102000FD0F0008CD0F0008E10F0008420000206E
:1010300038B504460D46002D14DD052003F0CFF829
:10104000204608F033FE204608F035FE0028FAD18D
:10105000204608F034FE204608F036FE0028FAD17B
:10106000013DE8E738BD000070B53E4D90B0284620
:1010700009F02CFC3C4880213C4B06900A91202032
:101080004FF40051002409264FF4807205930D900F
:101090004FF480630E91284605A90C930B92079498
:1010A00009940F94089609F089FC2846012109F05B
:1010B000B2FC009403942E4C01254FF4602220468C
:1010C000694602928DF804508DF805508DF8106035
:1010D00008F0B6FD20460A212A46032308F001FE47
:1010E00020460B210222032308F0FBFD03222046A9
:1010F0000C21134608F0F5FD20460D2104220323A0
:1011000008F0EFFD20460E210522032308F0E9FD3B
:1011100020460F210323062208F0E3FD2046052187
:101120000722032308F0DDFD2046062108220323C1
:1011300008F0D7FD324603232046072108F0D1FDF1
:101140002046294608F0A9FD2046294608F09CFDC6
:1011500020460221FFF76CFF2046294608F0B8FD23
:1011600010B070BD08000240F00500204C24014082
:1011700000240140002070475E4B2DE9F0411C78AF
:10118000002C58D002214FF0804009F016F90128B8
:1011900008D1594C594B21884FF08040198009F0F3
:1011A000FFF8208002214FF0804009F011F95248E9
:1011B000524902880B889A4201D9D21A01E0D843D9
:1011C000121893B2B3F57A6F4D4A03D90023137006
:1011D000BDE8F081A3F2EF2188B240F2DA518842F3
:1011E0001ED81278072A1BD84648032A00EBC201F2
:1011F000CB80454909D840F2D930834205D9012333
:1012000003FA02F2087802430A7009780F2907D11D
:101210003E483D4B016800221A700A68536898479F
:1012200037483A4B01784A1C0270186801680A680E
:101230009047BDE8F0812546354850F8347000EB02
:10124000C402B7F1804F9688B2F806804DD1384677
:10125000414609F0B2F8012847D13846414609F025
:10126000B7F80C2E1CD8DFE806F0071B1B1B0C1B65
:101270001B1B111B1B1B16004FF0804009F090F840
:101280000DE04FF0804009F08EF808E04FF080400C
:1012900009F08CF803E04FF0804009F08AF8054629
:1012A000184AE00012F83410131839B9012019490E
:1012B00002F8340002225D804A8011E05F889D8040
:1012C000BD4201D9EF1B01E0F9436F18DF80002711
:1012D00017540E4A10680368196888470D494F80F3
:1012E0004FF080400E8008F0BFFF0134082CA3D1DE
:1012F000BDE8F0810D060020100600200E0600203B
:1013000054060020140600200C060020C410002003
:1013100000000020020600202DE9F04300248FB0D9
:101320000A2706460D463A46214604A801940BF0CA
:1013300035FC214610220AA80BF030FC844B854A6C
:101340001D6085487578337840F2DC510570D18096
:10135000D181D182D183D184D185D186D187002B0F
:1013600000F0948007A821463A460BF017FC03943E
:101370002820002D42D0012502A98DF80B004FF046
:1013800002087648ADF808508DF80A8008F0A0FBF6
:101390001C2203A88DF80C208DF80D408DF80E50FE
:1013A0008DF80F5008F0F4FC07A808F0DDFE4FF6AA
:1013B000FF704723ADF8200007A94FF08040ADF83B
:1013C0001C30ADF81E4008F087FD65494FF08040A5
:1013D0004C80CC800C810C808D80624C08F044FFE6
:1013E0004FF0804041462A4608F0E1FE4FF0804031
:1013F000294608F0C2FEA946277047E002221F24B2
:101400008DF80B0002A955488DF80A20ADF8084068
:1014100008F05EFB01241C2103A88DF80C108DF848
:101420000D508DF80E408DF80F4008F0B1FC07A864
:1014300008F09AFE4FF6FF704723ADF8200007A989
:101440004FF08040ADF81C30ADF81E5008F044FD60
:10145000434A55809480D5801581434C4049631997
:10146000988808802859083508F0FEFE202DF4D110
:101470004FF080401E21012208F099FE01214FF01B
:10148000804008F07AFE374904250D7018254FF486
:101490007071ADF804108DF8075001A9022533488A
:1014A0008DF8065008F014FB04A808F05DFE33899F
:1014B0002F48472290FBF3F4611EADF814102D481D
:1014C00004A9ADF8102008F007FD4FF47A704FF42E
:1014D0008071702200230124ADF82E00ADF8341085
:1014E00024480AA9ADF82820ADF82C30ADF82A40E0
:1014F000ADF8305008F03AFD0AA91E4808F07AFD10
:101500000AA91C4808F0BAFD0AA91A4808F0F8FD13
:101510000821184808F054FE0821164808F058FE23
:101520000821144808F05EFE0821124808F062FE07
:101530002146104808F021FE21460E4808F029FEF9
:101540000C48082108F03CFE0FB0BDE8F08300BF56
:10155000C4100020140600200D06002000080140E1
:10156000020600201206002000000020000C0140AE
:1015700040420F0000080040044B1A78824203D911
:10158000034B53F820000180704700BF1206002073
:10159000ACDB000870470000024B03EBC000C088C2
:1015A000704700BF14060020F8B5134B05469B8911
:1015B0000E461446ECB116B116F8017B00E0FF2789
:1015C0000D48022108F036FB0028F9D00A483946B8
:1015D00008F02BFB0848012108F02CFB0028F9D06B
:1015E000054808F024FBC0B20DB105F8010B013C21
:1015F000E0E70120F8BD00BF003800402DE9F047CA
:10160000012188B04FF4804009F05CF8374C01218B
:101610004FF4804009F06EF803214FF42040182366
:10162000ADF800008DF80310204669468DF80230B1
:101630004FF0040802F0E6FA2D4E4FF480422046A7
:101640006946ADF800204FF480554FF0100A8DF830
:10165000028002F0D7FA69462046ADF800508DF8B6
:1016600002A002F0CFFA304608F082FA07214FF4C8
:10167000007000230222ADF81600ADF81C104FF0E8
:101680000109304603A94FF48277ADF80C30ADF86C
:101690001030ADF81A30ADF81220ADF80E70ADF87C
:1016A00014901F46ADF818A008F094FA3046494649
:1016B00008F0AFFA9F238DF804308DF805708DF88F
:1016C00006708DF807700DEB08014246656102A8AF
:1016D000FFF76AFF25619DF80900B0F1EF014A426A
:1016E00052EB010008B0BDE8F08700BF000C0140DC
:1016F000003800401D481E49026800608A4200F020
:101700001F80002100F004B81A4B5B58435004318D
:1017100019481A4B42189A42FFF4F6AF184A00F0E3
:1017200003B8002342F8043B164B9A42FFF4F9AF8A
:1017300008F0B0F80BF03AF901F010F8FFF7FEBF2F
:10174000114E124830601248016821F0706101604A
:10175000410201600F4C182020600F490F480860BB
:101760000F48D0F800D0406800470000F04F00203C
:10177000EFBEADDEB001010800000020D40500205E
:10178000D405002020170020181002400900000096
:1017900004000140140C0140000C01404434434457
:1017A00000F0FF1FFFF7FEBF014B186802F065BA9B
:1017B000101700200149002000F07ABEA917000888
:1017C00010B5FFF7A3F90A49FFF7F4F90949FFF744
:1017D000A5FA094B044618680078FFF797F9014607
:1017E0002046FFF7E7F9FFF7D1FB80B210BD00BF3D
:1017F0003333534000F07F456806002038B50D4C68
:1018000000202578FFF7B6FC0B4A05F0070322F805
:1018100013000135002325701846D15A02334018B1
:10182000102B80B2F9D1C008FFF7CAFF034A10702D
:1018300038BD00BF5506002056060020C810002005
:10184000074B084A19781088884207D3064B1A6854
:10185000907888428CBF002001207047002070479C
:10186000C8100020CA10002068060020124B70B576
:101870001860202400250020FFF77CFC2D180A208A
:1018800002F0ADFC013CF6D1C5F34F10FFF798FF15
:10189000094902230A6851784D006619B04203D302
:1018A0000133062B0C44F8D104489278037053435B
:1018B00003490B8070BD00BF680600204000002077
:1018C000CA1000202DE9F04F0446008885B048B9C1
:1018D000B4F9023043B9B4F90420D2F1010138BFA0
:1018E000002102E0002100E0014611F0010377D160
:1018F0003D4D00B22B7000F00BFD0646B4F902001E
:1019000000F006FD0546B4F9040000F001FD0446B0
:10191000304609F0A3F80746304609F013F980462F
:10192000284609F09BF80646284609F00BF90546BB
:10193000204609F093F88246204609F003F939461B
:1019400081465046FFF736F9394683464846FFF749
:1019500031F9514601904046FFF72CF94946029073
:101960004046FFF727F9314603905046FFF722F92A
:101970001E4C4946206006F10040FFF71BF929463E
:101980006060A5600298FFF715F901460198FFF71E
:1019900009F82946E0600398FFF70CF9014658461C
:1019A000FEF7FEFF3146206108F10040FFF702F923
:1019B000294660615846FFF7FDF801460398FEF797
:1019C000EFFF2946A0610198FFF7F4F8014602985D
:1019D000FEF7E8FF3946E0613046FFF7EBF820629A
:1019E00005B0BDE8F08F00BF410000206C0600206C
:1019F0002DE9F8434D4B0C460168013A1960808887
:101A00009880072A30D8DFE802F004080F14191E66
:101A10002226188820805A8803E0598821801A8855
:101A2000524262809A881EE01988484220805A8873
:101A3000F6E75988484220801A88F2E71988484218
:101A4000208058880CE05A882280188808E019887D
:101A500021805A8803E05988484220801A885042E1
:101A600060809B885A42A280314B1A78002A5AD152
:101A7000B4F90000FFF74AF88046B4F90200FFF716
:101A800045F80746B4F90400FFF740F8294D06462B
:101A900029684046FFF78EF8E96881463846FFF727
:101AA00089F801464846FEF77DFFA9698146304620
:101AB000FFF780F801464846FEF774FF09F002F888
:101AC000696820804046FFF775F8296981463846E5
:101AD000FFF770F801464846FEF764FFE969814662
:101AE0003046FFF767F801464846FEF75BFF08F00F
:101AF000E9FFA96860804046FFF75CF869698046A5
:101B00003846FFF757F801464046FEF74BFF296A73
:101B100007463046FFF74EF801463846FEF742FFCB
:101B200008F0D0FFA080BDE8F88300BF9006002039
:101B3000410000206C060020F8B5154C06462378BD
:101B4000274663B902F03AFB124D2A6832329042BE
:101B500005D30123237002F031FB2860F8BD3878EB
:101B6000A0B102F02BFB0B4C2168731898420DD3E7
:101B700007480022027002F021FB074920600B7821
:101B80000BB15A1E0A70054901200870F8BD00BF4C
:101B900096060020A0060020980600209906002046
:101BA00037B58DF805101F498DF807300B788DF883
:101BB000040002A88DF80620C21812F8044C0D4645
:101BC000443CE0B20A2828D81749022B31F81040CB
:101BD00003D814B12046FFF7AFFF2B78022B0BD9A7
:101BE000124D2D6802F0EAFA021B954204D20D490B
:101BF0000F4B0020087018700E4802780146012A29
:101C000000D074B9074B1878022801D8421C1A700A
:101C100000230B7008490B7003E03224022BD9D942
:101C2000DBE73EBD9B060020CCDB0008A0060020C1
:101C3000980600209906002096060020014B1860A7
:101C4000704700BFC410002070B53D4B04465A7B5E
:101C50003C4802B1012202704FF4007000F068F9B4
:101C6000002828D0384E394B316858780D6800303C
:101C700018BF0120AA68904748B13368344D1868EE
:101C8000012102692970904708B1022129702E4D67
:101C90002B681868C268904728B12C494B7813B953
:101CA0002B4A0220107029680B689869804710B190
:101CB000274900220A70202005F010F860B1204862
:101CC000244B827A0AB9C17A21B12048C27A0AB972
:101CD000012100E0002119701D4B1878022802D163
:101CE0004C204E211DE0012807D14D2153204C22CC
:101CF0000B46BDE87040FFF753BF164A1178012923
:101D000003D1532001464E2206E00E4B18780128DD
:101D100004D15320014602464D23EAE724B1532063
:101D20004D210A464423E4E70B4A117821B13220C1
:101D3000BDE87040FFF700BF084B1C7070BD00BFCE
:101D40009416002097060020C4100020831600205F
:101D50009C0600209A060020980600209606002087
:101D60000E4B1A78402A16D15888B0F5667F12D1EA
:101D70001979BE290FD193F895230020EF2A0CD1B1
:101D800013F8011B064A48409342F9D1D0F10100F3
:101D900038BF0020704700207047704700F80108E6
:101DA00098FB010838B50F4C204605F061F80E4B42
:101DB00020461F3CB3F8D010B3F8D220254605F0DA
:101DC00071F815F8BE0B02F0B7FC284603F0F0FEE0
:101DD000601C03F0ABFF04F1B400BDE8384000F034
:101DE0006BBC00BF87140020CC10002010B5FFF79B
:101DF000B7FF10B90A2002F095FA0E4C0E492046A2
:101E00004FF466720AF01CFE94F89433022B02D948
:101E1000002084F8940394F89413CC2202FB01432D
:101E2000064803F598710AF00BFEBDE81040FFF775
:101E3000B9BF00BFCC10002000F8010868140020D2
:101E400008B5FFF7D3FF0F2014210122BDE8084099
:101E500007F000BD08B5054BCC2202FB0030044959
:101E600000F598700AF0ECFD08BD00BFCC10002012
:101E700068140020224A38B5402313704FF466706E
:101E80000023BE21EF245080117182F8954382F81F
:101E900096331D461A4A985C0133B3F5667F85EA8E
:101EA0000005F7D182F8965308F01EFB04250024A4
:101EB000691E11F0FF0516D0342008F029FB1148E7
:101EC00008F07CFB0F4C04280BD10F4A2046A15888
:101ED00008F04AFB0D4B04349C42F4D1042804461C
:101EE00001D00446E4E708F00BFB042C02D1FFF715
:101EF00037FF20B90A20BDE8384002F013BA38BDD8
:101F0000CC10002000F80108CC18FE1798FB01083F
:101F1000C82314211E22038001238170C270037123
:101F200064214FF496722823C18002814381704757
:101F3000034B996808420CBF00200120704700BF86
:101F4000CC100020024B9A6810439860704700BF85
:101F5000CC1000202DE9F347AE4AAF4D1068516810
:101F6000AE4C6B4603C34FF46672002128460AF05C
:101F700015FECC22002120460AF010FE402003214D
:101F8000287002206971FFF7DDFFFA22A5F8F22020
:101F90002A236E22A5F8EE304FF4FA7085F804215A
:101FA0002B2340F24C42A5F8F60085F8053121209C
:101FB00002F54873202185F80601A5F8163140F294
:101FC0007E404FF47A7300274FF001094FF41676E4
:101FD00085F8F410A5F8142140F2DC5100F52F72B9
:101FE000A5F8D00003F5CB70A5F8F060A5F81211A4
:101FF000A5F8D22085F89473A5F8F870A5F8FA70C2
:10200000A5F8FC7085F8E27085F8E37085F8E47057
:10201000A5F8E670A5F8E870A5F8EA7085F8ED7007
:1020200085F8EC9085F8077185F82C7185F82D718D
:1020300085F82E7185F8107185F8187185F8197179
:1020400085F81A91A5F8D430A5F8D6006C30A5F81B
:10205000D8004FF4C870A5F8DE004FF416503223B4
:1020600040F2B452C5F8240140F6AC50A5F8DA208D
:10207000A5F8DC301A46A5F8E030A8814FF4E1332A
:102080001E20C5F82031E07252232073552085F8B8
:102090002A31E07017230B204FF028086375A375D1
:1020A00060712D2314204FF0080E63732271A0710C
:1020B00085F81C7185F81D7185F8287185F82971DE
:1020C000AF7385F81B71277084F8018084F8028053
:1020D000E775A7732776E773677684F810E0607476
:1020E0005020E076E1845A200421A3764FF00E0AB6
:1020F00020722375E077412384F82E10484849491F
:1021000084F807A04FF0640C4FF00A0A4FF0780EE5
:1021100084F82030444B84F8212060631522E16369
:10212000424805F5847184F812A084F81CC084F834
:10213000098084F80AE084F81E9084F83120A363B3
:1021400084F8237084F8247084F8257084F8227051
:102150006785A785278584F82F8084F8308084F8E8
:10216000409004F0DDFE4FF44872C8204FF49663AF
:1021700040F2D9313E4684F86C7084F86D7084F872
:102180006E8084F86F9084F87270A4F8702084F8E0
:10219000B4A084F8B500A4F8B630A4F8B8104FF491
:1021A0007F724FF4FA601DF80710A4F87420A0F5B0
:1021B000FA73FF220137A4F87600A4F8783084F887
:1021C0007A1084F87B200834082FE8D113480124C2
:1021D00080F8BA4080F8BB4080F8BC40BE30FFF7C2
:1021E00097FE00200C4B0021C2181030C02811614E
:1021F000F8D100240E48CC2220180849CC340AF02B
:102200001FFCB4F5197FF5D102B0BDE8F047FFF728
:1022100031BE00BF94DB0008CC1000206814002001
:102220009A99193F3D0A773FF6287C3FE2DB000888
:10223000FC11002008B5FFF793FD18B9BDE8084070
:10224000FFF788BE08BD0000024B9A6822EA000032
:1022500098607047CC100020014B9868704700BF11
:10226000CC100020884203DB8242B4BF11460146F5
:10227000084670470023036170472DE9F041066965
:1022800004460136012E0D46066105D1002361602A
:1022900021608360BDE8F081D0F8008008464146A7
:1022A000FEF77EFB07463046FEF730FC0146384617
:1022B000FEF734FD01464046FEF774FB06466060BB
:1022C00031462846FEF76CFB01463846FEF772FCA5
:1022D000A168FEF767FB2660E060A060BDE8F081C2
:1022E00010B504460069012807DD0138FEF70EFC31
:1022F0000146E068FEF712FD10BD002010BD08B5D4
:10230000FFF7EEFFBDE8084008F0AABC000000009F
:1023100008B5FEF779F804A3D3E90023FEF7DAF84D
:10232000FEF7EAFA08BD00BF399D52A246DF913F91
:102330002DE9F041069C06460F46002B0CBF4FF0DE
:1023400020084FF03008204610F8013B0BB9154625
:1023500003E0002AFBDD013AF6E7002D04DD3046FC
:102360004146B847013DF8E714F8011B11B130466A
:10237000B847F9E7BDE8F0812DE9F04389B006469A
:102380000F4603921C46039A134613F8011B03934E
:10239000002900F08A80252901D0304683E0002002
:1023A00004905578911C302D039105D19578033216
:1023B00003924FF0010800E08046A5F13003D8B247
:1023C000092806D8284603A90A2204AB00F00CF914
:1023D00005466C2D05D10399012211F8015B03918B
:1023E00000E00022642D2FD010D8582D3AD006D806
:1023F000002D5AD0252DC6D13046294653E0632DF5
:10240000C1D130462178251DB8474AE0752D0DD041
:10241000782D27D0732DB6D1251D24683046009421
:102420003946049A0023FFF783FF3AE0251D206810
:102430000A2122B1002205AB00F060F802E005ABF2
:1024400000F08CF82C4623E005AD04F10409206867
:10245000294612B100F077F801E000F0A4F84C46EC
:10246000009517E004F104092068102142B1B5F18C
:102470005804634253EB040205AB00F03FF806E05A
:10248000B5F158035A425A4105AB00F067F84C4683
:1024900005A8009030463946049A4346FFF748FFA6
:1024A00071E72C466FE7B8476DE709B0BDE8F083E8
:1024B000024B196002490860704700BFA406002063
:1024C000A80600200FB407B5094904AB08680949FC
:1024D00053F8042B09680193FFF74EFF064B186869
:1024E00001F0EAFB0028F9D0BDE80E4004B07047C7
:1024F000A8060020A406002010170020F0B5012433
:10250000B0FBF4F58D4201D34C43F9E70026C4B18A
:10251000B0FBF4F504FB1500B4FBF1F41EB9002D7B
:1025200001DC002CF4D1092DEFB204DD002A0CBF30
:102530005725372500E03025ED1903F8015B0136FA
:10254000E5E71C70F0BD00280B4603DA2D2240425F
:1025500003F8012B0A210022FFF7D0BFF0B50124B8
:10256000B0FBF4F58D4201D34C43F9E70026C4B12A
:10257000B0FBF4F504FB1500B4FBF1F41EB9002D1B
:1025800001DC002CF4D1092DEFB204DD002A0CBFD0
:102590005725372500E03025ED1903F8015B01369A
:1025A000E5E71C70F0BD00280B4603DA2D224042FF
:1025B00003F8012B0A210022FFF7D0BFA0F130035E
:1025C000DAB2092A01D818467047A0F1610105293D
:1025D00001D857387047A0F14103052B01D837388F
:1025E00070474FF0FF3070472DE9F8430D680446FF
:1025F0000F469046994600262046FFF7DFFF002849
:1026000006DB404504DC08FB060615F8014BF3E742
:102610003D602046C9F80060BDE8F883014B002208
:102620009A807047AC060020034BB3F90400D0F148
:10263000010038BF00207047AC0600200649074B58
:102640000A68B3F90400137805214B439842D4BFBC
:1026500000200120704700BFB4060020AC06002017
:1026600010B50446FFF7EAFF002814BF20460020FB
:1026700000F0010010BD0000074B084A1968B2F9CC
:1026800004004B780A78D118052251438842D4BF00
:1026900000200120704700BFB4060020AC060020D7
:1026A000044B9A8811B2142901DD143A00E000228B
:1026B0009A807047AC060020024B00221860024846
:1026C00082807047B4060020AC060020034B04490A
:1026D0001860044800220160C2807047B8060020DC
:1026E000ECDB0008AC06002008B502F00DF8024B48
:1026F00000221A7008BD00BF8316002010B5FFF736
:102700009DFFE0B1104B5C78201C18BF0120FFF743
:10271000A7FF70B10D480E4B01680E484A89016849
:102720001A805A809A804A88DA800B4BD888411CDC
:10273000D980FFF7A1FF00B90CB9FFF7D5FF064B11
:102740009A88501C988010BD83160020B80600207F
:10275000CC160020B4060020AC06002070B5804CDA
:1027600086B0A07B003018BF012001F043FDFFF7C9
:1027700021F8FFF75FFDFFF739FB94F8073133B11C
:10278000012B01D0092B02D18DF8003004E000218B
:102790008DF8001084F807116846FEF765FC714853
:1027A000FFF790F8022004F0A3FA02F091FC6C4AC3
:1027B00055790E2D01D0082D01D1012600E000260B
:1027C0004FF480708DF80A60FFF7B2FB18B908204B
:1027D000FFF7AEFB00E0012000F0010440208DF87F
:1027E0000640FFF7A5FB8DF807000120FFF7A0FBCF
:1027F0008DF805000820FFF79BFB80F001008DF8A5
:10280000040003F0B5F8584B554D93F8BC108DF803
:102810000800B5F8DE604FF47A70B5F8E040C1F317
:102820008002ADF810004FF480408DF80920ADF81B
:102830000C60ADF80E40FFF77BFB18B1B5F8DA304D
:10284000ADF81030BDF80C10B1F5FA7F02D90022B6
:10285000ADF81020444CB5F8126195F80751B4F862
:10286000B800012DADF81260ADF8140004D0092DA8
:1028700001D1072500E000253C488DF80B50FFF7FB
:1028800025FF3B4E3060FFF7D9F901A83168FEF70C
:1028900043FD3648316804F071FA4FF48070FFF759
:1028A00047FB68B10820FFF743FB48B92C4B314A7E
:1028B00093F81D0193F81C11A2F1BD0303F086FAF1
:1028C0002D4C4FF400414FF4805261610A26C4F848
:1028D0001028294C013EE06880F40045E560274D52
:1028E0001920EB6883F48051E96001F078FC19202D
:1028F00001F075FC16F0FF06EBD14FF400404FF4E9
:1029000080522A61206100F0EBFE01F0A1FF02205D
:10291000FFF70EFB10B11A48FEF7A8FF194805F0A3
:10292000CBF84FF40060FFF703FB10B1164804F03A
:10293000B3FD01F029FC0A4D144C6B792060052B86
:1029400003D14FF4C87000F017FD4FF47A70104EA9
:1029500000F018FE0121717300F002FAFCE700BFDD
:10296000CC100020B211002068140020D4110020E7
:10297000C41000202615002000080140001001406E
:10298000D0110020EC11002010170020C8060020F4
:102990008316002008B5034BB3F9D40002F0B4FC51
:1029A000FEE700BFCC1000200B4B0C481A8852B930
:1029B000817841B142786AB9012141700848094BD8
:1029C00002881A807047437823B90220FF21012230
:1029D00006F040BF704700BF20070020831600208C
:1029E0007A150020421500202DE9F04FB54BB64A6C
:1029F000B3F90600D18C85B088420FDBB0F5FA6FD1
:102A000092F8254007DA451A6C43A1F5FA6694FB63
:102A1000F6F4643403E0C4F1640400E06424AB4AD7
:102A2000A94BB2F8127192F9EC2093F82310009799
:102A3000574293F86C50019193F86D60B9B293F8D6
:102A400024300291002103930A469E4FDDF8008056
:102A500031F907C040F2E637C8EB0C0303F2F31E6E
:102A6000BE4503D8002BB8BF5B4201E04FF4FA73B8
:102A7000022ADFF864822CD025B1AB42CCBFC5EB73
:102A8000030300236427DFF880A293FBF7FE6FF0B7
:102A9000630B3AF81E900BFB0E3B0EF1010E3AF958
:102AA0001EA00FFA89FECEEB0A0E0EFB0BFE9EFB5C
:102AB000F7FEF14428F80190DDF8048003FB08FEDE
:102AC000834B9EFBF3F3DB199BB2634393FBF7F756
:102AD00012E026B1B342CCBFC6EB03030023029F32
:102AE0005F43A8F80470039F002BB8BF5B427B4391
:102AF000774F93FBF7F76437734B02EB030E9EF8A7
:102B00000190642307FB09F898FBF3F9DFF8FC81D7
:102B100002F808909EF80B909EF815E007FB09F864
:102B200007FB0EF798FBF3F9DFF8E48197FBF3F36B
:102B300002F80890DDF80080664FC445D35503DAEB
:102B4000654BCF5A7F42CF5201320231032A7FF4C4
:102B50007CAF5E4C4FF4FA62B4F81411FFF782FBBD
:102B6000B4F814614FF47A75801B4543C6F5FA63D7
:102B7000B5FBF3F56421594895FBF1F36FF063065B
:102B800030F8132006FB0355013330F9130013B25C
:102B9000C01A4543524B504C95FBF1F1587A8A18B4
:102BA000E280002838D04F4F4F4D3E882988721A56
:102BB00010B2FFF7ADFB074607F050FF0646384658
:102BC00007F0C0FF0546B4F90200FDF79FFF074676
:102BD000B4F90000FDF79AFF31468046FDF7EAFFA1
:102BE000294681463846FDF7E5FF01464846FDF790
:102BF000D7FEFEF7A5F9314620803846FDF7DAFF0B
:102C0000294606464046FDF7D5FF01463046FDF70A
:102C1000C9FEFEF795F960800220FFF789F990B1AF
:102C2000324806220378591CCBB20370B3FBF2F092
:102C300002FB103111F0FF0F05D1FEF7DFFDFEF7AB
:102C4000FFFD2B4B18702A4A1078003018BF012066
:102C5000FEF7FAFF27490B881BB9274A108828B9C5
:102C60000AE0022004F03AF80028F6D0234BDA6894
:102C700082F48051D9600EE0194B997819B11F4A3E
:102C80004FF4805010615B781BB11C484FF48051A9
:102C9000416104F0DDFB1A481A4A01681368C81A3A
:102CA000002839DB0E4B587BA0BB9870134B01F505
:102CB000F421D86880F48050D86001F590731360D7
:102CC0002AE000BFCC16002068140020CC100020A1
:102CD0000CFEFFFF73150020AA160020B41600207A
:102CE000831600207A15002042150020E7060020F8
:102CF000E0060020EA060020200700200010014026
:102D0000C4060020CC060020F01600207615002016
:102D1000701500200121997004F0DAFE0C4A107839
:102D200030B94FF40060FFF703F908B104F0CCFBB1
:102D3000202003F0D3FF18B10649086803F0B4FF60
:102D4000054B9A680AB10548904705B0BDE8F08F79
:102D50002C100020C4060020581500203615002035
:102D600038B50820FFF7E4F890B1A14B93F81001B3
:102D700003280CD8DFE800F00202050804F016FB77
:102D800006E004F05FF903E004F01AFA00E0002026
:102D90009849994A0B681168591A002902DA0028E3
:102DA00000F0298203F59C4494482034944914602F
:102DB00004F006F84FF48040FFF7BAF820B1914DC7
:102DC0002B780BB901F0A0FC894A92F81B11B1B124
:102DD0008D4CC81C34F910504FF47A720021A5F5BF
:102DE0007A70FFF73FFAFDF791FE8849FDF796FFED
:102DF0008749FDF7DFFEFEF7C9F8864B18804FF4D0
:102E00000070FFF795F820B1834A1168086844699B
:102E1000A047774D0022B5F81401B5F816411346C6
:102E200079499B08555E8542C4BF63F07F03DBB2DE
:102E3000A542B8BF43F040030232082AF0D17748D8
:102E4000774A047805469C4204D11078F92803D8C3
:102E5000411C00E0002111704FF480402B70FFF7FF
:102E600067F868B1624D684BB5F81211B5F8DC200F
:102E7000B3F90640881A844202DD8B189C420CDBB1
:102E80004FF48040FFF754F8D8B95F4C5849B4F973
:102E90000650B1F81421954213DA01F03DFC01F01F
:102EA00043FC6048B0F842305BB1564C5E4925782F
:102EB000002D00F02D820A78002A00F02982FFF709
:102EC00073FD574B1C78142C40F0D880564D6C780D
:102ED000ECB1544BB3F842502DB950490A785F2AEF
:102EE00001D101F011FC424890F81841002C00F08B
:102EF000C5804C4BB3F84250002D40F0BF8047498D
:102F00000A787D2A40F0BA8001F0FEFBB6E0434D1E
:102F10002978572918D1454B4FF47A744FF48070B3
:102F20001C80FFF705F808B102F0AEFE042003F0A4
:102F3000D5FE10B13E490A250D80082003F0CEFED3
:102F4000D8B93C4A108018E00420FEF7F1FFA0B188
:102F50002A785A2A11D1384803781BB1047001220B
:102F6000364809E0364C3748257885F00101217054
:102F700009B1022200E003220270284804785D2C87
:102F800000F0CD815B2C00F0CC815E2C00F0CB8179
:102F90002448B0F8424034B9204B1D786F2D02D13F
:102FA000FFF702FD15E012491C4891F818211AB1EB
:102FB00014B904787E2CF3D00378972B04D12248DF
:102FC0004FF4C872028004E0A72B02D116490125F4
:102FD0008D73124C2378BB2B03D1124CA18D8D1C09
:102FE00004E0B72B32D10F4CA38D9D1EA58539E08F
:102FF000CC100020C4060020BC060020D411002004
:10300000B216002094160020CC16002000007A444E
:1030100000C07F4440150020C4100020C0060020DE
:10302000D806002068140020831600202007002006
:10303000100700207A150020E6060020E806002090
:10304000D006002098060020EA060020BE2B03D1FF
:10305000774D688D821C04E0BD2B0FD1744D698DB6
:103060008A1E6A85734A744C92F89403FEF7F2FE46
:10307000FEF700FFFEF7E4FE002020700420FEF7BC
:1030800057FF00282CD06D4C207888B16C4B5D78B0
:1030900075B16C49674AB1F90600B2F8143198422B
:1030A00006DD694D2A781AB96849322008802270F5
:1030B000654C637C53B1664B1D782DB9654A107819
:1030C00010B9624C32212180012408E0614D2A7838
:1030D00032B15B48417819B95F4B297001241C70EB
:1030E00000235E4C1A4634F8020F40F2135501B229
:1030F000A942CCBF0025012505FA03F5A0F2155021
:10310000B0F5C77F8CBF002001202A435D1C00FA68
:1031100005F0024340F2A4608142D4BF00210121A6
:10312000981C01FA00F103330A430C2B92B2DAD156
:1031300000233F49444C01EB4300B0F842100A42DF
:103140000CBF0020012018550133152BF1D16278F6
:1031500022B1022003F0C2FD68B914E04FF4007000
:10316000FEF7E6FE78B13E4C21680868C3689847D0
:103170000028EED107E0324CE17839B901F0CCFA01
:103180000120E07002E02E4C0022E2702E4B2C4C0D
:10319000987830B121790022E27019B901F0BCFAB7
:1031A00001202071284B26491A780AB9012008709D
:1031B000CA782C4B12B92249087918B14FF4004152
:1031C000596102E04FF400421A61202003F086FDAD
:1031D00008B103F00BFD1C4B19481A7B02B1012208
:1031E000144982724B79082B01D00E2B45D1144A19
:1031F0000020507241E01C480368042B3DD8DFE8F2
:1032000003F00305080B35000122026001684B1C26
:1032100003600268511C0160134803685A1C026075
:103220004FF48070FEF784FE00B302F0DDFE24E070
:1032300068140020CC100020D8060020D006002002
:1032400083160020CC16002094160020E4060020EF
:10325000D1060020E6060020E8060020D216002055
:10326000C410002000080140DC0600203648002180
:1032700001604FF40050FEF75BFE00F085FF334B1A
:1032800033499A890860334B1AB11968411A0029E9
:1032900059DB84181C6001F0EBFCFFF7A5FB00F084
:1032A00073FF2D4B2A4A19681060441A18602B4886
:1032B0002B4A90F87230148053B12A49CC780CB95B
:1032C0000A792AB12848294BC48819880A19C2806A
:1032D000202003F003FD40B12248C3790BB9017AE5
:1032E00019B1047B0CB103F0F7FB2148214A174BBD
:1032F00000F11E011468B3F8F62000F12903A0477D
:1033000002F014F801F090FFBDE8384001F0E8BF8A
:10331000487800283FF4D5AD01F0F6F9D1E5012356
:1033200002E0022300E00323DDB2084A691E82F8AE
:103330009413FEF79FFDFEF759FD022028212A462F
:1033400006F088FA24E638BDDC060020CC10002008
:10335000C4060020D4060020C806002068140020FF
:10336000E206002083160020AA160020880B002009
:103370006914002044000020014B1880704700BFF2
:10338000EA060020F8B5664B1D88002D40D00023CA
:103390001946B5F5C87F634A01D100205050624EEE
:1033A00050589F5F5F4CC0195050604A002098539E
:1033B0009E1802330431062BA6F8F800E9D1012D3E
:1033C00022D121684FF4C87301F1C80191FBF3F1D8
:1033D000A2F8F8106168C83191FBF3F1A2F8FA1075
:1033E000A168C83191FBF3F3514909885B1A51492F
:1033F000A2F8FC304885888592F89403FEF72AFDF0
:10340000FEF738FDFEF71CFD45480288531E038079
:103410000420FEF78DFD00286FD047490A88322A24
:1034200011D1424D454CB5F8F860B5F8FA00B5F841
:10343000FC30404926806080A3804D8D404C8E8DAD
:103440002580668001E0002A32D000231946322A06
:103450003C4801D100244450334D44585E5FA619C6
:103460004650324800245C531D1802330431062BA9
:103470002646A5F8F840EAD1012A16D1324B334945
:103480001A70334B0C70022119702C4B1988A0F85C
:10349000F81059889B88A0F8FA102949A0F8FC3048
:1034A000244B0888498858859985234B013A1A800E
:1034B0002848017809B30022027022481B4B046897
:1034C000322194FBF1F4A3F8F8404468806894FB3F
:1034D000F1F490FBF1F11648A3F8FA400088091ABC
:1034E0001448A3F8FC104285828593F89403FEF7F4
:1034F000B1FCFEF7BFFCFEF7A3FC0B4B0B4A188890
:10350000B2F8F810401A1880B2F8FA105888B2F8D9
:10351000FC20401A99885880881A9880F8BD00BF0E
:10352000EA060020EC06002098150020CC100020B0
:103530004200002068140020E4060020FA06002063
:103540000C07002000070020E6060020D10600201E
:1035500098060020E806002010B5074B074C596874
:1035600020468847064A204621461278FEF740FA50
:10357000BDE81040FFF706BF441500209815002055
:10358000E9060020014B1880704700BF200700208B
:103590002DE9F84F414B188800286ED000242546AD
:1035A00026463E490A88B2F57A7F08D13C4B3D4910
:1035B00000271420EF5000FB0610FEF75BFEDFF83B
:1035C000F0A0374F3AF90400EA59DFF8D890131801
:1035D000EB51FDF79BFA4FF0140B0BFB069B0146DA
:1035E0004FF000085846FEF748FE24F80A80DFF83E
:1035F000ACA02D48BAF8001024F80080012933D17E
:103600005846FEF77CFE294A834692F8F400E0B162
:10361000FDF77CFA01465846FDF788FCA8B14FF447
:103620007A714846AAF80010FEF724FE09F114004A
:10363000FEF720FE09F12800FEF71CFEC7F80880FF
:10364000C7F80480C7F800800EE0154B4FF47A727B
:10365000E858154B00F5FA7191FBF2F0E0520F219A
:103660000A20012206F0F6F8013604350234032E52
:1036700097D10A480288531E03800D4B0A4A1888C6
:103680001188401A1880518858889288401A998861
:103690005880881A9880BDE8F88F00BF2007002066
:1036A00014070020240700205A0B0020CC10002013
:1036B0008015002010B5074B074C596820468847F5
:1036C000064A204621461278FEF792F9BDE81040DE
:1036D000FFF75EBF5815002080150020220700204C
:1036E00001480249FDF78CBC441500205815002004
:1036F0002DE9F84F9C4C2068838A9BB213F001029D
:1037000039D0018821F400631A04110C01800121D1
:1037100007F0BAF8954A964B117800201870D9B185
:10372000944803781BB9944A1178FF2914D10123D6
:10373000037092480278022A06D18B490B681888D8
:1037400082B242F4006119808D4B87481978006875
:10375000012207F0B3F82FE18948834B017800225A
:10376000186807F0ABF8844A1178FF2900F024812B
:10377000FF207F4BDEE003F00201C9B200293DD0FB
:10378000BFF35F8F7D4D2E78012E354616D17749D8
:103790000B789BB177490B7883B1114607F074F829
:1037A000BFF35F8F20683146038B07F061F8754ADD
:1037B000206816704FF480613246FBE0038BBFF344
:1037C0005F8F6E490A78022A09D1684B1A7832B1A4
:1037D000684B1A781AB1002107F056F8E5E009782D
:1037E000032907D1614B1A7822B162490B78002B6B
:1037F00040F0DD804FF480610122DBE003F004063D
:10380000F6B2002E71D0594BDFF878811A78012674
:1038100088F80060574B002A4DD01A78002A4AD009
:10382000564D2F78524D022F574F29D907F02CF8BB
:10383000206895F80090D7F800A007F03CF84FFA00
:1038400089FB0AF80B0009EB060031462870206856
:1038500007F00EF8206888F800603F6895F800804F
:1038600007F029F84FFA88F907F80900B0442068F2
:103870004FF48061324685F8008007F011F82BE0A4
:10388000314606F0F5FF20682E78D7F8008007F063
:1038900012F84FFA86F9731C08F80900D9B22068AB
:1038A0004FFA81F83F68297007F005F8033607F8EA
:1038B00008002E7010E01B78012113B9334A1378E9
:1038C0002BB106F0D5FF2A480278511C03E006F020
:1038D000C3FF284801210170234A11680B8803F4B3
:1038E000807082B2002AF9D166E003F040010F46F1
:1038F0001F4D09B3244B2F78D3F8008006F0DBFF6F
:103900004FFA87F908F80900781CC1B229701B4DDD
:103910004FB22A780337BA4205D120684FF480614C
:10392000324606F0BDFF124B28781A7851B2884211
:1039300042D1501C18703FE01B063DD52B785EB27B
:10394000721C27D0124901330A682B70915D06F072
:10395000B0FF0A4895F90020017891422CD12068E7
:103960004FF480613A4625E0780700207607002072
:1039700074070020750700206307002064070020FB
:103980007D07002062070020680700206C070020E8
:1039900070070020154A2970117806F08AFF144834
:1039A000017811B9134B1A7832B9134800684FF4F3
:1039B0008061002206F074FF0E4A104B117893F9D3
:1039C00000004A1C90420ED10D4B0E49187800227F
:1039D0000A7028B1084908684FF4407106F060FF8A
:1039E000094B00221A70BDE8F88F00BF6307002062
:1039F0007607002064070020780700207407002065
:103A000062070020750700207C070020FFF770BECA
:103A1000FFF76EBEF0B5484C89B04FF440651C23EB
:103A200007460226204602A9ADF808508DF80A3054
:103A30008DF80B6000F0E6F84048142107608DF81F
:103A40000E10204603A9ADF80C508DF80F6000F061
:103A5000D9F825610825384CA268520503D40A20FC
:103A600000F0B2FBF7E74FF480660A20666100F0D1
:103A7000ABFB6F1E0A20266100F0A6FB17F0FF05C6
:103A8000E9D14FF4006767610A2000F09DFB666191
:103A90000A2000F099FB26610A2000F095FB022025
:103AA00027611C218DF80F002046244C4FF4406301
:103AB0008DF80E1003A9ADF80C3000F0A3F82068C3
:103AC00006F02CFE04A806F0ADFE20682A464FF44E
:103AD000407106F0E5FE1A484FF480434BF6FF7242
:103AE000049001212068ADF81C30ADF81620ADF827
:103AF000145006F0A5FE04A9206806F029FE4FF434
:103B0000A06006F03BF92221012201A88DF80410E3
:103B10008DF805508DF806508DF8072006F038F91D
:103B2000212301A82E468DF804308DF8055006F0AB
:103B30002FF909B0F0BD00BF000C0140780700204C
:103B4000801A0600274B37B51868818A8AB201921D
:103B5000019B13F4706F02D0234A01211170019B65
:103B600013F4E06F31D04FF480610022038B06F034
:103B700097FE0198810528D41A4D2868018801F420
:103B8000007293B20BBB048804F480718CB29CB1B8
:103B9000028802F4807399B20029F9D1012106F05C
:103BA00067FE10480068028802F4007399B2002989
:103BB000F9D1FFF72FFF08E0012106F059FE286830
:103BC0004FF44071224606F06BFE06480268938A65
:103BD00023F470610804030C0449938200220A70E4
:103BE0003EBD00BF780700206D0700207C07002045
:103BF000FFF7A8BFFFF7A6BF014B188880B2704738
:103C0000600700202DE9F0410F88002347FA03F2F6
:103C1000D2072DD58A7803F00705DC08AD0012F035
:103C2000100F18BF91F803C002F00F0618BF46EA44
:103C30000C064FF00F0C0CFA05FC06FA05F550F8CF
:103C40002480282A28EA0C0C45EA0C0540F8245068
:103C500006D1012202FA03F2C46824EA020206E055
:103C6000482A05D1012202FA03F2C4682243C26045
:103C70000133102BCAD1BDE8F08108B503681A687A
:103C8000904708BD38B505460C4614F8011B19B11C
:103C90002846FFF7F2FFF8E738BD08B50368596812
:103CA000884708BD08B503689968884708BD08B506
:103CB0000368DA68904708BD08B503681969884742
:103CC00008BD08B503685A69904708BD7047036B83
:103CD00013B15A68006C01E0026AC069101A18BF7B
:103CE00001207047436B13B190F844007047826A1B
:103CF000406A111A4B4253EB01007047836A816995
:103D0000426BC918D160416A994203D9CB1A5360FA
:103D1000816204E00169CB1A5360002282620021B3
:103D200080F84410406B012106F075BE30B50446A2
:103D3000007985B000230D460091C107ADF804302D
:103D4000ADF80630ADF80830ADF80C30ADF80A30FB
:103D500002D50422ADF80A20820705D5BDF80A1065
:103D600041F00803ADF80A30A06C694606F034FB58
:103D7000A56005B030BD026B034610B5406942B185
:103D80001A6CD9688C1A013A18BF1146005D196483
:103D900010BD196ADA68405C0131B1FBF2F402FB34
:103DA0001411196210BD10B5426A8469A154416AA8
:103DB00002690131B1FBF2F402FB1411426B416262
:103DC00032B11368DB070BD4BDE81040FFF796BF94
:103DD000806C40F227710122BDE8104006F060BB04
:103DE00010BD0000214B13B5986021480C46586166
:103DF0002048214A2149186314381A6099614FF408
:103E00008072586301214FF48040DA601A6106F035
:103E10004DFC4FF4007102231822ADF80010A107E9
:103E20008DF803308DF8022003D515486946FFF759
:103E3000E9FE48234FF48060E207ADF800008DF8FA
:103E4000023003D50E486946FFF7DCFE01220E2141
:103E500001A88DF804108DF805208DF806208DF846
:103E6000072005F095FF01481CBD00BF400A002057
:103E70003E0900205800024008DC0008BE07002070
:103E8000000801401F4B13B51F4A98600C46802064
:103E90004021D86019611D481D491A601D4A98616A
:103EA00099644FF4003001215A6106F00BFC0223A3
:103EB000042218208DF80330A307ADF800208DF8F8
:103EC000020003D514486946FFF79CFE08214823E9
:103ED000E007ADF800108DF8023003D50E486946B2
:103EE000FFF790FE012026228DF8050002218DF8B3
:103EF000070001A88DF804208DF8061005F048FF92
:103F000000481CBD8C0A002008DC00087E07002049
:103F100000440040BE080020000801402DE9F041A7
:103F20001E46584B90B0984205468846174604D125
:103F300010463146FFF756FF07E0534800248542FC
:103F400004D110463146FFF79DFF0446002106F0DC
:103F500004022671A7600197A5642162E161A16254
:103F60006162C4F82C80ADF8081002F0FF0732B18E
:103F70004FF40053ADF80A304FF4806701E0ADF81C
:103F80000A700020ADF80C7016F00107ADF81000B3
:103F900002D1ADF80E7002E00421ADF80E1006F06B
:103FA000020606F0FF082EB1BDF80E2042F008030D
:103FB000ADF80E30284601A906F00EFA0121284678
:103FC00006F062FA05A806F019FD0023281D4FF43B
:103FD0008051802205900E910F9309930B930A92C2
:103FE0000C9317B3206BD0B16269E168079320236B
:103FF0000D930692089106F069FC206B05A906F066
:10400000DDFC206B012106F006FD2846402101223F
:1040100006F060FA206B06F013FD206405E02846E8
:1040200040F22551012206F03BFAB8F1000F24D0EE
:10403000606BE0B1266910210896002607910D9665
:1040400006F044FC606B05A906F0B8FC0122606B29
:10405000022106F0EBFC606B314606F0EFFC606B72
:10406000802146600122284606F034FA05E0284601
:1040700040F22771012206F013FA204610B0BDE885
:10408000F08100BF003801400044004010B50B4CE7
:104090004FF4005006F0D8FC0021606B06F0BBFC2A
:1040A000626AA36A9A4204D02046BDE81040FFF736
:1040B00025BE012084F8440010BD00BF400A002046
:1040C0000D4B986C028802F080018AB29AB19A6A0C
:1040D000596A8A420AD09969895C013281801969DA
:1040E000B2FBF1F001FB10229A62704740F2277197
:1040F000002206F0D5B97047400A00201C4B10B5CD
:104100009A6C1488A4B204F0200188B290B1D96AE4
:1041100019B1938898B288470CE09288D969586998
:10412000D2B24254D869DA68411CB1FBF2F002FB0A
:104130001011D96104F08004A4B2C4B10C4B9A6A86
:10414000586A82420BD09869996C805C01328880F1
:104150001969B2FBF1F001FB10229A6210BD986C54
:1041600040F227710022BDE8104006F099B910BD59
:104170008C0A002070470000024B1A68501C18601F
:10418000704700BFD80A002010B5094A09491368D2
:104190008C6810688342F8D1074A106811684FF4A0
:1041A0007A725043001BB0FBF1F102FB031010BD0B
:1041B000D80A002010E000E0DC0A0020014B18685B
:1041C000704700BFD80A002038B50446FFF7DCFF6F
:1041D0000546FFF7D9FF401BA042FAD338BD10B502
:1041E00004462CB14FF47A70FFF7EEFF013CF8E77C
:1041F00010BD000070B53E4B8AB0054601AC0FCB38
:1042000084E80F00284605F0A5FB0121394806F097
:1042100059FA012144F61D2006F048FA0120014612
:10422000354D06F037FA06F071FA00214FF6FF70AF
:10423000ADF800008DF80210284669462F4EFFF7B2
:10424000E1FC2F486946FFF7DDFC69463046FFF781
:10425000D9FC2C4B5A6842F000705860FFF78AFF77
:104260004FF480514FF40043274A31612B611068AD
:104270002649884206D19DF80A30142B02D110221B
:104280008DF80A20211D0198FFF7BCFC1E481F4B2A
:104290000168994206D19DF81220142A02D11020FB
:1042A0008DF8120004A90398FFF7ACFC05A806F0EE
:1042B000A3F9059B1649174AB3FBF1F016491060A4
:1042C00008684FF47A73B0FBF3F2511E1348144A96
:1042D000F023416082F823300021072381600360CE
:1042E000FDF78CF96420FFF77AFF0AB070BD00BFBC
:1042F0009CDB00080700400000080140001001405E
:10430000000C01400000014084010020001BB700A8
:1043100040420F00DC0A00208801002010E000E08D
:1043200000ED00E010B540F2DB1460430D4B4FF49C
:1043300000424FF480515A61841EC3F81018094896
:10434000C26882F40043C360D0F80C1881F4805234
:10435000C0F80C282046FFF742FF1920FFF73FFF67
:10436000EDE700BF0008014010B1034A034B1A609B
:1043700003480449C8607047EFBEADDEF04F00202F
:104380000400FA0500ED00E02DE9F04F89B0079335
:10439000754B07460692B3F90000B3F902200028D6
:1043A000B8BF4042002AB8BF524200248242B8BF80
:1043B000024605922546A146A0460494A2462646FA
:1043C0006A49CB7813B90A79002A38D0022E36D040
:1043D000674B6548EA5EDDF818B0295E02EB4100E4
:1043E000CBF100015A46FDF73DFF6249DDF81CC0E4
:1043F0006B5E3CF90520C01A8318F879FA7E5843A1
:1044000064214FF0050E90FBF1F06FF00401514371
:104410000EFB02F20393FDF725FFDFF878B1039B53
:10442000824654F80B00544942F210721818FDF7F6
:1044300019FF7A7C44F80B005043011304914B4858
:10444000C3781BB102790AB9022E2FD146495020F8
:1044500035F90180DFF828B100FB08F2BB5DDFF819
:10446000389135F90B0092FBF3F154F809300A1A30
:10447000D01842494FF47A52FDF7F4FE35F90B108B
:1044800049F804000029B8BF4942B1F5207F02DD98
:10449000002049F8040059F80420B9197D23887ACE
:1044A00092FBF3FC00FB0CFE4FEAAE192F4B1A797E
:1044B000B2B1022E14D0DDF814B0DDF810C00BFB41
:1044C00008F0CBF5FA7303FB0A020BFB09F003FBC0
:1044D0000C034FF4FA7192FBF1F293FBF1F308E055
:1044E000D97809B1022E02D14B46424601E0049B25
:1044F00052462349DFF8A4B0695A16F80BC008B237
:104500000CFB00FB6FF04F0C9BFBFCFC94441D4A22
:10451000CDF800C035F902C0A952CCEB00001A4A10
:10452000DFF87CC0019054F80C10A0584018019995
:1045300002904018A15844F80C100199A150134A58
:104540000434B15C202201FB00F090FBF2F1581A18
:10455000009B0F49C21801366A520235032E7FF4C0
:104560002FAF09B0BDE8F08FAA16002083160020F7
:104570003E0D0020440B0020F0D8FFFF80C1FFFF5C
:10458000540B00200C0B0020140B0020731500208E
:104590006A150020F80A0020EC0A00207615002099
:1045A000E00A00202DE9F04F002485B00393054672
:1045B0008946924606462346474AD17809B910797A
:1045C000B8B1022C17D0454B454F33F9140037F9D9
:1045D0001420CAF1000102EB40005246FDF742FEF2
:1045E0004049039F31F9143037F91420C01A831859
:1045F0000AE0022C08D1394A99F80570B2F9041082
:104600001B374F43791114E03348C17871B9334FE8
:1046100099F8042037F914101B324A43007911111C
:1046200038B16A7C5A4301EB222102E0EF795F4303
:1046300039112D4FDFF8C4C037F91400BCF8002041
:104640000F1A295D7A437943DFF8B480D0124FEA1C
:10465000E11B58F82420B17A01FB0020234948F8D7
:1046600024004FF400120293CDF804C0FDF7FAFDC8
:104670001F4BDDF804C053F8241043F82470791A56
:10468000BCF800704FF6FF723B09B2FBF3F74F43E3
:10469000184BDFF870C048F824005CF8241053F879
:1046A0002480BF1108EB010243F82470337DD11937
:1046B00059430BEB6030104A00EB21214CF8248069
:1046C00022F8141001340136032C029B7FF474AFDE
:1046D00005B0BDE8F08F00BF83160020AA160020A9
:1046E0003E0D0020440B0020540B00200000E0FF92
:1046F000000B00202C0B00206A150020E206002091
:10470000EC0A0020200B0020024B5A780AB100204E
:104710005870704783160020024B00221A605A60BE
:10472000704700BFF80A0020024B00221A605A604E
:104730009A607047EC0A00200128034B14BF034A1B
:10474000034A1A60704700BF4400002089430008F4
:10475000A5450008000000002DE9F84F384E04463A
:104760003768384606F07AF90546384606F0EAF921
:1047700076688046304606F071F98346304606F08A
:10478000E1F9D4F80490064629464846FCF712FAA7
:10479000A768824641463846FCF70CFA0146504667
:1047A000FCF7FEF8216882465846FCF703FA4146BA
:1047B00004464846FCF7FEF93146FCF7FBF9014692
:1047C0002046FCF7EFF8314604463846FCF7F2F98C
:1047D0002946FCF7EFF901462046FCF7E3F80146CD
:1047E000504606F03BFA1749FCF7E4F9FBF71EFECA
:1047F00011A3D3E90023FBF797FF134B0446186876
:104800000D46FBF713FE02460B4620462946FBF7F2
:10481000AFFC00220D4BFBF787FFFCF76DF806F0AD
:1048200051F981B20A0444BF00F5B47189B208B2EB
:10483000BDE8F88FAFF30080182D4454FB210940E8
:104840004C0B00200000E1448C0B002000002440B1
:1048500010B5194C2088FCF759F91849FCF7AAF94A
:1048600006F030F9164B18802088FCF74FF9014606
:104870001448FCF753FA1449FCF750FA134908603E
:104880001348B0F87000FCF741F901461148FCF7F5
:1048900045FAFBF7CBFD06A3D3E90023FBF71AFE8D
:1048A000FCF72AF80C4A106010BD00BFAFF300807F
:1048B0003B597E90A9E7814042000020C903683F30
:1048C000480B00200AE81C4100401C4694150020BB
:1048D0006814002000006144B0150020AFF3008090
:1048E0002DE9F041044600680D460146FCF762F9E7
:1048F000D4F80480064641464046FCF75BF9014681
:104900003046FCF74FF8A768064639463846FCF7AC
:1049100051F901463046FCF745F806F0A1F90021AF
:104920000646FCF7DBFA70B920683146FCF7F6F969
:10493000314628606068FCF7F1F931466860A0688C
:10494000FCF7ECF9A860BDE8F0812DE9F04F0C68A8
:10495000836889B0D0F800A0D0F8048006462046CD
:1049600003938B4606F07AF80746204606F0EAF8ED
:10497000DBF804408146204606F070F805462046E4
:1049800006F0E0F8DBF8082004461046019206F035
:1049900065F88346019806F0D5F8394602905846E6
:1049A000FCF708F9394604900298FCF703F95946D8
:1049B00005904846FCF7FEF8029906904846FCF739
:1049C000F9F8294607905846FCF7F4F80146504696
:1049D000FCF7F0F8214683460698FCF7EBF8014611
:1049E0000598FBF7DFFF01464046FCF7E3F8014678
:1049F0005846FBF7D7FF214683460498FCF7DAF8C0
:104A000001460798FBF7CCFF01460398FCF7D2F864
:104A100001465846FBF7C6FF3060029905F1004099
:104A2000FCF7C8F801465046FCF7C4F82146834617
:104A30000798FCF7BFF801460498FBF7B1FF014661
:104A40004046FCF7B7F801465846FBF7ABFF214656
:104A500083460598FCF7AEF801460698FBF7A2FFDF
:104A600001460398FCF7A6F801465846FBF79AFF63
:104A7000214670605046FCF79DF82946044609F12E
:104A80000040FCF797F801464046FCF793F80146D2
:104A90002046FBF787FF394604462846FCF78AF88C
:104AA00001460398FCF786F801462046FBF77AFF9B
:104AB000B06009B0BDE8F08F1FB50B684A6889681F
:104AC0000193039101A90292FFF73FFF05B000BDDA
:104AD00080EAE073A3EBE0738B4206DB002801DD84
:104AE000401A704702D040187047002070470000FD
:104AF0002DE9F041524B86B01A685B6802F1004222
:104B000003F1004301934F4B0646B3F900000092B6
:104B1000FBF7FCFF00F10040FBF788FC46A3D3E95C
:104B20000023FBF7D7FCFBF7E7FE474C0290B4F9F4
:104B30000000FBF7EBFF0390B4F90200FBF7E6FF80
:104B40000490B4F90400FBF7E1FF6946059003A85F
:104B5000FFF7FBFE3D4B93F84030012B16D13C484C
:104B6000417869B93B4C4025226892FBF5F7D01B90
:104B7000FBF7CCFF0599FBF715FFFCF7E1F9206087
:104B8000344B4021186890FBF1F001E0324B18885B
:104B9000FBF7BCFF01460598FBF702FF0590304686
:104BA000FBF7B0FF2D490746FBF7FCFE01463846F0
:104BB000FCF7B4F82A4D07462C6805982146FBF708
:104BC000EFFE01463846FBF7F5FF01462046FBF7AE
:104BD000E9FE244C28601D4D07460398D4F8008058
:104BE00005F070FF95F83010FFF772FF08EB000238
:104BF00004982260D4F8048005F064FF95F8301022
:104C0000FFF766FF08EB000338466360D4F80880BE
:104C100005F058FF95F82F10FFF75AFF1249134B74
:104C20000A684044A0601868B6180E60411C1960FC
:104C300006B0BDE8F08100BF399D52A246DF913F2A
:104C40004C0B00207A150020A815002068140020C5
:104C500083160020780B0020420000203661823C41
:104C6000640B002088150020600B0020740B0020CE
:104C70002DE9F04F87B0FEF71DFD022002F02EF85F
:104C8000002800F0AB81FEF767FCFFF77DFAAC4C23
:104C900005462768C71B3846FBF734FFA949C96892
:104CA000FBF788FF8346A848256090F82E800025F2
:104CB0002C462E46A54A105FFBF728FF5946FBF706
:104CC00079FF03AB5851B8F1000F27D04046FBF7EE
:104CD0001DFF01464FF07E50FCF720F8DFF8AC9244
:104CE000824651464FF07E50FBF75AFE55F80910A8
:104CF000FBF760FF96490346085F0193FBF706FF49
:104D00005146FBF757FF01460198FBF74BFE49F868
:104D10000500FCF715F98F4A105303E08C498D4AC2
:104D2000605AA0528B4B0435E15E0234062C01FB25
:104D30000166BFD1884A6420138846435B43874895
:104D400003A996FBF3F6FFF7B7FE082001F0C6FFB4
:104D500020B1834803A9FFF7AFFE07E0814803A90C
:104D6000FFF7AAFE7F480146FFF7BAFD493E7E499C
:104D7000B4B23B2CB1F8F00007D97B4E0820B6F84E
:104D8000F25001F0ABFF30BB4FE0FBF7BBFE4FF042
:104D90007E518046FBF706FE01464FF07E50FBF742
:104DA000BDFF002406466D4D404655F81410FBF734
:104DB00001FF81466748005FFBF7A8FE01464846B1
:104DC000FBF7F0FD3146FBF7F5FE45F81400023421
:104DD000062CE8D1D1E7B6F8F200FBF793FE804647
:104DE0002846FBF78FFE4FF07E51FBF7DBFD0146B7
:104DF0004FF07E50FBF792FF00240646584D404688
:104E000055F81410FBF7D6FE584A8146105FFBF7A1
:104E10007DFE01464846FBF7C5FD3146FBF7CAFE5D
:104E200045F814000234062CE8D1514B4B4DB3F930
:104E30000000FBF76BFEAC68014620460126FCF73C
:104E400075F800B906464B4968684E73214605F06F
:104E500005FF494CD5F808802060286800F100461D
:104E600068680146FBF7A6FE414605464046FBF74B
:104E7000A1FE01462846FBF795FD05F0F1FE01462F
:104E8000304605F0EBFE60602068FBF7CFFA2AA3FE
:104E9000D3E90023FBF71EFBFBF72EFD05F012FE06
:104EA000364D28806068FBF7C1FA23A3D3E90023BD
:104EB000FBF710FBFBF720FD05F004FE68800820DF
:104EC00001F00CFF2E4C08B1254800E02548FFF703
:104ED00043FC1D4D20803846FFF70AFE95F87220EE
:104EE000002A7FD01D4B18689C6801465F68FBF75D
:104EF00061FE394606463846FBF75CFE0146304601
:104F0000FBF750FD214606462046FBF753FE0146BF
:104F10003046FBF747FD05F0A3FE01462046FBF7B0
:104F2000FDFE18490446FBF7EDFF88B31648002143
:104F3000018057E0AFF300803B597E90A9E78140A4
:104F4000700B0020581500206814002080150020E8
:104F500098150020A815002042000020B41500205C
:104F60007C0B002048000020CC10002050150020B1
:104F7000480B0020831600204C0B0020440B00201F
:104F80007A1500208FC2753C880B0020380B00205A
:104F9000204605F013FE264B1968FBF70BFE05F0C3
:104FA00091FDB0F5617FA8BF4FF46170FBF72CFA5B
:104FB0001DA3D3E90023FBF7B7FBFBF79DFC05F02E
:104FC000C1FD044695F87200FBF7A0FD2146FBF7F2
:104FD000F1FD05F077FD174B188003E0164B1880A4
:104FE00058809880154A5379012B154B07D01548E6
:104FF00019885A889B8801804280838011E0124979
:10500000B3F90420B1F9000002EB4000032290FB49
:10501000F2F080B20B4A088019885B88908011807A
:10502000538007B0BDE8F08FA2EB0FE5DD16964088
:10503000B0150020880B002098150020CC1000200F
:1050400080150020540B00206C0B0020AFF3008073
:1050500010B5054C00202188FCF79CFA61880120DE
:10506000BDE81040FCF796BA540000200A4A02EB53
:10507000C00393F87B10FF2904D019B1074830F81A
:10508000110007E00728DABF02EBC000B0F8780093
:1050900040F2DC5000B2704768140020CC160020AB
:1050A00010B500244FF48040FCF742FF064B10B1CE
:1050B000B3F8DA0001E0B3F8D400044AA052023495
:1050C000182CEFD110BD00BFCC100020D815002047
:1050D000F8B53B4D3B4E6B793B4C06EBC30041783A
:1050E00020202160FCF724FF324608B1012626600B
:1050F0006B79162B1CD10024314E0021A619306982
:10510000FBF7ECFE28B14FF48040FCF711FF50BBD9
:1051100023E02E4B06F110001D190FC885E80F0083
:105120002B4910340A78531CC02C0B70E4D1EAE7E9
:10513000274F12F8336002EBC3003E704768002F20
:10514000E1D00024B442DEDA204D21016D187A1836
:105150000FCA013485E80F00F4E719481D4B417967
:10516000082923D124E01A4E3678012EF5D91A4C9D
:1051700000251034B542F0DA54F8100C4FF07C5191
:10518000FBF718FD4FF07C5144F8100C54F8140C48
:10519000FBF710FD4FF07C5144F8140C54F80C0C44
:1051A000FBF708FD013544F80C0CE2E70E2901D1AC
:1051B000012200E000221A74BDE8F840FFF770BF3A
:1051C000CC10002090DD0008980B0020A00B0020E0
:1051D000940B002083160020A80B0020F0B50023BC
:1051E000461C0E4A002198181033C02B0161F8D1DB
:1051F0000B4F07EBC6035F6807B9F0BD0024084AF0
:1052000012F83600844208DA064D21014D197B1848
:105210000FCB013485E80F00F1E7F0BDCC10002082
:1052200090DD0008DC100020284B10B5186800281D
:105230004AD027494A79531E142B3DD8DFE803F0A2
:105240000B3C3C24403C3C1C3C3C3C3C3C2C3C3C13
:105250003C3C3C242C001F4890F8BB1031B11E4B45
:1052600000205989BDE81040FCF794B91B4A5078DA
:105270000028F4D10146F5E7174C0020E188FCF73F
:1052800089F901202189EDE7134C00202189FCF7E1
:1052900081F901206189E5E70F4C0020E188FCF7E6
:1052A00079F901202189FCF775F902206189FCF761
:1052B00071F90320A189D5E72020FCF739FE18B148
:1052C000BDE81040FFF7C4BE10BD00BF980B002022
:1052D000CC10002068140020540000208316002009
:1052E00010B50024064B1878A04208D9054920467D
:1052F00031F814100134FCF73FF9E4B2F2E710BDC5
:10530000940B0020C0150020064B1A780023D9B258
:10531000914204D2044921F813000133F7E7FFF763
:10532000DFBF00BF940B0020C01500202DE9F84F0F
:10533000B24B187803280FD9B149B24CB1F9042007
:105340006FF06305002AB8BF5242A91AB4F90400ED
:105350006432FCF787FFA080A84A1678012E1DD87A
:10536000A94EAA4C75796A1E142A00F2F981DFE869
:1053700012F0C200F701F7018400D500F701F70130
:105380007101F701F701F701F701F701F100F701EA
:10539000F701F701F701F7015E00C7019B48994B40
:1053A00090F9BA90964FB3F90440C9F10001B7F8EB
:1053B00006A004FB01F95F88B3F80080944C002537
:1053C0001034B542CCD20FFA8AF0FBF79FFB54F8A9
:1053D000101CFBF7EFFB834638B2FBF797FB54F842
:1053E000081CFBF7E7FB01465846FBF7DBFA834650
:1053F0000FFA88F0FBF78AFB54F80C1CFBF7DAFB7A
:1054000001465846FBF7CEFA83464846FBF77EFB3B
:1054100054F8041CFBF7CEFB01465846FBF7C2FAD2
:10542000FBF78EFD7B4B23F815000135C8E794F898
:105430009A20744D12F0010F6B880CBF01264FF0BB
:10544000FF365E43744CB7B204202781FFF70EFE8F
:1054500029886E4D381895F8A230208113F0010F7D
:105460000CBF01224FF0FF324A43052096B26681FD
:10547000FFF7FCFD3718678172E194F89A50614894
:1054800005F002084FFA88F6002E0CBF01214FF0FC
:10549000FF3115F0010F45880CBF01224FF0FF329C
:1054A0006A438688042001FB06F497B2FFF7DEFD0D
:1054B0001FFA84F808EB00035448F91890F8A2701A
:1054C000554C07F0020253B22181002B0CBF012181
:1054D0004FF0FF314E4317F0010F0CBF01204FF08A
:1054E000FF3045430520FFF7C1FDB6B2ADB2371816
:1054F000EA19628134E1434994F8A2408E8814F09D
:10550000010F0CBF01234FF0FF3305205E43FFF76F
:10551000ADFDB5B2404F2818788121E10020FFF79A
:10552000A5FD3E4F94F97A30B7F902603A4D7343C6
:10553000322693FBF6F1401828800120FFF796FDF4
:10554000B7F9002094F98240544394FBF6F3C7184E
:105550006F8005E1324C607820B9B6F8D4202E4B2C
:10556000DA810AE02649B6F8D220B1F90600B6F889
:10557000D010FCF777FE284DE881274E254CF7899F
:105580002780214F97F8190130B3204D0220FFF7F3
:105590006DFDB5F98410B5F98620FCF763FE214B4B
:1055A000B7F812111A880C1A16B220B2864203DA22
:1055B00097F81961B41803E003DD97F81971D41B4B
:1055C0001C8095F98A50B3F9003064226B43124F66
:1055D00093FBF2F00918B980114C0F4DA67A56B121
:1055E000074B1A880324EA802A81988868815988A1
:1055F000A981094D18E0034BF3E700BF940B00208D
:10560000AA1600206A150020CC1000206814002083
:10561000A00B0020C015002054000020440B0020E7
:10562000831600209C0B0020AA4FB5F9062007EB3B
:10563000C40696F97A3064205A4392FBF0F7EF8063
:105640002046FFF713FD01343918E9800235072C95
:10565000EAD185E0A04B5A7822B9B6F8D4709F49B8
:10566000CF810AE09E48B6F8D010B6F8D220B0F943
:105670000600FCF7F7FD994EF081964E974B964A3F
:1056800096F89270974DDC89907A17F0010F2C8074
:105690000CBF01254FF0FF3508B1914900E0924958
:1056A000488807F00204454396F89A60098862B278
:1056B000002A0CBF01274FF0FF3716F0010F0CBF77
:1056C00001244FF0FF3407FB0155604306F002024E
:1056D00057B2DD80002F0CBF01254FF0FF3505FBD1
:1056E000010018810320FFF7C1FC7C4EF388C1182C
:1056F0000420F180FFF7BAFC3489021932812FE0CF
:10570000794F0324BF88734B03EBC40090F87A6091
:10571000C4F1060306F002014DB2002D0CBF0122B8
:105720004FF0FF327A437049580831F8105016F0A4
:10573000010F0CBF01264FF0FF3606FB0522674D17
:1057400096B225F814602046FFF790FC331825F830
:1057500014300134072CD6D1614F6249F888088093
:105760002020FCF7E5FB002841D00020FFF77EFC5D
:105770005A4C054620800120FFF778FC5B4A608088
:10578000137AA3B3534F5A4A97F8BC1001F002069C
:10579000F3B2CBB1B2F9003097F9821097F97A7071
:1057A000B2F9022059437B425343322691FBF6F172
:1057B0006FF0310789B293FBF7F28F187D1993FBD5
:1057C000F6F625808E1910E097F97A10B2F902608A
:1057D00097F982704E43B2F900203221574396FB6D
:1057E000F1F3ED18258097FBF1F680196080414CAC
:1057F000384D04F11006B4F90200B5F97410B5F98A
:105800007620FCF72FFD24F8020F0835B442F2D1C0
:10581000304991F8BC3003F00402D7B22FB93148B7
:10582000354B07881C7801221CE0344D68790E281E
:105830000AD0082808D0324C04EBC0014B78002B6A
:1058400014BF0225002500E0042500242D4F621915
:1058500007EB4401D0B209890134FBF79BFE042C0D
:10586000F4D1DCE7A24209D21E483FB230F912104F
:105870000132B942A8BF0F46BFB2F3E70024A046E9
:105880001D4A1178884567D21C4D3BB2B5F8D2004D
:10589000834204DD134DC21B615B501860534FF40B
:1058A0008040FCF745FB0F4D70B3164B40F2DC51C6
:1058B000B3F90620114B8A42285FC7BFB3F8D8104E
:1058C000B3F8D220B3F8D410B3F8D620FCF7CAFC52
:1058D000285336E06814002083160020540000206E
:1058E000AA160020C01500206A150020941600207A
:1058F000440B002052000020940B0020CC1000200C
:1059000090DD0008CC160020144E285FB6F8D010A9
:10591000B6F8D220FCF7A6FC114BB6F81411B3F977
:10592000062005EB04098A4228530ADA1020FCF706
:10593000FFFA10B9B6F8D00001E0B6F8D400A9F823
:105940000000084A507818B90749084B625AE252D9
:1059500008F10108023493E7BDE8F88FCC1000206D
:10596000CC16002083160020D8150020C01500207A
:10597000024B1868003018BF01207047980B0020B8
:1059800044F25063984203DDA0F50C40A038704704
:1059900003498842BCBF00F50C40A030704700BFEF
:1059A000B0B9FFFF10B5FBF7B1F800210446FBF7D3
:1059B000BDFA08B1204601E004F100400549FBF7BB
:1059C000ADF90549FBF7F6F805F048F8034B186008
:1059D00010BD00BF8096184B35FA8E3C6400002045
:1059E00010B5044C002320702361FEF7E7FB6061D3
:1059F00010BD00BF18160020F8B51D4614460E460F
:105A0000FBF784F86968FBF7D5F83146FBF7D2F865
:105A10002168FAF7C7FF2060FBF792FAED680746A6
:105A200005F10040FBF78CFA06462846FBF788FA9A
:105A3000314602463846FCF715FCFBF767F8206054
:105A4000FBF77EFAF8BD0000F8B5101A0C461F46A9
:105A5000FBF75CF80546381BFBF758F8174B079E19
:105A60001968FBF7A7F8294604462846FBF7A2F871
:105A7000214607462046FBF79DF801463846FAF7CF
:105A800091FF05F0EDF80E49FBF794F8FBF77EFA6D
:105A900006990860214605F1004005F0DFF8094944
:105AA000FBF788F80849FAF77DFFFBF749FA002869
:105AB000BCBF00F50C40A0303060F8BD6400002091
:105AC0002C7D8E3FA00CB34500A00C4610B50446BB
:105AD000002003460D49CA5CA2B12E2A04D101332D
:105AE00094B1C91800220A55084A0A21D25C4843D9
:105AF000A2F13001092901D8303880180E2B02D8C4
:105B00000133E7E710BD002010BD00BF480D0020A5
:105B10002DE9F843224B074648681D68381A0C46A1
:105B20009146FAF7F3FF2946FBF7F8F81D49206183
:105B30000A6880469078FAF7E5FFFAF777FC16A333
:105B4000D3E90023FAF7C6FC02460B4600201649AB
:105B5000FAF7EAFDFAF7D0FE2946FAF723FF0146E5
:105B60002846FBF7DBF8A668054631464046FAF7BB
:105B700017FF01462846FBF71DF801463046FAF7A5
:105B800011FFD9F8081020616760A060FBF712F8D8
:105B9000FBF7D6F9BDE8F883182D4454FB211940D2
:105BA0006C0D0020341600200000F03FAFF30080A1
:105BB000014B1860704700BF34160020F8B52D4B1C
:105BC000187810B1012850D10AE02B4B2B4A587895
:105BD0002B4B02EB001149685868FEF768F841E06A
:105BE000274D6868FEF768F800283ED0224C2178DF
:105BF000264601291ED1FEF7E1FA06466069321AEF
:105C0000632A35D92169042912D81C4F686807EB2B
:105C100001135968FEF74BF8607807EB0017B96875
:105C20006868FEF72FF822696661511C21611CE04B
:105C3000022018E022693AB96478104B686803EBD7
:105C400004114968FEF733F833690B4C8B2B09D8E4
:105C50000C4A0B48D15C4068FEF70FF821694B1CD9
:105C6000236102E00320FFF7BBFE034A00205060DF
:105C7000F8BD00BF3D0D002018160020B0E200085E
:105C80001017002022E2000810B50B4CE37A8BB10C
:105C90000A48017804290DD9094A0A4B106851684D
:105CA00018605960FFF77EFE0748084B0288012103
:105CB0001A80217310BD00BF8316002070160020CB
:105CC000581600203C1600207A1500202A0D0020CE
:105CD000002370B51C460F48002119521420604360
:105CE0000D4A0E4E0E4D995200223250595335181E
:105CF0000C4E6960AA60325035180B4E0134696051
:105D0000AA6002333518022C32506960AA60E2D1D1
:105D100070BD00BF041600203E0D0020DC0C0020EA
:105D20000A1600208C0C00207C0D002070B5044663
:105D30000079FAF7E7FE1E49FAF7F0FF1D4D1E4EF7
:105D40002860A07BFAF7DEFE1949FAF7E7FFEE605C
:105D500068606079FAF7D6FE1849FAF7DFFF184D48
:105D60002860E07BFAF7CEFE1149FAF7D7FF6860AA
:105D7000607EFAF7C7FE1349FAF7D0FFEE60A8601D
:105D8000A079FAF7BFFE0D49FAF7C8FF0E4D28605B
:105D9000207CFAF7B7FE0649FAF7C0FF6860A07EDC
:105DA000FAF7B0FE0749FAF7B9FFEE60A86070BDD8
:105DB0000000C842080D00200000FA440000204105
:105DC0005C0D002000007A44C80C00202DE9F04151
:105DD000134C9846134E144B0546002031701A6040
:105DE000FFF7FEFD6570FEF7E9F9A0603078002747
:105DF0006760B8420CBF012403244046FFF796FFBA
:105E00000A49234601EB05156A6839460848FEF73A
:105E100085F8084A50600120BDE8F041FFF7E0BD79
:105E2000181600203D0D002034160020B0E20008B6
:105E30000044004010170020F8B51B4B18780328C9
:105E40002ED11A494FF480524FF40044A1F5006559
:105E50000A612C61164C6068FDF71FFF60B1134D9D
:105E60004FF480566E6160682768FDF71BFF01469E
:105E70003846FDF702FF2E610D4C2068FDF70DFF3F
:105E80000028E7D00B4D4FF4004694E881006E6186
:105E9000FDF708FF01463846FDF7EFFE2E61D9E712
:105EA0004FF0FF30F8BD00BF181600200010014071
:105EB0001017002000080140F7B50368164C174D75
:105EC00023600968164E61600068FFF76BFD94E877
:105ED0000C0014480196009095E80300FFF7B4FD0C
:105EE0006B68114A61683668C81A1660FAF70EFEC8
:105EF0000E4A0F4F1168FAF75DFEFBF721F829688B
:105F0000786020680B4A431A0B483B6001681660B2
:105F10000A4BCA881A80FEBD300D0020581600209A
:105F2000A80D0020440D00202C0D0020640000204E
:105F3000D00D0020B80D002034160020CA0D00201E
:105F4000264BF0B51D68024600F110011678144684
:105F5000AB195B78013203F00403DBB263B18A4210
:105F6000F4D10020F0BD13B10A225343DBB210F884
:105F7000011B30395B18DBB2211A0229F3DC002146
:105F8000844209D911B10A225143C9B210F8012B38
:105F9000303A8918C9B2F3E72E2E11D1013404200A
:105FA00000220A2672432678AF197F7807F004078B
:105FB000FFB217B1303A921901340138F1D100E043
:105FC0000022074C6420614300FB021106240548AF
:105FD000B1FBF4F200FB0320F0BD00BFA4010020E0
:105FE00040420F00809698002DE9F04F9A4B8BB0FD
:105FF0005868B8B9994C21784A1E032A00F2618585
:10600000DFE812F0F304F3043E0528056068FDF7AD
:1060100049FE934904460B78012B00F0DF8008D33A
:10602000022B06D08C4C6068FDF737FE0028EDD1BE
:10603000E0E7242C07D18B4B8B4A8C4C0021197044
:1060400011702170C5E02C2C02D02A2C40F08280E7
:10605000854D844A2978864B157800205854854A06
:10606000B5B918781570472868D15978502965D185
:106070009878472840F01385D978472940F00F8554
:106080001B79412B40F00B850120107000F007BDFB
:10609000117801293AD1022D05D11846FFF750FF9A
:1060A000754908604AE0032D07D11978532945D175
:1060B000714802685342036040E0042D05D1184640
:1060C000FFF73EFF6C4B586038E0052D07D11B7879
:1060D000572B33D168494A68504248602EE0062D5C
:1060E00007D119786548302994BF00210121C17278
:1060F00024E0072D04D1FFF7E9FC614A10701DE090
:10610000092D1BD1FFF7E2FC5E4B16E0022915D1E9
:10611000072D0CD10120FFF7D9FC41F21842504362
:106120004FF47A71584BB0FBF1F0188006E0082D5F
:1061300004D10120FFF7CAFC544B1880494B4A494F
:10614000013500202A2C1D70087039D150480124D7
:1061500004703EE00D2C4E4A01D00A2C26D1147852
:10616000FCB1434C21786478A1F13000C3B2092B13
:1061700084BFA1F13703DBB2A4F1300003F00F02BA
:10618000C3B21101092B84BFA4F13703DBB2374C32
:1061900003F00F0289182078CBB2C21A514251EB9A
:1061A00002043B4B002018707CB912E02E490B789A
:1061B0000E2B03D82E48C45401330B70127842B909
:1061C0002A4B1A7854401C7003E02A4A10780128A0
:1061D00000D00020C00700F1338123E72D4B0022BF
:1061E000197808293FF61EAFDFE801F00A051119FA
:1061F00027607C96A000622801D1022105E01A7078
:10620000B52C7FF40FAF1C78611C19700AE7224986
:10621000224A03261E7008701070214B0BE01F4E9F
:106220000421197032781E4BA1181878CAB21018C0
:1062300018701C4B32701C70F4E605211970174B56
:10624000174E1A783078A118CAB210183070164E4E
:106250001A703480E6E600BF1017002018160020E0
:106260003D0D0020C20C00203C0D0020D80C002069
:10627000480D0020230D0020581600208316002012
:1062800070160020021600200E160020B40D00200B
:10629000890C0020280D0020BC0D0020200D0020BE
:1062A000210D0020BD0D0020C40C00206C490626E5
:1062B0001E700A786B4BA6181878F2B21018187076
:1062C000694B0A70198801EB0424A6B2B6F5007F69
:1062D00001D81E8003E000221A80644B1A7000244B
:1062E00063497FE35E495F4E0A783078A318DAB2DB
:1062F000101830705E4E0A7033885B4AC72B98BF07
:106300005C49108898BFCC545C1CA1B28842318093
:106310007FF488AE072107E0514808261E700378F5
:10632000A3423FF47FAE0021504B6EE74D4E1A70F2
:10633000337883427FF476AE4F4C207806283BD0EA
:1063400005D8022813D003287FF46CAE23E012286E
:1063500047D030287FF466AE464A484C1679454A05
:10636000102E88BF102626702178002347E0414C6C
:10637000434E6368A06821697360424B4FF47A72A0
:106380003060414C91FBF2F6187840492680C87283
:1063900001223F4923E037494A7912F0010004D035
:1063A0000E79F41E634253EB04003649087000284E
:1063B00039D1364AD07236E02E4EF47A14F001010B
:1063C00004D0B07AC21E534253EB02012D4E3170FD
:1063D00009B92E4CE17227482E4990F82F200A70F7
:1063E00021E024482C498669426942F210742B4B03
:1063F00096FBF4F00A80188001222949EFE70C325D
:106400008B4210DA12F8046C264812F8034C1E5422
:10641000254E26489C5512F8014C16781C54244CE5
:106420001E550133EBE71A490A78002A3FF4FAAD0A
:106430001B4B1E78002E3FF4F5AD00240C701C7031
:106440001C4CA068E060FDF7B9FEA060202000F0C1
:106450004FFC19490A78012A30D100232FE000BFF0
:10646000200D0020210D0020C40C0020280D00204C
:10647000040D0020DC0D0020BD0D00207116002051
:1064800058160020C80D0020021600208316002098
:10649000220D0020701600200E160020B40D0020E2
:1064A000BE0D0020F11500204616002060160020C9
:1064B0007216002018160020CC0D002001237E4CFF
:1064C0000B70E07A00283FF4ADAD7C490A78042ACD
:1064D0007FF6A8AD677807B92773257B15B90FB18B
:1064E000FFF7D2FB764E05213378764F5C1C94FB88
:1064F000F1F001FB10423270734E97F800C0734DFB
:1065000006EB82020023724C72491F59DFF810E239
:106510007148724E5F5097FBFEF1195006FB0170F7
:10652000DFF8009203EB040A42F2107490FBF4F7D8
:106530001668BCB253F809701060C6EB07084044F7
:10654000052643F8090090FBF6F00EFB01016448B4
:10655000BCF1010F25F8024F195005D1023CB4F5EA
:10656000797F98BFCAF8001004331432082BCAD1BF
:10657000FDF724FE5B4D5C4C2A68801AFAF7C2FADC
:106580005A49FAF7CBFB2060FDF718FE2860256812
:106590004FF07E512846FAF7ABFC08B94FF07E5514
:1065A000256006A907AC4A48514B0194009103C8E5
:1065B0000CCBFFF749FA069A64234E49B2FBF3F07D
:1065C0000880079A3C4892FBF3F34B4C027B2380F4
:1065D0000AB90A80228049490C78002C36D0424FF3
:1065E0004FF07E503968FAF799FB454D384E2B68CD
:1065F00004463068C01AFAF789FA2146FAF7DAFA3F
:10660000FAF79EFC726869683E4D0746501AFAF721
:106610007DFA2968FAF7CEFA2146FAF7CBFAFAF7AB
:106620008FFC04B238480225B0F902303FB2E218BC
:1066300092FBF5F1B0F900208BB2B918334C91FB05
:10664000F5F291B263802180438001802B4B0120C1
:106650001F4C1870184B6168294A20681C7A5160D9
:1066600010601CB9DA79002A3FF4DCAC284E294DC1
:10667000294C01960095164F94E80C00FFF7E4F9B9
:1066800061687868254E081AFAF740FA1D4B1968B8
:10669000FAF790FAFAF754FC70600A48226890F909
:1066A00000303C68012BC4EB020131603CD0022B6E
:1066B0007FF4B8AC9FE000BF831600207016002066
:1066C000D80D0020880C0020600C0020560D002002
:1066D00058160020C00D0020700D0020806967FF53
:1066E000B80C0020380D00206C0D002000007A440A
:1066F0003C1600203816002044160020C90D00204A
:10670000180D002064000020240D0020780D0020CA
:10671000A80D0020440D0020300D0020D00D0020D9
:1067200080969800AC0D0020002634463546DFF8F0
:1067300018C3AF4F5CF825B0CDF80CC05846FAF737
:10674000E5F93968FAF736FAFAF7FAFBDFF8DC927E
:10675000A84934F80920DFF8DC82801A83B21FB21E
:10676000635238460497A44FFAF7D0F93968FAF71C
:1067700021FAFAF7E5FB4FF0140A0AFB058A82B208
:106780009E4B0498196805923B4658445246FFF7C1
:1067900033F90599DFF8B4B2DDF80CC00A1824F813
:1067A0000B205CF8250051463A46FFF7B1F99449B1
:1067B0004FF4FA62FBF756FD34F8093034F80B2039
:1067C000313399B2622998BF0020801883B224F82F
:1067D0000B308C4940F6B83218B2FBF743FD58F83D
:1067E0000610894A01352BF80400B15002341436E2
:1067F000022D9CD116E4854F2D683E686C08B6F9D1
:106800000820A24228BF2246814C97B2268839B27E
:1068100030B2814209DD794B7E491868FAF7CAF92E
:10682000FAF78EFB8719BFB227807B4A7B4E14682C
:106830003168661A3046FFF7A3F80028D8BF4042F7
:1068400041F293139842CCBF0020012050B3304650
:10685000FAF75CF97249FAF7ADF904F073F90646F4
:106860002846FAF74FF901463046FAF7A3F9FAF746
:1068700067FB6C4A6349108000B240F6B832FBF700
:10688000F1FC201848F6A044A04203DDA0F50C401E
:10689000A03804E00028BCBF00F50C40A0306249DD
:1068A000086001E0604D2C605F4B1D68C5F50C5021
:1068B0002830FAF72BF95A49FAF77CF9064604F022
:1068C000CDF80990304604F03DF9002508902C469B
:1068D0002E4638B2FAF71AF908AA52F82610FAF733
:1068E00069F980465148DFF80C91005FFAF70EF91C
:1068F00001464046FAF754F8FAF722FB4FF47A7251
:1069000024F809004A4900B2FBF7ACFC81B20BB293
:10691000DFF83C8124F8091018460493FAF7F6F8DA
:10692000D8F80010FAF746F9FAF70AFBDFF8D8A012
:106930004FF0140B0BFB06AB049A30491FFA80FC96
:106940000968434610465A46CDF80CC0FFF754F884
:1069500042460346594639F904000493FFF7D8F834
:10696000049ADDF80C80801808EB000CDFF8DC805E
:106970001FFA8CF124F8081008B240F6B832214909
:10698000FBF770FC55F80A202A4B013628F8040062
:10699000EA5002341435022E9BD11C480368197941
:1069A00031B1214A64201468234A94FBF0F111802C
:1069B000224C1B88206898420ED91749174B0A6849
:1069C0001C68101BFEF7DCFF42F210710028B8BFF4
:1069D000404288427FF726AB194B1A4A01201C8897
:1069E000154910700C80FFF71DBBFFF7E7F868E052
:1069F000080D0020B40C00205C0D00206C0D002060
:106A000030F8FFFF48F4FFFF7C0D00203416002013
:106A1000CA0D00200000C842A80D0020B80D0020BB
:106A2000D3023739C00C00202C0D0020780D002037
:106A300018FCFFFF8C0C002068150020440D00207E
:106A40002A0D0020880C0020D00D00200A160020FE
:106A5000C80C002062686078531C411CCAB2636095
:106A60000523B2FBF3F003FB10216170FDF7A6FBD9
:106A7000154AA06015480023C372137001200BE073
:106A8000FDF79CFBA36840F6C411C01A884218D9D0
:106A9000202000F035F90420FEF7A2FF11E00C4998
:106AA0008A78522A7FF44AABCB784D2B7FF446ABE1
:106AB000087943287FF442AB064A02211170FFF7A0
:106AC0003DBB0BB0BDE8F08F701600208316002090
:106AD000480D0020230D00203D4B2DE9F047B3F970
:106AE0000000FAF713F83B49FAF764F8044604F09B
:106AF00029F80646204603F0B1FFDFF8EC90054682
:106B0000D9F80000344F90F80380B8F1000F2BD073
:106B1000324CB7F90210B4F802A00FFA8AF2881AC0
:106B2000FEF72EFFC8F100014246FBF79BFBB4F8CD
:106B3000008000EB0A03B7F900000FFA88F7C01BCA
:106B40006380FEF71DFFD9F80010CA785142FBF7A9
:106B500089FB00EB080297B22780B4F90200F9F72D
:106B6000D5FF804638B206E0B7F90200F9F7CEFF4C
:106B70008046B7F90000F9F7C9FF294607464046A5
:106B8000FAF718F8314681463846FAF713F8014605
:106B90004846F9F705FF1249FAF7C0F8FAF7D0F9B5
:106BA000104C314620804046FAF704F82946064644
:106BB0003846F9F7FFFF01463046F9F7F3FE08497A
:106BC000FAF7ACF8FAF7BCF96080BDE8F08700BFCF
:106BD0007A15002035FA8E3C0A1600200416002093
:106BE000000020413E0D00203416002038B5254C11
:106BF000E37A2246002B3ED02348017804293AD973
:106C00002248817A79B1E179002939D12048214B94
:106C1000012221721970011DE271FFF74DF91E4921
:106C20000220087038BDC37AE171C3B11B4A1068F5
:106C3000408900F073F890B1237A002B20D11548D9
:106C40001749037017480A684B680125011D026047
:106C500043602572FFF730F90F48057038BD0D48C5
:106C6000084B02780021197252B901210170BDE868
:106C70003840FFF72DB80023D3711372064A137002
:106C800038BD00BF83160020701600209416002027
:106C90003C16002068000020880C002034160020DC
:106CA0005816002010160020094B1A68811A002976
:106CB0000DDB084A1178042909D900F5123000F5D6
:106CC000F8721A60044BD96881F40040D8607047AC
:106CD000A40D00207016002000080140034B196825
:106CE00008420CBF00200120704700BFA40E002006
:106CF000024B1A6810431860704700BFA40E0020B2
:106D0000024B1A6822EA000018607047A40E0020A7
:106D1000014B1868704700BFA40E0020094BB3F95F
:106D20000020002AB8BF5242824209DAB3F90210A9
:106D30000029B8BF49428142ACBF00200120704702
:106D400000207047AA160020037A0A46032B0FD8AA
:106D5000DFE803F00202060A0649074B00F0ECBA2E
:106D60000449054B00F040B90249034B00F00ABA50
:106D7000704700BFB2160020E80E002038B5044668
:106D80000D46002361890B4A99520233242BF9D115
:106D90000820FBF7CDF828B120462946BDE8384049
:106DA000FFF7D2BF0448054A2946BDE8384000F045
:106DB000D9B800BFCC160020B2160020E80E002083
:106DC0002DE9F843074608208846FBF7B1F870B173
:106DD0000024224A414613683846E2B298472049C7
:106DE00021F814000134082CF3D1BDE8F8831D4AC2
:106DF0001D4D1378591CCCB204F00306147005EB3A
:106E00004609044606461548414603683246384658
:106E1000984729F824002A886988AB885018EA889E
:106E2000C118881803B2991C042291FBF2F00C4A95
:106E30000E4BA15EE052CB1E984201DA811CA1529A
:106E4000135FD91C884201DD023810530136F6B2B7
:106E500002340835082ED6D1BDE8F883E80E0020AC
:106E6000CC160020EC0E0020A80E0020EE0E002014
:106E700010B544780078002303FB03F1193961430E
:106E800001F6C4115943414340F6C41291FBF2F19B
:106E9000034A22F813100133072BEDD110BD00BFB8
:106EA000F01600202DE9F04F85784FF00A0C0CFB0E
:106EB00005FCC778C5F164086E425FFA88F8C7F12F
:106EC0006409B6B2002330B2002804DCB8BF2C46F7
:106ED00002DB012400E0444600FB00FB64430BFBA3
:106EE00007FB9BFBF4F44C4444434FF00A0B94FB28
:106EF000FBF00CEB000420B2C1EB020A00FB0AF429
:106F00004FF47A7094FBF0F404480C191C520233CD
:106F10005E44182BB6B2D6D1BDE8F08FB41600206F
:106F2000F8B505460F46441E14F8011F49B1054E39
:106F3000304605F0EFFE0028F6D0861B631BBB55DC
:106F4000F2E7F8BD00E3000810B50446805CFAF7EC
:106F500023FBA0F2EE2291B240F2DC53994288BFAB
:106F6000608910BD024B082113600170704700BF9B
:106F7000496F0008825C044B53F82200410801F578
:106F8000777290B2704700BF000F002038B50446FA
:106F9000FDF7FAF8104B40F6C4111A68821A8A42BB
:106FA0001A460E4B01D9002119701B7810600BB9DD
:106FB0000F2C10D10A4800210170084A4BB1094D2D
:106FC000182B1D4405F8014C03D1012303701170E7
:106FD00038BD0133137038BD200F00203D0F002055
:106FE000FE0E0020240F002038B540891C460E4BB1
:106FF0000D461A60A0F577710C4A4B001360536080
:107000009360D360136153619361D3610849094868
:10701000094A0523FCF782FF0849C8600CB10848FB
:10702000206008232B7038BDC4100020000F002002
:107030008D6F000800440040A0860100101700205A
:10704000756F000870B5294D287800284CD0284C61
:10705000A67DC6F3C006002E44D1264B18680168F1
:107060000A68904761782278234B01F0070042EAD2
:1070700000221A60A2782E7002F03F00400140EA20
:10708000D1015960E078810041EA9211227902F041
:10709000010041EA80219960617901F00F00C0018F
:1070A00040EA5202DA60A27902F07F00000140EA71
:1070B00011111961E079410041EAD212217A01F0FF
:1070C000030042EA40225A61627A02F01F00800106
:1070D00040EA91019961A07AC10041EA5212DA6155
:1070E000012070BD0020287070BD00BFFE0E002082
:1070F000240F0020C4100020000F0020825C034BEE
:1071000053F82200C0F3CF00704700BF600F00208B
:1071100010B50446FDF738F8154B1A68811AB1F519
:107120007A6F1A46134B01D9002119701060187834
:1071300020B9A82C1AD1104B187006E0022802D1F1
:107140000E4A147001E0142801D80D490C540B4963
:107150000130C3B20878074A4100481D83421370CA
:1071600004D100230449137001220A7010BD00BF2E
:10717000580F00203E0F0020540F00205C0F00200D
:107180003F0F002038B51C46084B0D461A600849D1
:1071900008484FF4E1320123FCF7C0FE0649C860FD
:1071A0000CB10648206008222A7038BDC4100020A7
:1071B000117100080044004010170020FD70000805
:1071C000154B10B51A780AB9002010BD13490020DC
:1071D00018704B78012BF7D1114A106801680B68C1
:1071E000984710480278082A01D9082101700178CF
:1071F0000D4A0023D8B2023288420AD212F8010C9A
:1072000012F8024C40EA0424084840F823400133B5
:10721000F0E7012010BD00BF540F00203F0F0020F9
:10722000C41000205C0F0020420F0020600F0020DF
:107230001F4B2DE9F0431B7823B31E4C1E4D2778BE
:1072400091F800C095F8008002231C4C03F101095D
:10725000E65C46FA07F606F00F05EEB266450BD27D
:107260000B2E09D8E65C14F8094006EA080604EB80
:107270000626134C44F825600233102BE5D10C4B45
:1072800000241C700978914202D90E4B197811B96B
:107290004089BDE8F0830C4B825C1978084B53F8A9
:1072A000220001B1400800F5777188B2BDE8F08393
:1072B000810F0020800F00208A0F0020FE16002082
:1072C000900F0020880F0020890F0020134B01220F
:1072D00010B51A700446FCF757FF114A01461068B2
:1072E00011600B1A0F4841F288318B4203600E4B3C
:1072F00001D900221A7018780C49E4B20F280C54F6
:1073000008D10B4B0B491A680120087010680168FE
:10731000884710BD044A431C137010BD880F00201D
:10732000840F00208C0F00208B0F0020FE16002001
:10733000C4100020810F002010B51C46134B1A60AA
:10734000027A5AB1012A13D1114B03201870114B44
:1073500007201870104802700C2208E00C4B022025
:1073600018700C4B032018700B48027007220A702B
:107370000A490B484FF4E1320123FCF7CFFD0949DC
:10738000C8600CB1084B236010BD00BFC4100020C2
:10739000800F00208A0F0020890F0020CD72000886
:1073A000004400401017002031720008014B18788B
:1073B000704700BF810F002008B54FF40060FAF756
:1073C000B7FD08B9002008BD4020FAF7B1FD094B10
:1073D00020B993F82D21501E0128F3D993F82C01E0
:1073E000012805D1034991F82D31002BEAD008BDC1
:1073F000012008BDCC100020084B93F82D215AB96C
:1074000093F82E0110B9064A537801E005490B7D27
:10741000181C18BF0120704701207047CC100020B5
:10742000831600209416002010B5084B93F82C21E9
:107430001C460AB900F0A0F894F82C01012803D1E9
:10744000BDE8104000F056BA10BD00BFCC100020BF
:1074500038B50E4B1878C0B1FFF7CEFF0C49044683
:107460000A78824211D060B10A4D95F82C310BB9DF
:1074700000F08CF895F82C01012804D100F032FAC4
:1074800001E0FFF7D1FF02490C7038BDC10F0020A9
:10749000C00F0020CC10002010B504464020FAF7A1
:1074A00047FD074B002283F82D212068A060FFF7DD
:1074B00083FF04490870BDE81040FFF7C9BF00BF53
:1074C000CC100020C10F00200B4B10B5187888B1EC
:1074D000FFF792FF70B1094991F82C210C460AB9C7
:1074E00000F06CF894F82C31012B03D1BDE810406A
:1074F00000F008BA10BD00BFC10F0020CC10002062
:1075000038B5064C05465E21A068FCF7B6FBA068BE
:107510002946BDE83840FCF7B0BB00BF101700207B
:10752000024B5E219868FCF7A8BB00BF1017002033
:1075300010B50A4C5E280146A06805D15D21FCF714
:107540009CFBA0683E2105E05D2903D1FCF795FB7B
:10755000A0683D21BDE81040FCF78FBB101700204C
:1075600010B50446C0B2FFF7E3FFC4F30720BDE83F
:107570001040FFF7DDBF0000034B93F82D0108B961
:1075800000F092BA704700BFCC100020044B93F873
:107590002D0118B94FF4165000F078BA704700BFAB
:1075A000CC10002008B5044B9868FCF776FBD0F1AE
:1075B000010038BF002008BD101700202DE9F04160
:1075C000FFF7F0FF002800F04081FCF7F7FDA04B2B
:1075D0001A68811A7C2940F2388118609D48047825
:1075E000651C0570002404F12406F0B2FFF788FF43
:1075F000994B33F91400F9F789FA984A054610882F
:10760000F9F784FA01462846F9F788FB9449F9F717
:10761000D1FAF9F795FC013400B2FFF7A1FF032C72
:10762000E1D13020FFF76CFF8E49B1F90000FFF780
:1076300097FFFFF775FF8748067816F0030629D1F4
:10764000894D1020FFF75CFF2B68642493FBF4F254
:1076500010B2FFF785FF2120FFF752FF296891FB49
:10766000F4F004FB101484EAE473A3EBE47318B29F
:10767000FFF776FF1420FFF743FF7C4AB2F90000C2
:10768000FFF76EFF1C20FFF73BFF3046FFF768FF58
:10769000FFF746FF6F490878430740F0B080744D0C
:1076A0000220FFF72DFFB5F900300A2593FBF5F016
:1076B000FFF756FF0220FAF73BFC002847D06D4F3A
:1076C0006D4E3878347840F63401B4FBF0F26B4CF0
:1076D0004A4321882A2391FBF0F800FB1810B2FBE3
:1076E000F3F24FEA001399B241EA022C1FFA8CFE22
:1076F000C2F303224EEA02080620FFF701FF0FFA49
:1077000088F0FFF72DFF20883F78431C9AB292FB48
:10771000F7F107FB1120367820806E24744315237F
:1077200094FBF3F43A206427FFF7EAFEB4FBF7F684
:107730003046FFF715FF3B20FFF7E2FE07FB16423E
:1077400091B24C1D94FBF5F000B2FFF709FF202029
:10775000FFF7C4FA002850D0494C1320FFF7D0FEA1
:107760002568484F002DB8BF6D4295FBF7F630B243
:10777000FFF7F6FE1B20FFF7C3FE23680A26002B47
:10778000B8BF5B4293FBF6F142F2107591FBF5F244
:1077900005FB121000B2FFF7E3FE2320FFF7B0FE57
:1077A0002368002BACBF4E205320FFF7D9FE1220D8
:1077B000FFF7A6FE61680029B8BF494291FBF7F2C6
:1077C00010B2FFF7CDFE1A20FFF79AFE606800287E
:1077D000B8BF404290FBF6F696FBF5F305FB13614C
:1077E00008B2FFF7BDFE2220FFF78AFE6268002A7A
:1077F000ACBF45205720FFF7B3FEFFF791FE1548B9
:107800000378282B21D100240470FCF7D7FC4FF417
:107810007A753C24B0FBF5F61720FFF771FEB6FB36
:10782000F4F5B5FBF4F104FB1152100200B2FFF7BE
:1078300097FE1820FFF764FE04FB156318B2FFF7EC
:107840008FFEBDE8F041FFF76BBEBDE8F08100BFE1
:10785000C80F0020C20F0020A81500204200002001
:1078600000007A44900B0020680B00207A1500205D
:107870003615002040000020C8100020C40F002052
:1078800058160020A0860100154B2DE9F0418046D6
:107890000F4698680221FCF714FA00242646781E49
:1078A00084420F4D0DDA18F80410A8688E190134BF
:1078B000FCF7E3F94FF47A70B6B2FCF785FCE4B25A
:1078C000EDE7F1B2A868FCF7D8F94FF47A70FCF74D
:1078D0007BFCA8680121BDE8F041FCF7F2B900BFCC
:1078E00010170020024B01219868FCF7EAB900BF8D
:1078F00010170020024B03219868FCF7E2B900BF83
:1079000010170020F8B5544CA068FCF7C6F9002801
:1079100000F0A080A068FCF7C5F905460520FCF73B
:107920005EFC8A2D21D08E2DEDD14C4C00212E22D3
:10793000204605F033F94A4A7C2323701378E0206F
:107940007D21E07084F82C1014204FF4FA71A37795
:10795000237548227823207660766183657062847F
:1079600084F8243020462E2171E02020FFF7B6F95C
:107970000028C8D03B4C00212C22204605F00EF9EF
:10798000A021E170384B39497C207D22207084F899
:107990002B201878CA7A6570A076002A52D0344914
:1079A00034480F686625FE0F97FBF0FC6672324E76
:1079B0005FFA8CFC06FB0C7284F8295006256A439A
:1079C00042F21073B2FBF3FE03FB1E2749682773D4
:1079D00091FBF0F03F0AC0B26773CF0F06FB0011B6
:1079E0006943B1FBF3F5642203FB1513E9B202FB13
:1079F0000010010AE0732148217401885FFA8EFEAD
:107A000063741B0A02FB0CECA374B1FBF2F2242397
:107A10005A4390B21A4A010A1388E0712172180A77
:107A20001849207518480A8801884FEA1C2EE3740B
:107A3000130A84F80AC084F80BE0A7736275A37573
:107A4000217702E0202384F8293006482C21FFF713
:107A50001BFF58E7F8BD00BF10170020F80F0020EB
:107A6000C8100020CC0F00207016002083160020C4
:107A700058160020A08601006079FEFF0E16002037
:107A800038160020021600204416002008B50246D1
:107A9000032303480021FCF741FA024B186008BD9C
:107AA0000038014010170020024B18680068FFF7EB
:107AB000EDBF00BF2810002008B5044B1860FFF789
:107AC000F3FFBDE8084001F0EFB800BF2810002028
:107AD000034B187808B100F0F1BE01F05FB900BFA8
:107AE0002C100020232801D100F0E8BE044B1968B7
:107AF0008A7A824202D10120FCF736BC704700BF6F
:107B00002810002070B50646B6FBF2F4084615466C
:107B100014B12046FFF7F6FF05FB1464024B195D14
:107B200000F8011B70BD00BF84E400082DE9F0419E
:107B3000027803460130202AFAD0092AF8D02D2AEB
:107B400002D10346414D04E02B2A08BF03464FF003
:107B50007E551E460024334616F8010BA0F130076F
:107B6000F9B209290DD83A492046F9F723F8044615
:107B70003846F8F7CBFF01462046F8F713FF0446D6
:107B8000E9E72E2817D1324F334616F8010B30386B
:107B9000C2B2092A0FD8F8F7B9FF3946F9F7BEF88B
:107BA00001462046F8F7FEFE294904463846F9F713
:107BB00001F80746E8E71878652801D0452839D14B
:107BC0005E782D2E02D19F1C012605E02B2E01D0C0
:107BD0005F1C00E09F1C00267B1E002713F8012F6E
:107BE000303AD1B2092903D80A2000FB0727F5E76C
:107BF000B7F59A7F28BF4FF49A77B8464FF07E5179
:107C0000B8F1070F07D908461249F8F7D3FFA8F1D2
:107C100008080146F4E707F0070737B108460C49A2
:107C2000F8F7C8FF013F0146F7E72EB12046F9F704
:107C300075F804E04FF07E512046F8F7BBFF01468F
:107C40002846F8F7B7FFBDE8F08100BF000080BF0D
:107C50000000204120BCBE4C10B5441E14F8011F8A
:107C600021B1034B1868FCF708F8F7E710BD00BF17
:107C7000101700200148FFF7EFBF00BFA9E400087C
:107C800010B50748FFF7E8FF0024064B06481A190D
:107C9000E15852680C34FAF715FCC02CF5D110BD30
:107CA000D7E40008A8E30008EDE4000870B5FCF78D
:107CB00085FA244C244B4FF47A71B0FBF1F11A7819
:107CC00022482378FAF7FEFBFFF722F80546204802
:107CD000204902682048B2FBF1F1FAF7F3FB0024D7
:107CE0001E4B53F8241051B1012000FA04F0284231
:107CF00002D01B48FAF7E6FB0134E4B2F0E70220B9
:107D0000FEF7ECFF68B1174A174B1178174853F884
:107D10002110FAF7D7FB1648017A11B11548FAF786
:107D2000D1FB154C1548FFF797FF2488FBF764FF3C
:107D30000246134821464FF46673BDE87040FAF7D7
:107D4000C1BB00BF40000020C8100020F5E40008BF
:107D50008801002040420F0033E50008C8F2000807
:107D600051E50008F806002068E4000855E5000821
:107D7000441500205FE50008E206002012E8000834
:107D800063E5000838B50C680546204605F09EF806
:107D9000024628682146BDE8384005F0C7B8000013
:107DA00008B50548FFF758FF0A20FCF718FA00202D
:107DB000BDE80840FCF7D8BA95E5000808B50748C3
:107DC000FFF74AFF064B93F89403FAF743F8FAF7E4
:107DD00051F8BDE80840FFF7E3BF00BFA4E5000885
:107DE000CC1000207FB5044605F070F8082825D196
:107DF00000231F49E25C086885186E7806F00301CD
:107E0000022908BF203AE2540133082BF1D10025A2
:107E1000665D1848314604F07DFF28B101356019D0
:107E2000314604F077FF18B11348FFF715FF1DE046
:107E3000082DEDD120461149FFF772F81048FFF7E1
:107E40000BFF00230F4A04A9981890F808218818FE
:107E5000084A995C0133082B00F80C1CF2D1002071
:107E60008DF80C0001A90848FAF72CFB7FBD00BF74
:107E7000A401002000E30008AEE50008D4110020B2
:107E8000CEE50008CC100020F0E4000808B5FDF7AE
:107E9000D3FF01300CBF03480348BDE80840FFF79B
:107EA000DBBE00BFE3E5000809E600082DE9F0416C
:107EB000054605F00BF80446FAF7CEF9064694B9E4
:107EC0002A48FFF7C9FE2A4951F8241049B1012276
:107ED00002FA04F2324202D02648FAF7F3FA0134E9
:107EE000F1E7254821E028462449224605F01EF8FE
:107EF00058B92348FFF7B0FE224C54F8041F00295C
:107F0000EFD01C48FAF7DEFAF7E72B782D2B04D1D7
:107F10000135013C4FF0010801E04FF00008002658
:107F2000134850F8267027B91748BDE8F041FFF70D
:107F300093BE28463946224604F0F8FFA0B9012036
:107F400000FA06F0B8F1000F03D0FAF77DF90F48F8
:107F500002E0F9F7F7FF0E48FFF77EFE0D483946BD
:107F6000BDE8F041FAF7AEBA0136D9E727E60008D6
:107F70000CE3000851E5000812E80008D2F0000800
:107F80003AE6000808E300084FE6000869E6000842
:107F900073E60008F0E4000810B504460848FFF74F
:107FA0005BFE084A084809490023036013700B7000
:107FB000FDF776F82046BDE81040FFF7FFBE00BF92
:107FC0007CE600082D100020601000202C100020FE
:107FD00008B50448FFF740FEF9F7BCFFBDE80840CC
:107FE000FFF7DEBE94E60008F8B5074604F06EFF22
:107FF000044638B91A491B4B4A791B48511E53F89D
:10800000211028E038461949224604F08FFF60B954
:108010001748FFF721FE174C54F8041F19B11648F2
:10802000FAF750FAF8E7154805E000250D4B53F82C
:10803000256026B91248BDE8F840FFF70DBE384666
:108040003146224604F072FF01350028EED1044883
:10805000314645710B48BDE8F840FAF733BA00BF26
:10806000CC1000204CE30008ADE60008D2F0000878
:10807000C1E6000848E3000851E5000812E80008DE
:10808000D4E60008ECE6000810B50446204604F0EB
:108090001DFF10F0FF0F07D10B490C4891F8941306
:1080A000BDE81040FAF70EBA204604F02DFC022875
:1080B00008D8054B064C83F89403F9F7DBFEF9F773
:1080C00095FEE3E710BD00BFCC100020FEE60008DF
:1080D00022EA000870B5044604F0F8FE08B920480A
:1080E00030E020461F4905F069FB0024264625465E
:1080F00078B12CB1012C06D104F006FC064602E052
:1081000004F002FC054600201649013405F056FB38
:10811000EEE70B2D05D914480C21BDE87040FAF7A5
:10812000D1B9012C08DC114A114832F91520294631
:10813000BDE87040FAF7C6B9A6F57A73B3F57A7F51
:1081400004D90C48BDE87040FAF7BCB90A48294682
:108150003246FAF7B7F9054820F8156070BD00BF40
:1081600014E70008ECE900084EE70008D8150020E5
:1081700074E700088CE70008AEE7000838B505464C
:1081800004F0A4FEC0B268B904461249124801EBDB
:108190004402B2F8422021460134FAF793F9152C33
:1081A000F3D138BD284604F0AFFB142804460BDC9D
:1081B0002021284604F0AEFD04F0A6FB054B03EB9E
:1081C0004404A4F8420038BD04481521BDE83840F5
:1081D000FAF778B968140020C7E70008D3E7000869
:1081E000931E222B88BF0A22031E10B50C4603DA09
:1081F0002D2001F8010B5842FFF784FC002101708B
:10820000204610BD30B587B005460C4603A80021B6
:108210000C2204F0C3FC28460021F8F787FE20B1A9
:1082200028462949F8F7BEFB03E028462649F8F717
:10823000B7FB2649F8F7BEFCF8F782FE054685EA4B
:10824000E570A0EBE5700A226946FFF7C9FF002D33
:1082500001DB202300E02D2368468DF80C3004F06C
:1082600035FE012807D130228DF80D208DF80E2023
:108270008DF80F200CE0022805D130218DF80D106B
:108280008DF80E1004E0032802D130208DF80D0087
:10829000694603A804F018FD03A804F017FEC51EE4
:1082A000EDB22A4603A9204604F0AEFE0023635532
:1082B0002046074904F008FD03A92046491904F0A7
:1082C00003FD204607B030BD6F12033A00007A4428
:1082D000A2E5000837B5037904460D46052B34D8CE
:1082E000DFE803F003060A0D1114816809782DE018
:1082F000806890F9001029E08368198826E0826878
:10830000B2F9001022E0816809681FE080686946C0
:108310000068FFF777FF01461148FAF7D3F8F5B187
:10832000E068F8F7F3FB6946FFF76CFF01460D487C
:10833000FAF7C8F82069F8F7E9FB6946FFF762FF2A
:1083400001460848FAF7BEF809E000210648FAF7A6
:10835000B9F825B10548E1682269FAF7B3F83EBDDE
:108360005CE500085BE50008FDE70008F9E70008A8
:108370002DE9F047064604F0A9FD054620B1012885
:1083800019D133782A2B16D14748FFF765FC002412
:1083900014266643454F4648F159FAF793F8B81941
:1083A0002946FFF797FF01344248FFF755FC6F2C31
:1083B000EED1BDE8F08730463D2104F0ABFC00284B
:1083C00057D0441C204604F09FFA82462046FFF70F
:1083D000ADFB0027054614247C43DFF8D09054F809
:1083E0000980404604F072FD41460246304604F0E2
:1083F0009DFD002835D14C44E068F8F787FB014625
:108400002846F8F789FD002829D02069F8F77EFB77
:1084100001462846F8F776FD002820D020792279F9
:10842000052818BF5546052A0FD8DFE802F00303D8
:108430000606090CA1680D7007E0A268158004E02B
:10844000A068056001E0A1680D6041461A48FAF78E
:1084500039F820460021BDE8F047FFF73BBF174839
:1084600003E001376F2FB6D11548BDE8F047FFF79D
:10847000F3BB0446142565430C4F314655F807807D
:10848000404605F025F850B109484146FAF71AF878
:1084900078190021FFF71EFF0648FAF713F8013498
:1084A0006F2CE7D1BDE8F08700E80008E8F200088B
:1084B000DFE8000812E8000815E8000820E80008D6
:1084C00045E800082DE9F043584885B0584CF9F7C5
:1084D000F9FF5848FFF752FE6279574B511E574833
:1084E00053F82110F9F7EEFF20690021F8F7F6FCA8
:1084F000002858D10025266900213046F8F7EEFC07
:1085000000284CD101354E482946D4F81490D4F8AF
:108510001880E769F9F7D6FF30460021F8F7E8FC44
:1085200010B14848F9F7CEFF69463046FFF76AFEBA
:1085300001464548F9F7C6FF48460021F8F7D8FC40
:1085400010B14048F9F7BEFF69464846FFF75AFEAA
:1085500001463D48F9F7B6FF40460021F8F7C8FC50
:1085600010B13848F9F7AEFF69464046FFF74AFEBA
:1085700001463548F9F7A6FF38460021F8F7B8FC60
:1085800010B13048F9F79EFF69463846FFF73AFECA
:1085900001462E48F9F796FF10340C2DABD12C482C
:1085A000691CF9F78FFFF9F757FE2A4C064654F875
:1085B000041F19B12848F9F785FFF8E70D46274849
:1085C00050F8251049B1012202FA05F2324202D0D8
:1085D0002348F9F777FF0135F1E7154B214ACE180B
:1085E00096F808418B5C04A801310519082905F8A3
:1085F000103CF2D100241C4869468DF80840F9F778
:1086000061FF14256543194E1948A959F9F75AFF16
:1086100000217019FFF75EFE01341648FFF71CFBBE
:108620006F2CEED105B0BDE8F08300BF62E8000812
:10863000CC10002022EA00084CE3000892E8000871
:108640009DE80008ECE900085CE50008F0E400089B
:10865000A5E8000808E30008B7E800080CE30008F4
:10866000C5E8000800E30008D2E80008E8F20008C6
:10867000DBE8000812E800082DE9F04389B0044661
:1086800004F024FCC6B2002E6AD17948FFF7E4FA60
:10869000784C20690021F8F721FC38BB0136764878
:1086A0003146F9F70FFF206904A9FFF7ABFD01463A
:1086B0007248F9F707FF606904A9FFF7A3FD0146B7
:1086C0006E48F9F7FFFEA06904A9FFF79BFD01467C
:1086D0006A48F9F7F7FEE06904A9FFF793FD014640
:1086E0006748F9F7EFFE10340C2ED2D10025654C07
:1086F0002F46A8464FF000091034B14514DA404621
:1087000054F8101CF8F74EF954F80C1C8046284613
:10871000F8F748F954F8081C05463846F8F742F9C6
:1087200009F101090746E7E75748CDF804800295AB
:108730000397FFF791FA002401A82358534923F027
:108740000040F8F7F3FB5249524A0434002814BFA2
:1087500010460846FFF780FA0C2CEDD14E4870E029
:1087600020464E49052204F0E1FB38B9414B002276
:10877000C1181030C0280A61F8D176E02046484977
:10878000042204F0D3FB0546204605BB202104F05B
:10879000C1FA002869D0461C304604F097FB2C46ED
:1087A0000746404850F824500DB93F4849E030464C
:1087B0002946FAB204F0BAFB38B92046FCF70EFDA0
:1087C0003A482946F9F77EFE47E00134E9E704F02C
:1087D0009BF8461E0B2E074643DC2046202104F062
:1087E00099FA054640B1451C2846FFF79FF9214BF1
:1087F0003F01D851012400E004462846202104F01E
:1088000089FA054640B1451C2846FFF78FF91949FA
:10881000013401EB061250612846202104F07AFA57
:10882000054640B1451C2846FFF780F9114B01343D
:1088300003EB061188612846202104F06BFA18B971
:108840001B48FFF709FA10E00130FFF76FF9094AFA
:10885000032C02EB0616F061F2D11648FFF70CFF6D
:1088600003E015480C21F9F72DFE09B0BDE8F083AF
:10887000EDE80008CC10002018E900081EE9000807
:10888000F0E40008E010002022E900080AD7233CA9
:10889000E9E80008E5E8000812E8000831E9000806
:1088A00037E900084CE30008D4E600083CE900087A
:1088B0004FE9000822EA000889E90008F0B5694B91
:1088C00087B01A783AB9012018706748FFF7C4F9E1
:1088D0006648FFF7C1F9664C2068FBF7DEF900280F
:1088E00000F0BD802068FBF7DDF909280146614AE8
:1088F00001D03F2851D1002517685F4C2E462FB17B
:108900005E4821683A4604F011FB10B9254606B9C5
:1089100026465B490C348C42F1D3C6B13468D5F895
:1089200000E03B46E05C1EF8031081420DD1534A43
:1089300041B92D2B06D820244E48D454013303606E
:10894000D15404E0D0540133ECE74A490B60494A62
:1089500014681CB1AE4201D13C4612E04948FFF711
:108960007BF9AE4209D856F80C0BFFF775F9404B6E
:1089700009211868FBF781F9F3E73C48FFF76CF928
:1089800000243C4B18688442A5D239493B4A086808
:10899000115DFBF772F90134F3E713682BB9042872
:1089A00038D13648FFF7F8FA59E00C2801D136489B
:1089B0008CE70A2901D00D2948D12E4D3348FFF705
:1089C0004BF92E4C2A6832490023A354049300919A
:1089D00003A8294910220C23039403F099FF0546AC
:1089E00038B1006804F072FA0130AA682018904784
:1089F00002E02848FFF730F9002130221F4804F038
:108A0000CDF818481B4B027800211960002A7FF42A
:108A10005FAF24E00C28CAD07F2903D15BE72F2B5E
:108A20003FF659AF1F297FF656AF7E293FF653AF69
:108A300013B920293FF44FAF104C0E480C4AE154B3
:108A4000013303601068FBF718F944E77F29E6D18A
:108A50000A485C1E0021015514600F4839E707B031
:108A6000F0BD00BF2C100020B1E90008E9E90008C2
:108A70001017002060100020A8E300082D1000202F
:108A800068E40008EEE90008F3E9000812E80008CD
:108A9000857D0008FEE900081FEA0008F8B5174EBA
:108AA000174C184D0746C1B230682170FBF7E5F846
:108AB00022782B78C7F3072182EA030028703068F8
:108AC0002170FBF7DAF821782A78306881EA02030E
:108AD000C7F307412B702170FBF7CFF82078297876
:108AE00080EA0102390E306821702A70FBF7C5F860
:108AF0002B78207880EA03012970F8BD1017002038
:108B00006410002065100020F8B50D4E0D4D0E4C80
:108B1000C1B2074630682970FBF7AFF82A7823788E
:108B2000391282EA0300207029703068C9B2FBF75D
:108B3000A4F823782A7882EA03002070F8BD00BFE9
:108B400010170020C110002065100020054B10B543
:108B5000044621461868FBF790F803480278544011
:108B6000047010BD1017002065100020034B04494D
:108B70001A78885C01321A70704700BF67100020B5
:108B80008010002010B5FFF7F1FF0446FFF7EEFF5D
:108B900004EB002080B210BD10B5FFF7F3FF0446D0
:108BA000FFF7F0FF04EB004010BD000038B50446AD
:108BB00024200D46FFF7CAFF4D20FFF7C7FF002C0A
:108BC0000CBF3E202120FFF7C1FF064B00222846A4
:108BD0001A70FFF7BBFF04480078BDE83840FFF784
:108BE000B5BF00BF651000206A10002001460020BC
:108BF000FFF7DCBF01460120FFF7D8BF014B187813
:108C0000FFF7A4BF6510002070B5054608460E4664
:108C1000FFF7ECFF2C467219D0B2E3B2984204D0B1
:108C200014F8010BFFF792FFF5E770BD10B5441E75
:108C300014F8010F10B1FFF789FFF9E710BD00002C
:108C40002DE9F843002701240025144B18788542AC
:108C50001CDA1349134B15F801800C2202FB083073
:108C6000406804F033F981460CB13F180CE0264609
:108C70004E4509DA0B4A0C2101FB08235868805D38
:108C8000FFF764FF0136F3E70135DEE724B1F8B200
:108C9000FFF7ACFF0024D7E7BDE8F8836810002099
:108CA0006B1000206C00002070B5394DFF2115229B
:108CB000284603F073FF002302202B70FEF70EF806
:108CC000012418B102206C70A87003240420FEF760
:108CD00005F868B12E4E03214FF400503155651C44
:108CE000F9F726F918B104227255023400E02C4637
:108CF0000220FDF7F3FF48B1254B05201E19062180
:108D0000072518557170B570033404E00820FDF78D
:108D1000E5FF0028F0D12020F9F70AF918B11C4B23
:108D200008221A5501344FF48070F9F701F930B177
:108D300017480A2601190B2506554D700234154AAD
:108D4000134B5079082801D00E2802D10C261E554D
:108D500001340D2104201955651CF9F7E9F818B103
:108D60000B4811224255A51C0A49132391F82E21C4
:108D7000074E6C1C101C18BF01207355F9F7D8F86A
:108D800010B114203055AC1C034B1C7070BD00BFDB
:108D90006B100020CC10002068100020F8B5B54CF6
:108DA0002068FAF77AFF002800F047852068FAF774
:108DB00079FFB14A0346117871B9B0F124046342D6
:108DC00053EB040111700029E9D1AC4A5478002C0E
:108DD000E5D1FEF787FEE2E7012904D14D280CBF5B
:108DE0000223002321E0022904D13C280CBF0323E5
:108DF00000231AE003290FD140284FF0000101D9C8
:108E00001170CCE79E489F4C03709F482170017001
:108E10009E490B70042308E0042908D19B499C4813
:108E20000C78037063400B7005231370B7E70529B6
:108E3000B5D19448924C017822788A42934A07D956
:108E400014785C401470934A53544B1C0370A6E78B
:108E50001078984240F0EC848D4B19787B2900F013
:108E6000318300F2C5806E2900F07B8360D86829C9
:108E700000F0448325D8652900F0108219D86429B0
:108E800040F0D1840720844CFFF7B0FEE620FFF7C6
:108E90005DFE6079FFF75AFE0020FFF757FE94F859
:108EA00019017E4B7E4A00280CBF1046184600F080
:108EB0006BBC662900F07082672940F0B484794861
:108EC0001DE36B2900F02B8323D8692900F01B8355
:108ED0006A2940F0A8841020FFF788FE6748724C8A
:108EE000C07AFFF733FE71490878FFF72FFE20683C
:108EF000FFF7D4FD6068FFF7D1FD6D4AB2F90000BD
:108F0000FFF702FE6B4BB3F90000FFF7FDFD6A4A65
:108F100024E36C2900F015836D2940F08484062039
:108F2000FFF764FE65490868FFF7B8FD644A15E37A
:108F3000732900F083833CD8702900F04183C0F08E
:108F40002183712900F04F83722940F06C84524CC8
:108F50001620FFF74BFE0020FFF7D6FDB4F9D00036
:108F6000FFF7D2FD574DB4F9D200FFF7CDFDB4F9AC
:108F7000D400FFF7C9FDB5F9B600FFF7C5FD002025
:108F8000FFF7C2FD0020FFF789FDB5F928000A238D
:108F900090FBF3F0FFF7B8FD94F80401FFF7D6FD5E
:108FA00094F80601FFF7D2FD94F80501FFF7CEFD16
:108FB00073E3762900F04D830DD8742900F02B83DC
:108FC000752940F030842F20FFF710FE3E48FFF750
:108FD0002DFE00F02BBC772900F02083782940F08B
:108FE0002284384C3820FFF701FE04F1400537E2B7
:108FF000D02900F0878300F2CA80CA2900F00F81CF
:109000006CD8A42900F0EE8310D8A02940F00B847E
:109010000C20FFF7EBFD2D492D4C0868FFF73EFDB6
:109020002C4A1068FFF73AFD2068ADE3C82900F02C
:10903000ED80C92940F0F783FFF798FD0F4B1A4CDC
:10904000D872FFF793FD19490870FFF7A5FD20605E
:10905000FFF7A2FD6060FFF795FD154A1080FFF74E
:1090600091FD144B18801C48017841F002040470F3
:10907000E4E000BF10170020C0100020831600207D
:109080006610002069100020671000206510002085
:109090006A10002080100020CC1000201C000080EE
:1090A0001400008054000020581600207016002084
:1090B000021600200E160020B40D0020A01500207E
:1090C000900B00206814002094FB0008E8F7FF1FB5
:1090D000F0F7FF1FECF7FF1FCC0D0020CD2900F0AB
:1090E0001B8322D8CB2900F0AB80CC2940F09B8396
:1090F000FFF73CFDC74CE077FFF738FD84F8200010
:10910000FFF734FD84F82300FFF730FD84F82400D6
:10911000FFF72CFD84F82500FFF728FD84F82100D7
:10912000FFF724FD84F8220088E0CE2900F0FE82BB
:10913000CF2940F07883FFF725FDFFF723FDB64CDC
:10914000B44DA4F8D000FFF71DFDA4F8D200FFF73E
:1091500019FDA4F8D400FFF715FDA5F8B600FFF738
:1091600011FDFFF719FDFFF70DFD0A235843288570
:10917000FFF7FCFC84F80401FFF7F8FC84F8060113
:10918000FFF7F4FC84F80501FFF7F0FC56E0D52961
:1091900000F0A6810FD8D2296BD0C0F08282D329EB
:1091A00077D0D42940F03F839A4C0020FFF71EFD72
:1091B00004F1400568E1F02900F0D9820CD8D629E5
:1091C0004ED0EF2940F02F83FFF7DCFC914CA085B7
:1091D000FFF7D8FC608531E0FA2900F0AF82FE2964
:1091E00040F021830820FFF701FD8C4C8C488D4B0B
:1091F00001682068B1FBF3F2B0FBF3F34FF47A712E
:1092000001FB0234884AD4800024A8E20024FFF73E
:10921000B9FC864A10530234102CF8D10EE0844C6D
:1092200004F10A05FFF7A2FC01346070FFF79EFC11
:10923000E072FFF79BFCAC426075F3D100208BE23B
:1092400000247C4801788C42F8D27B4D655DFFF7A5
:1092500099FC704A013402EB4505A5F84200F0E79D
:109260000024FFF78FFC754A10530234102CF8D1FC
:10927000E4E7734C6478002CE0D1FFF777FC664993
:10928000022881F8940388BF81F89443F8F7F2FD2F
:109290003FE2FFF777FC6B490880CFE76A4D0B2070
:1092A000FFF7A4FCB5F90000FFF72EFCFAF7A4FCC9
:1092B00000B2FFF729FC0220FDF710FD054604204F
:1092C000FDF70CFD04460820FDF708FD820042EA88
:1092D0004401294320208CB2FDF700FD44EAC00080
:1092E00084B21020FDF7FAFC44EA001318B2FFF72D
:1092F0000BFC534A1079D17884005378907944EA72
:109300004101194341EAC0045179537A44EA4110BA
:1093100040EA83144D48C17944EAC113047A417A82
:1093200043EA042343EA4124D379117A44EA8324AB
:10933000927A44EAC123417B43EA0234827B44EAC5
:109340004133017C43EA8234027944EA0143417C9F
:1093500043EA0214827C44EA4143C17C43EA8244EA
:10936000007D44EAC142334B42EA005400201978A0
:1093700003468B420AD2304D01225D5D02FA05F5AB
:1093800025421CBF9A4010430133F2E7224CFFF7FD
:1093900085FB94F8940381E11220FFF727FC2C4908
:1093A0000C88B4F5806F2B4CB4F9000008D8FFF797
:1093B000ABFBB4F90200FFF7A7FBB4F904000EE021
:1093C000082590FBF5F0FFF79FFBB4F9020090FB36
:1093D000F5F0FFF799FBB4F9043093FBF5F01E4C60
:1093E000FFF792FBB4F90000FFF78EFBB4F902001F
:1093F000FFF78AFBB4F90400184CFFF785FBB4F9BA
:109400000000FFF781FBB4F90200FFF77DFBB4F920
:109410000400B6E168140020CC1000208801002070
:109420008401002040420F0038150020CC16002097
:1094300067140020681000206B100020D815002051
:109440008316002068150020E206002094160020F4
:1094500042000020A8150020540B002050150020C9
:10946000B4F97400FFF750FBB4F97600FFF74CFB3A
:10947000B4F97800FFF748FB94F87A000834FFF756
:1094800065FBAC42ECD1D1E1FFF77CFBA4F87400A2
:10949000FFF778FBA4F87600FFF774FBA0F57A726B
:1094A000072893B298BF84F87B00B3F57A7F98BF02
:1094B000A4F87800FFF75AFB84F87A000834AC422D
:1094C000E2D1B3E10820FFF791FB0024B04AA318D2
:1094D00093F87B000834FFF739FB402CF6D1A5E167
:1094E0000020FFF783FB0024FFF740FBA84AA318E6
:1094F0000834402C83F87B00F6D197E1A548102171
:10950000FFF782FB92E11020FFF770FB0024A248D6
:10951000005F0234FFF7F8FA102CF8D186E105203D
:10952000FFF764FB9D4BB3F90000FFF7EDFA9C4891
:10953000B0F90000FFF7E8FA9A490A7802F0010052
:10954000ACE0994C0620FFF751FBB4F90000FFF79F
:10955000DBFAB4F90200FFF7D7FA944AB2F9000037
:109560000FE10720FFF742FB91480078FFF7EEFA82
:109570000020FFF7C9FA8F4BB3F90000FFF7C4FAD8
:109580000020FEE0824C0720FFF730FBE07FFFF772
:10959000DDFA94F82000FFF7D9FA94F82300FFF7DA
:1095A000D5FA94F82400FFF7D1FA94F82500FFF7D4
:1095B000CDFA94F82100FFF7C9FA94F822006DE083
:1095C0001E20FFF713FB7C4C04F10A050134607880
:1095D000FFF7BCFAE07AFFF7B9FA607DFFF7B6FA59
:1095E000AC42F3D122E175490A78540004F0FE0040
:1095F000FFF7FCFA0024714803789C4280F0168142
:109600006F496348625C013400EB4203B3F94200E6
:10961000FFF77AFAEFE7FFF713FB07E1674900244A
:109620000878FFF7E3FA654A1078844280F0FE80FC
:10963000634B185DFFF78AFA0134F4E70820FFF75F
:10964000D5FA0124E0B20134FFF780FA092CF9D1F0
:10965000ECE0FFF78BFA06461220FFF7C7FA0EB9C7
:10966000584902E0102E03D157490D684C6801E0BB
:10967000002425463046FFF769FA2846FFF70EFA20
:109680002046FFF70BFA514A1068FFF707FA00204F
:10969000FFF73AFA0020FFF737FA0020FFF756FAF3
:1096A000C4E0FFF763FA0546FFF776FA0746FFF7CF
:1096B00073FA0646FFF770FA0446FFF763FAFFF7FE
:1096C00061FAFFF753FA65B93E4841490122076044
:1096D0004660CD710A73002C3FF4B0AD3B4B1C606B
:1096E000ACE5102D7FF4AAAD3748076046600CB199
:1096F000364A1460374B344802211970011DFCF7BB
:10970000DBFB9BE53248417800297FF497ADF8F701
:1097100021FCF8F76BFB91E52D4C6378002B7FF46F
:109720008DAD2D494FF4C870088087E528484178F1
:1097300000297FF483AD012282737FE5244B5C789E
:10974000002C70D1254991F89403F8F783FBF8F7C2
:1097500091FBF8F74BFB2046FFF748FA66E02048FC
:10976000005F0234FFF7D0F9082CF8D15EE0084C16
:109770000420FFF73BFAB4F92C00FFF7C5F9B4F960
:109780002A00FFF7C1F951E0FFF788F94EE000BF6A
:1097900068140020C0150020CC16002038160020C8
:1097A00044160020CC0D0020440B00207A15002028
:1097B000C810002040150020671400206810002009
:1097C0006B1000203C16002010160020A41500206D
:1097D00083160020880C0020EA060020CC10002010
:1097E00038150020154C23789800411CC8B2FFF7AB
:1097F000FDF92078FFF7AAF90024104A13789C425B
:1098000014D20F48005DFFF7A1F90E49085DFFF77C
:109810009DF90D4A105DFFF799F90C4B185DFFF7A4
:1098200095F90134E9E70020FFF7E4F9FFF7E6F9DD
:10983000074900200870FFF7B2BAF8BD7116002082
:10984000F115002046160020601600207216002038
:10985000C01000202DE9F041074688461646002436
:10986000B44213D00025BD420AD0094B0135DA6855
:10987000EDB282F48050D8604046FAF7B0FCF2E7CF
:109880003C200134FAF7ABFCE4B2E9E7BDE8F08133
:10989000001001400F4B1A6842F00100186059682F
:1098A0000D4A0A405A60186820F0847121F4803211
:1098B0001A60186820F4802119605A684FF41F015B
:1098C00022F4FE0058609960044B4FF000629A60E9
:1098D000704700BF001002400000FFF800ED00E0FC
:1098E000164A174B516801F00C00042803D00828D1
:1098F00005D0144801E014490868186011E0516867
:109900005068C1F383410231C00301D40F4A06E01D
:1099100052680D4812F4003F026818BF52085143C4
:109920001960064B0A485A68054BC2F30311415CA3
:109930001A6822FA01F21A60704700BF0010024054
:109940008801002000127A008401002000093D00F7
:10995000740100201FB50023574C4FF4E011009311
:10996000019302930391226842F480332360A1693A
:1099700041F01002A261504C236803F400310191C0
:10998000009A531C0093019919B9009AB2F5A06F7F
:10999000F1D12168484B11F4003401D0022416E0C3
:1099A0001A6842F0010119600094434B1C6804F0EE
:1099B0000202019200994C1C0094019A1AB9009974
:1099C000B1F5A06FF1D11B6899073BD501243B4944
:1099D00002940A6842F010030B600C6824F0030242
:1099E0000A600B6843F002040C60A1F580535968CB
:1099F00059605A685A605C68314A44F48061596021
:109A0000146824F0704111602E4C2F490C605C6882
:109A100024F47C145C60146844F00044146094687E
:109A200024F400449460043A9268120449BF274A1F
:109A30004FF4E0120A604FF4801203920299012958
:109A400001D119E0FEE702291AD168B10398B0F5F7
:109A5000801F02D14FF4A01205E0039BB3F5E01F75
:109A600002D14FF400120392134B5968039841EA54
:109A7000000242F4803002E0596841F460105860FE
:109A80000D4B1A68184642F08071196002680A4B43
:109A90009201FBD5596821F0030058605A6842F0E2
:109AA00002015960044B586800F00C02082AF9D1F1
:109AB000FFF716FF1FBD00BF00100240002002404C
:109AC0000410014000127A0084010020001BB7003E
:109AD000CB78F0B5DA0648BF8A78098803F00F051D
:109AE00048BF154311F0FF0F1ED004680022012764
:109AF00007FA02F707EA0106BE4211D197004FF0BC
:109B00000F0C0CFA07FC05FA07F724EA0C04282BC3
:109B100044EA070401D1466102E0482B08BF066110
:109B20000132082AE3D10460FF2920D944680022C9
:109B300002F10806012707FA06F707EA0106BE4206
:109B400011D197004FF00F0C0CFA07FC05FA07F73C
:109B500024EA0C04282B44EA070401D1466102E000
:109B6000482B08BF06610132082AE1D14460F0BDEC
:109B700008B5154B98420BD101214FF4805000F0ED
:109B8000ADFD4FF480500021BDE8084000F0A6BDB7
:109B90000E49884207D14FF48040012100F0AAFD10
:109BA0004FF4804009E00A4A90420BD14FF4004044
:109BB000012100F09FFD4FF400400021BDE8084066
:109BC00000F098BD08BD00BF0030014000380040E3
:109BD000003C00400B8810B54C88028823438C88D9
:109BE00002F441522343CC8823430C8923434C89FC
:109BF00023438C892343CC89098A23431A4393B294
:109C00000380828B22F400631A04130C8383018285
:109C100010BD038819B199B241F0400303E023F06D
:109C200040010A04130C03807047818170478089CA
:109C300080B27047038919420CBF00200120704791
:109C4000426810B522F470230A6823F4807444EA51
:109C500002030C7943EA04224260CB688A68846874
:109C60001A43084B234013434A7943EA4203836073
:109C7000097CC26A4B1E22F47002D9B242EA015238
:109C8000C26210BDFDF7F1FF836811B143F001011D
:109C900001E023F0010181607047836811B143F452
:109CA000807101E023F4807181607047836843F024
:109CB0000801816070478068C0F3C0007047836806
:109CC00043F00401816070478068C0F380007047F2
:109CD000836811B143F4A00101E023F4A001816085
:109CE0007047092970B54FF003040CD94C43072580
:109CF0001E3C05FA04F503FA04F3C66826EA0505D6
:109D00002B43C3600BE04C43072505FA04F503FA27
:109D100004F3066926EA050545EA03040461062AF8
:109D20004FF005030DD8013A53431F2202FA03F204
:109D300001FA03F1446B24EA020242EA010343639D
:109D400070BD0C2A0DD853431F22233B02FA03F2A5
:109D500001FA03F1046B24EA020242EA01030363FD
:109D600070BD53431F22413B02FA03F201FA03F193
:109D7000C46A24EA02021143C16270BD40F0BF60B0
:109D8000024B40F40031D960704700BF00ED00E0A5
:109D9000C37810B503B3164CE168CB43C3F3022478
:109DA0004178C4F1040201FA02F10F2222FA04F20E
:109DB0008478037822400A43110103F16043CAB258
:109DC00003F5614181F800230078012200F01F03B0
:109DD000410902FA03F007E00078012200F01F03B6
:109DE000410902FA03F02031024B43F8210010BD73
:109DF00000ED00E000E100E030B5048C24F0010546
:109E00002C04250C0584048BA5B225F0F3052A4308
:109E100042EA0313114A048C9042A4B29DB215D0B9
:109E200002F50063984211D0B0F1804F0ED0A3F537
:109E3000983290420AD002F58063984206D003F52A
:109E40008062904218BF24F00A0401D124F0020479
:109E500044F0010421430583018430BD002C0140FE
:109E600030B5048C24F010052C04250C0584048BDB
:109E7000058C24F440742405240D44EA022242EAAD
:109E80000333144AADB290429BB212D002F5006285
:109E900090420ED0B0F1804F0BD0A2F59832904294
:109EA00007D002F58062904203D002F580629042B2
:109EB00007D125F0200242F0100545EA011189B2D0
:109EC00004E025F0A00545F0100529430383018433
:109ED00030BD00BF002C0140224A038890429BB253
:109EE00012D002F5006290420ED0B0F1804F0BD03C
:109EF000A2F59832904207D002F58062904203D0DA
:109F000002F58062904203D14A8823F07003134324
:109F1000154A904208D002F58062904204D023F4A2
:109F20004073CA889BB2134303808B880A88838559
:109F30000C4B028598420FD003F5006290420BD083
:109F400002F54063984207D003F58062904203D047
:109F500002F58063984201D1097A0186012282824A
:109F6000704700BF002C014000100040038C70B50A
:109F700023F001021404250C0584068C8388028BCF
:109F80009CB222F073052B040D881A0C26F00206F1
:109F900033042A434E880D891B0C3543ADB22B4345
:109FA000134DA8420FD005F50065A8420BD005F56A
:109FB0004065A84207D005F58065A84203D005F5A5
:109FC0008065A8420ED123F008064B898D881E4378
:109FD00026F004032B43CE898D8924F44074354345
:109FE000ADB22C43C988848002838186038470BD0E
:109FF000002C0140038C30B523F010021404250C12
:10A000000584038C8288048B23F0200324F4E64526
:10A010002C040D88240C44EA05241D042B0C0D8906
:10A0200092B243EA05134D88A4B243EA0513124DD8
:10A030009BB2A84203D005F50065A84215D14D8911
:10A0400023F080039BB243EA05134FF6BF751D4012
:10A050008B8822F4406245EA0315ABB28D8942EA4F
:10A060008502CD8942EA850292B2C9888280048342
:10A070000187038430BD00BF002C0140038C30B544
:10A0800023F480721404250C0584038C8288848B4D
:10A0900023F4007324F073052C040D88240C2C4346
:10A0A0001D042B0C0D8992B243EA05234D8843EA27
:10A0B0000523124D9BB2A84203D005F50065A842C6
:10A0C00015D14D8923F400639BB243EA05234FF673
:10A0D000FF351D408B8822F4405245EA0325ABB280
:10A0E0008D8942EA0512CD8942EA051292B2C988E9
:10A0F000828084838187038430BD00BF002C0140AF
:10A10000038C30B523F480521404250C0584038C91
:10A110008288858B94B225F4E64215042A0C0D88BA
:10A1200023F4005342EA05221D042B0C0D8992B240
:10A1300043EA05334D8843EA05330A4D9BB2A842F2
:10A1400003D005F50065A84205D18D8924F480442B
:10A1500044EA8514A4B2C98884808283A0F84010A0
:10A16000038430BD002C014000214FF6FF73838033
:10A170000180C180418001727047038819B199B292
:10A1800041F0010303E023F001010A04130C0380F2
:10A190007047B0F8443029B16FEA43436FEA534146
:10A1A0008AB201E059044A0CA0F844207047838920
:10A1B0009BB20AB1194301E023EA01018181704792
:10A1C000038B23F0080213041A0C11430183704718
:10A1D000038B23F4006213041A0C42EA01218BB2B0
:10A1E00003837047838B23F0080213041A0C114376
:10A1F00081837047838B23F4006213041A0C42EAB4
:10A2000001218BB283837047038B23F00C0213046C
:10A210001A0C0283038B9AB2114301837047038B9C
:10A2200023F4406213041A0C0283038B9AB242EAAD
:10A2300001218BB203837047838B23F00C0213043C
:10A240001A0C8283838B9AB2114381837047838B6C
:10A2500023F4406213041A0C8283838B9AB242EA7D
:10A2600001218BB283837047F8B50B880D460446F5
:10A270004988AA8843B92B89FFF7BEFDE9882046A3
:10A28000BDE8F840FFF7C0BF042B08D12B89FFF7CA
:10A29000E7FDE9882046BDE8F840FFF7C0BF082B7E
:10A2A0000E462F89008C3BD120F480731804030CD8
:10A2B0002384A08B83B223F0F30343EA0717374BC1
:10A2C000208CBFB29C4280B247EA020212D003F552
:10A2D00000639C420ED0B4F1804F0BD0A3F59833AD
:10A2E0009C4207D003F580639C4203D003F5806352
:10A2F0009C4207D120F4007040EA06218BB243F45F
:10A30000807305E020F4206041F4807140EA01038D
:10A31000E9882046A2832384BDE8F840FFF78CBF7C
:10A3200020F480531804030C2384A38B208C23F483
:10A3300040731B051B0D43EA022242EA0733174A0A
:10A3400080B294429BB212D002F5006294420ED0C9
:10A35000B4F1804F0BD0A2F59832944207D002F5A9
:10A360008062944203D002F58062944207D120F4C7
:10A37000005040EA063291B241F4805205E047F6BF
:10A38000FF52024041F480510A43E9882046A383EA
:10A390002284BDE8F840FFF75ABF00BF002C0140FF
:10A3A000808E80B27047008F80B27047808F80B2FD
:10A3B0007047B0F8400080B27047038A828911EA82
:10A3C000030092B203D011420CBF0020012070475D
:10A3D000C9438AB202827047038A30B50D460446EB
:10A3E000EA8898B220F4405111432182A389288938
:10A3F000A98823F4B05340EA0102688923F00C01D4
:10A4000002430804030C1A4391B2A181A08AAA89CD
:10A4100083B223F4407187B01143A18201A800F0F8
:10A42000EBF81848A38984420CBF0498039819B22A
:10A4300000294FF019032A6803FB00F001DA5100EC
:10A4400000E09100B0FBF1F16423B1FBF3F21201E3
:10A45000100903FB1011A08900B2002806DAC90018
:10A460003231B1FBF3F303F0070005E009013231AB
:10A47000B1FBF3F303F00F00024390B2208107B069
:10A4800030BD00BF00380140838919B199B241F451
:10A49000005303E023F400510A04130C8381704736
:10A4A000C1F3421310B5012401F01F01A34204FAC5
:10A4B00001F101D10C3004E0022B01D1103000E099
:10A4C0001430036812B143EA010201E023EA0102F9
:10A4D000026010BD838A9BB20AB1194301E023EAEE
:10A4E0000101818270470000034A044B02F1883069
:10A4F0005A605860704700BF230167450020024042
:10A50000024B1A6942F08000186170470020024037
:10A51000014BD860704700BF00200240084BDA684A
:10A52000D20709D4D868400708D4D96811F0100FB1
:10A530000CBF0420032070470120704702207047A1
:10A540000020024010B50446FFF7E8FF012806D1BD
:10A550001CB1FFF7E3FF013CF8E7052010BD002C1C
:10A5600008BF052010BD000073B5002306464FF458
:10A5700000500D460193FFF7E5FF04281AD10E4C59
:10A58000AAB2206940F0010121614FF400503280ED
:10A59000FFF7D8FF042808D102360196019B2D0C45
:10A5A0001D804FF40050FFF7CDFF216941F6FE7288
:10A5B0000A4022617CBD00BF0020024038B505463C
:10A5C0004FF43020FFF7BEFF042812D1094C236955
:10A5D00043F002002061656121694FF4302041F0B1
:10A5E00040022261FFF7AEFF216941F6FD730B4087
:10A5F000236138BD00200240204B10B55A6802F09C
:10A600000C01042903D0082905D01D4B01E01D4C85
:10A610002368036011E05C685968C4F38342941CAA
:10A62000C90301D4184A06E016495B680A6813F4A6
:10A63000003F18BF520854430460104B5968C1F3DF
:10A64000031212498C5C026822FA04F242605C68D0
:10A65000C4F302240C5D22FA04F484605C68C4F341
:10A66000C224095D22FA01F2C2605B680849C3F3A3
:10A670008133CB5CB2FBF3F2026110BD00100240EB
:10A6800000127A008401002000093D0090010020A2
:10A690008C010020044B5A6909B1104301E022EA01
:10A6A00000005861704700BF00100240044B9A69D7
:10A6B00009B1104301E022EA00009861704700BF31
:10A6C00000100240044BDA6909B1104301E022EAAC
:10A6D0000000D861704700BF00100240044BDA68E8
:10A6E00009B1104301E022EA0000D860704700BFC2
:10A6F00000100240044B1A6909B1104301E022EA3C
:10A7000000001861704700BF00100240024B5A6AF7
:10A7100042F08070586270470010024008B50B4B41
:10A72000984207D14FF400100121FFF7E3FF4FF4E7
:10A73000001006E04FF480000121FFF7DBFF4FF42B
:10A7400080000021BDE80840FFF7D4BF005400405E
:10A75000F0B58688044687B026F03F000D46010418
:10A7600001A80E0CFFF748FF2C4A0399B1FBF2F049
:10A7700087B23E43A680238823F0010213041A0CFB
:10A7800022802B68264A93420AD85B00B1FBF3F083
:10A79000013783B2BFB22784032B98BF042320E084
:10A7A000EE884BF6FF72964204D103225343B1FB6D
:10A7B000F3F305E019225343B1FBF3F141F4804375
:10A7C00099B20A054FF4967208BF41F00101504357
:10A7D00041F400434FF47A7190FBF1F0421C91B2C6
:10A7E0002184A383228891B241F001032380208831
:10A7F00020F4816222F002010B04AA886989180CF6
:10A8000041EA02032989AA89184380B241EA020376
:10A81000208098B2208107B0F0BD00BF40420F00F9
:10A82000A086010041F28833002103604BF6FF72DD
:10A830004FF480438180C2800181418183817047D0
:10A84000038819B199B241F0010303E023F001013B
:10A850000A04130C03807047038819B199B241F4BC
:10A86000807303E023F480710A04130C03807047A3
:10A87000038819B199B241F4007303E023F4007125
:10A880000A04130C03807047038819B199B241F48C
:10A89000806303E023F480610A04130C0380704793
:10A8A00083889BB20AB1194301E023EA0101818048
:10A8B000704701827047008AC0B2704712B141F000
:10A8C000010101E001F0FE010182704702684FF6CC
:10A8D000FE73134003602D4B0021984201604160DC
:10A8E0008160C16022D02A49884229D0294B9842F0
:10A8F00030D02949884237D0284B98423ED0284B47
:10A90000984206D153F8681C41F4700043F8680C73
:10A9100070472449884206D151F87C0C40F070629F
:10A9200041F87C2C7047204B984206D153F8042CF8
:10A9300042F00F0143F8041C70471C49884206D1BD
:10A9400051F8183C43F0F00041F8180C7047184BD0
:10A95000984206D153F82C2C42F4706143F82C1C19
:10A9600070471449884206D151F8403C43F4704086
:10A9700041F8400C7047104B984205D153F8542CC5
:10A9800042F4702143F8541C704700BF0800024095
:10A990001C000240300002404400024058000240C7
:10A9A0006C00024080000240080402401C04024087
:10A9B00030040240440402405804024070B5066866
:10A9C0008C680D6A26F4FF4222F070060A6945EA97
:10A9D00004034C6913438A692343CC6913431C4322
:10A9E0004B6A44EA03028B6A1A4332430260CB6823
:10A9F0000A68496843608260C16070BD00230360DB
:10AA000043608360C360036143618361C361036228
:10AA100043628362704719B1016841F0010303E0AA
:10AA200002684FF6FE7313400360704703680AB173
:10AA3000194301E023EA010101607047416070475A
:10AA4000406880B270470000C3004CBF014B024B0E
:10AA500058607047000402400000024000B540F614
:10AA6000D87320F00042C3F649739A4283B001467E
:10AA700015DDB2F1FF4F03DBF5F792FF03B000BD28
:10AA8000694600F095FB00F00302012A0098019945
:10AA90000ED0022A07D082B900F0A0FDEEE7002117
:10AAA00000F09CFDEAE700F099FD00F10040E5E7C9
:10AAB00001F040FC00F10040E0E7012201F03AFC27
:10AAC000DCE700BF30B5C0F3C754A4F17F031E2BF1
:10AAD00083B0014621DC581C1DDBCD0F162B0CDD8D
:10AAE00021F07F4323F4000040F40000963C00FA7C
:10AAF00004F005B1404203B030BD114850F8254084
:10AB00002046F5F74FFF019021460198F5F748FFE1
:10AB100020F0004121B90020EDE7F6F711FAEAE74D
:10AB200020F07F4222F40003C0F3C75043F4000139
:10AB3000C0F1960221FA02F0002DDCD0DAE700BF66
:10AB400074FC000800B540F6D87320F00042C3F64C
:10AB500049739A4283B0014616DDB2F1FF4F03DB21
:10AB6000F5F71EFF03B000BD694600F021FB00F0C1
:10AB70000300012815D002280BD0B8B9009801991C
:10AB8000012201F0D7FBEDE70021002201F0D2FB0A
:10AB9000E8E700980199012201F0CCFB00F10040A8
:10ABA000E0E70098019900F019FDDBE700980199B2
:10ABB00000F014FD00F10040D4E700BF70B58AB08A
:10ABC000064600F09BF8224C054694F9003001330C
:10ABD00003D0304601F0B0FD10B928460AB070BD70
:10ABE000304601F05BFD4FF07E51F6F79FF90028EB
:10ABF000F3D0184A012100253046019200910895B2
:10AC0000F5F714FC02460B461348CDE90423CDE9C1
:10AC1000022301F011FC94F90030CDE90601022B6A
:10AC20000BD0684601F006FC38B1089850B9DDE950
:10AC30000601F5F761FE0546CFE701F089FE212107
:10AC40000160F2E701F084FE089A0260EFE700BFBE
:10AC5000A00100207CFC000884FC000800F002BA7F
:10AC600070B58AB0054600F04FFC224C064694F9B8
:10AC70000030013308D0284601F05EFD20B128469F
:10AC80000021F6F735F910B930460AB070BD1A4AFE
:10AC9000012128460026009101920896F5F7C6FB8F
:10ACA0002478CDE90401CDE902017CB9002200231A
:10ACB000CDE90623684601F0BDFB88B10898A0B92C
:10ACC000DDE90601F5F718FE0646DDE70020002164
:10ACD00002460B46F5F728FD022CCDE90601E9D125
:10ACE00001F036FE21230360E8E701F031FE089908
:10ACF0000160E5E7A001002088FC0008F8B520F01D
:10AD00000043B3F17E5F044613D00BDCB3F17C5FEC
:10AD100014DAB3F10C5F00F3A48040F6DB70C3F6E5
:10AD2000C970F8BD0146F5F73BFE0146F5F7F6FFA1
:10AD3000F8BD002840F30E810020F8BD0028C0F2C5
:10AD40000E8101464FF07E50F5F72AFE4FF07C5100
:10AD5000F5F730FF044600F0D7FB4EF608710646C3
:10AD600020F47F65C3F611012046F5F723FF47F66F
:10AD70000471C3F64F21F5F715FE2146F5F71AFFCA
:10AD800041F24611C3F62451F5F70AFE2146F5F7C4
:10AD900011FF40F6A821C3F64E61F5F703FE2146E8
:10ADA000F5F708FF4BF29001C3F6A661F5F7F8FD41
:10ADB0002146F5F7FFFE4AF6AB21C3F62A61F5F707
:10ADC000F1FD2146F5F7F6FE4CF22E610746C3F67B
:10ADD0009D512046F5F7EEFE43F26131C3F6307126
:10ADE000F5F7DEFD2146F5F7E5FE45F22D71C4F2DB
:10ADF0000101F5F7D7FD2146F5F7DCFE4DF23911DB
:10AE0000C4F21901F5F7CCFD2146F5F7D3FE4FF05A
:10AE10007E51F5F7C7FD01463846F5F77FFF31460D
:10AE2000F5F7C8FE25F00F05074629462846F5F731
:10AE3000C1FE01462046F5F7B3FD294604463046DB
:10AE4000F5F7B0FD01462046F5F768FF01463846A4
:10AE5000F5F7A8FD2946F5F7A5FD0146F5F7A2FD92
:10AE6000F8BD0146F5F7A6FE4EF60871C3F61101CE
:10AE70000546F5F79FFE47F60471C3F64F21F5F737
:10AE800091FD2946F5F796FE41F24611C3F624518D
:10AE9000F5F786FD2946F5F78DFE40F6A821C3F6A5
:10AEA0004E61F5F77FFD2946F5F784FE4BF29001E0
:10AEB000C3F6A661F5F774FD2946F5F77BFE4AF661
:10AEC000AB21C3F62A61F5F76DFD2946F5F772FE51
:10AED0004CF22E610646C3F69D512846F5F76AFEF0
:10AEE00043F26131C3F63071F5F75AFD2946F5F7A3
:10AEF00061FE45F22D71C4F20101F5F753FD2946BB
:10AF0000F5F758FE4DF23911C4F21901F5F748FD75
:10AF10002946F5F74FFE4FF07E51F5F743FD014608
:10AF20003046F5F7FBFE01462046F5F743FE0146A5
:10AF300042F26810C3F2A230F5F732FD0146204616
:10AF4000F5F72EFD014640F6DA70C3F6C970F5F745
:10AF500027FDF8BD40F6DB70C4F24900F8BD4FF0A4
:10AF60007E51F5F71FFD4FF07C51F5F723FE4EF6AD
:10AF70000871C3F611010446F5F71CFE47F604718B
:10AF8000C3F64F21F5F70EFD2146F5F713FE41F20A
:10AF90004611C3F62451F5F703FD2146F5F70AFEE5
:10AFA00040F6A821C3F64E61F5F7FCFC2146F5F703
:10AFB00001FE4BF29001C3F6A661F5F7F1FC2146C4
:10AFC000F5F7F8FD4AF6AB21C3F62A61F5F7EAFC7E
:10AFD0002146F5F7EFFD0646204600F095FA4CF2C3
:10AFE0002E610546C3F69D512046F5F7E3FD43F279
:10AFF0006131C3F63071F5F7D3FC2146F5F7DAFD80
:10B0000045F22D71C4F20101F5F7CCFC2146F5F7AC
:10B01000D1FD4DF23911C4F21901F5F7C1FC2146F9
:10B02000F5F7C8FD4FF07E51F5F7BCFC0146304600
:10B03000F5F774FE2946F5F7BDFD42F26811C3F23B
:10B04000A231F5F7ADFC01462846F5F7ABFC014609
:10B05000F5F7A8FC014640F6DA70C4F24900F5F7AE
:10B060009FFCF8BDF8B521F00044B4F1FF4F034652
:10B0700017DC20F00045B5F1FF4F064611DCB1F1B9
:10B080007E5F42D08F1707F0020040EAD37775B990
:10B09000022F35D0032F08D140F6DB73CCF24903E1
:10B0A00003E01846F5F77EFC03461846F8BDD4B118
:10B0B000B4F1FF4F2DD0B5F1FF4F14D02C1BE41588
:10B0C0003C2C18DC002952DB1846F5F727FE01F06E
:10B0D000E5FA01F0B7F9012F46D0022F35D0002F45
:10B0E00025D10346E1E7002E40F6DB731CDBC3F6F7
:10B0F000C9731846F8BD40F6DB70C3F6C970EAE7BD
:10B1000040F6DB73C4F24903CFE7BDE8F84001F035
:10B1100099B9B5F1FF4F2FD0022FF1D0032FBBD03B
:10B12000012F34D00023C0E7CBF6C973BDE74BF63F
:10B130002E51C3F2BB31F5F735FC40F6DB71C4F29A
:10B140004901F5F72DFC0346AFE74BF62E51C3F24C
:10B15000BB31F5F727FC014640F6DB70C4F249002D
:10B16000F5F71EFC0346A0E700F100439DE714F14C
:10B170003C0FA9DA0020AEE7022F13D0032F0CD02A
:10B18000012F40F6DB7305D0C3F649738DE74FF00E
:10B1900000438AE7CBF6497387E74CF6E433CCF2F9
:10B1A000160382E74CF6E433C4F216037DE700BFD2
:10B1B0002DE9F04F40F6D87320F00044C3F64973F0
:10B1C0009C4289B006460D4640F38B804CF6E33135
:10B1D000C4F216018C4226DC4FF478610028C3F6D5
:10B1E000C97140F32B81F5F7DBFB4FF47D6224F04E
:10B1F0000F04C3F6C9729442064600F0818044F2FF
:10B200004341C3F23571F5F7CBFB01462860304668
:10B21000F5F7C6FB44F24341C3F23571F5F7C0FBC5
:10B220000127686061E04FF47867C4F24937BC4297
:10B2300040F38180B4F1FF4F5BDA4FEAE459A9F1A2
:10B240008609A4EBC9542046F5F77AFEF5F75EFCB3
:10B250000246014620460592F5F7A2FB4FF08741D2
:10B26000F5F7A8FC0746F5F76BFEF5F74FFC01462E
:10B27000044638460694F5F793FB4FF08741F5F7FF
:10B2800099FC00210790F5F729FE002800F0F680D0
:10B290000327204600210DF11808013FF5F71EFE97
:10B2A00040B158F8044D00212046013FF5F716FE45
:10B2B0000028F6D1924B02200090019305A83B464E
:10B2C00029464A4600F066FA002E07460DDA95E850
:10B2D0000C0002F1004103F1004229606A6047421C
:10B2E00003E00023286000274B60384609B0BDE822
:10B2F000F08F0146F5F754FB002768602860F4E7FB
:10B300004FF48841C3F23571F5F74AFB4AF2083130
:10B31000C2F685610446F5F743FB014628602046E6
:10B32000F5F73EFB4AF20831C2F68561F5F738FBC6
:10B3300001276860D9E701F0B1F94FF68411C3F62F
:10B3400022718046F5F736FC4FF07C51F5F72AFB69
:10B35000F5F7F6FD0746F5F7D9FB4FF47861C3F62C
:10B36000C9718346F5F726FC01464046F5F718FB00
:10B3700044F243418146C3F235715846F5F71AFC51
:10B380001F2F8246514648461FDC5E4B7A1E53F8FB
:10B39000223024F0FF029A4217D0F5F701FB8046D5
:10B3A000C5F8008041464846F5F7FAFA5146F5F7E8
:10B3B000F7FA002E686098DA08F1004800F10041C1
:10B3C000C5F8008069607F428FE7F5F7E9FAE31579
:10B3D0008046C0F3C750191A0829E1DD4FF48841AF
:10B3E000C3F2357158460393F5F7E4FB82465146A4
:10B3F0004846F5F7D5FA044621464846F5F7D0FA0F
:10B400005146F5F7CDFA4AF208318146C2F6856118
:10B410005846F5F7CFFB4946F5F7C2FA8246514642
:10B420002046F5F7BDFA039BC0F3C7528046981A31
:10B43000192841DCC5F80080A146B3E7F5F7B2FA58
:10B440004FF47D6724F00F04C3F6C977BC4206466B
:10B4500016D044F24341C3F23571F5F7A3FA014621
:10B4600028603046F5F79CFA44F24341C3F2357147
:10B47000F5F798FA4FF0FF37686036E7032719E7CA
:10B480004FF48841C3F23571F5F78CFA4AF208316E
:10B49000C2F685610446F5F785FA01462860204624
:10B4A000F5F77EFA4AF20831C2F68561F5F77AFAC5
:10B4B0004FF0FF37686018E74FF42341C2F685610B
:10B4C0005846F5F777FB804641462046F5F768FA7F
:10B4D000814649462046F5F763FA4146F5F760FA9A
:10B4E00043F232110446C2F28D415846F5F762FB31
:10B4F0002146F5F755FA8246514648464DE700BFCA
:10B5000010FD000890FC000820F00042B2F1FF4F4F
:10B51000F8B50446034646D2002A42D0002852DB42
:10B52000C415B2F5000F09D210F4000553D15B0029
:10B5300001351902FBD5C5F10100241823F07F4124
:10B540007F3C21F40006E20746F4000048BF4000BB
:10B5500043004FF08072002760109A423C462CDD79
:10B560005B004FF400021825A61851089E4205F111
:10B57000FF3502DCB4189B1BBF185B0062189A42AF
:10B5800002DC9B1A54187F185B004A08013DEBD17E
:10B5900013B107F001017F187C1004F17C5303EB19
:10B5A000C0542046F8BD0146F5F704FB014620468D
:10B5B000F5F7F8F904462046F8BD4FF0007403F1A2
:10B5C0007F431746CCE70146F5F7EAF90146F5F760
:10B5D000A5FB0446E5E70120AFE700BF2DE9F843EE
:10B5E00020F00046B6F1485F05460F465BDAF5F7F6
:10B5F000A7FC002800F0CA8029462846F5F7DAFAA9
:10B600004DF24E71CAF647510446F5F7D3FA47F2A8
:10B61000F641C3F20F11F5F7C5F92146F5F7CAFA5D
:10B620004FF27C21C3F29341F5F7BAF92146F5F7C1
:10B63000C1FA40F60151C3F2D071F5F7B3F92146D2
:10B64000F5F7B8FA40F66131C3F6B621F5F7A8F977
:10B650002146F5F7AFFA4AF6AB21C3F62A51F5F7C2
:10B66000A1F92146F5F7A6FA804620464FF07C5115
:10B67000F5F7A0FA414606462046F5F79BFA39460B
:10B6800004462846F5F796FA01462046F5F788F96C
:10B6900001463046F5F784F901464FF07E50F5F744
:10B6A0007FF9BDE8F8830146F5F784FA4DF24E7153
:10B6B000CAF647510446F5F77DFA47F2F641C3F260
:10B6C0000F11F5F76FF92146F5F774FA4FF27C2167
:10B6D000C3F29341F5F764F92146F5F76BFA40F6AA
:10B6E0000151C3F2D071F5F75DF92146F5F762FA21
:10B6F00040F66131C3F6B621F5F752F92146F5F768
:10B7000059FA4AF6AB21C3F62A51F5F74BF921460F
:10B71000F5F750FA49F69913C3F699639E428046AD
:10B72000A3DD0020C3F64870864227DC06F17F4681
:10B730004FF07E503146F5F733F9814620464FF001
:10B740007C51F5F737FA3146F5F72AF941460646B6
:10B750002046F5F72FFA394604462846F5F72AFA27
:10B7600001462046F5F71CF901463046F5F718F971
:10B7700001464846F5F714F9BDE8F8834FF0000993
:10B780000026C3F63879C3F69066D7E74FF07E50AF
:10B79000BDE8F8832DE9F04FDFB00C930C9D224BF0
:10B7A000689C0A91691ED61E48BF161D834653F831
:10B7B0002400F71027EAE7730890049104980D938A
:10B7C000089DDC43DDF834C002EBC4024119079246
:10B7D000C0EB0C0750D47E18699BC7EB06090136F5
:10B7E000002F03EB870522AC09F0010AC0F2FE82AC
:10B7F0002868F5F78BF90137B74220604FF004084D
:10B800003AD0BAF1000F26D0002FC0F2F18255F8DD
:10B810000800F5F77BF90137B74244F8080008F152
:10B82000040818D128E000BF2800010855F80800D6
:10B83000F5F76CF9013708F1040944F8080013D44E
:10B8400055F80900F5F762F90137B74244F80900E5
:10B8500009F1040810D0002FE8DA0020013708F1C0
:10B86000040944F80800EBD501370020B74244F83A
:10B87000090009F10408EED1089A002AC0F24585B2
:10B8800008990C9E8D004AAB5C19039549AF029450
:10B890004FEA860A049A002AC0F296820DF18808BF
:10B8A00008EB860555F8041CAAF10403DBF8000038
:10B8B000C3F38009F5F77EF901460020F5F772F829
:10B8C0000424043D544580462BD0B9F1000F0DD01F
:10B8D00055F8041DDBF80400F5F76CF90146404605
:10B8E000F5F760F80824544580461AD055F8041C32
:10B8F0005BF80400F5F75EF901464046F5F752F8AB
:10B900000434804655F8081C5BF80400F5F752F93A
:10B9100001464046F5F746F80434083D5445804654
:10B92000E4D1029847F8048F01368742B2D1039FD1
:10B930000EA9CE190996089EB2005EAB9D18002E86
:10B94000029255F8509C7DDD0DF5947C4FF06E51C0
:10B9500048460DACA7180CEB0205F5F72BF9F5F7E7
:10B96000EFFAF5F7D3F84FF087410190F5F722F998
:10B9700001464846F5F714F8F5F7E2FA0EAC2060F8
:10B980000198014655F8040DF5F70CF8BC428146C4
:10B99000C7F3800156D0E9B14FF06E51F5F70AF9BF
:10B9A000F5F7CEFAF5F7B2F84FF087410190F5F7C9
:10B9B00001F901464846F4F7F3FFF5F7C1FA019A99
:10B9C0000FAC2060114655F8040DF4F7EBFFBC42B4
:10B9D000814637D04FF06E514846F5F7EBF8F5F752
:10B9E000AFFAF5F793F84FF087418046F5F7E2F8A4
:10B9F00001464846F4F7D4FFF5F7A2FA41466060E5
:10BA000055F8040DF4F7CEFF4FF06E518146F5F76F
:10BA1000D1F8F5F795FAF5F779F84FF087418046B8
:10BA2000F5F7C8F801464846F4F7BAFFF5F788FA83
:10BA30004146A06055F8040DF4F7B4FF0834BC4249
:10BA40008146C7D10799484600F0A2FE4FF07851D1
:10BA50000546F5F7AFF800F025FE4FF08241F5F707
:10BA6000A9F801462846F4F79BFF0746F5F768FA60
:10BA70008146F5F74BF801463846F4F791FF0799F0
:10BA80000746002940F33981721E0EAC079D54F819
:10BA90002230C5F1080043FA00F101FA00F0C5F1C7
:10BAA00007041B1A43FA04F40DF1380C89444CF8CE
:10BAB0002230002C55DD002E09F1010940F394815C
:10BAC000029D0EABDDF808C053F8042B281F0DF1C2
:10BAD000380E00250EEB0C01C0F3800022B1C2F538
:10BAE000807243F8042C01258B4226D060B10F9A56
:10BAF0000433002D40F0F38022B1C2F5807543F885
:10BB0000045C01258B4218D053F8042B002D40F023
:10BB1000EC80C2F5807012B143F8040C012553F893
:10BB2000042B002D40F0DB80C2F58070002AE9D0A4
:10BB300001258B4243F8040CE6D1079900290DDD5D
:10BB4000012900F0E280022908D1701E0DF1380EA3
:10BB50005EF8202002F03F034EF82030022C00F067
:10BB6000E08038460021F5F7B9F9002800F0F380AD
:10BB70000898751EA84225DC029B0DF1380E0EEBCD
:10BB800003010B46DDF824C053F8042DCCEB010073
:10BB9000011F6345C1F3800011D030B153F8041D7B
:10BBA000DDF824E00A43734509D0099F53F8040DDA
:10BBB00053F8041D0243BB4242EA0102F6D1002AB7
:10BBC00040F01A81089F0EAD781E55F82020002AFB
:10BBD00040F0108105EB8004012354F8041D01336B
:10BBE0000029FAD0F018771C87420B9075DCDDF83D
:10BBF00010E00D9D0B9B0C9C0EEB0702DDF808C0BE
:10BC0000699F991B06EB05094AA8A61922AB07EB09
:10BC1000890900EB0C05571C8A0003EB860102958D
:10BC200006920591002659F8040FF4F76FFF059C62
:10BC3000A051049800285EDB22AD05EB8702AAF133
:10BC40000403C3F3800452F8041CDBF800000394DF
:10BC5000141FF4F7AFFF01460020F4F7A3FE4FF0E6
:10BC60000408D04505462DD0039971B154F8041D40
:10BC7000DBF80400F4F79EFF01462846F4F792FE35
:10BC80004FF00808D04505461CD054F8041C5BF85A
:10BC90000800F4F78FFF01462846F4F783FE08F109
:10BCA0000408054654F8081C5BF80800F4F782FF06
:10BCB00001462846F4F776FE08F10408083CD04512
:10BCC0000546E2D1DDF808E0069804364EF8045F38
:10BCD00001378642CDF808E0A5D10B9E2CE6C2F1D3
:10BCE000FF0243F8042C01250CE7C2F1FF0543F8DD
:10BCF000045C012513E70025E4E75ED1701E0DF119
:10BD0000380E5EF820301C12D3E6711E0DF1380C8F
:10BD10005CF82100022C00F07F024CF821207FF417
:10BD200020AF39464FF07E50F4F73AFE0746002D1B
:10BD30003FF417AF07994FF07E5000F029FD014600
:10BD40003846F4F72DFE074638460021F5F7C6F8C9
:10BD500000287FF40DAF0294079C38466142CDF86D
:10BD6000109000F015FD4FF087410546F5F7D4F827
:10BD7000002800F0D2824FF06E512846F4F71AFFE7
:10BD8000F5F7DEF8F4F7C2FE4FF087410746F4F707
:10BD900011FF01462846F4F703FEF5F7D1F80EA986
:10BDA00041F826003846F5F7CBF8079A01360832F5
:10BDB0000EAC079244F8260034E04FF07C51F5F7C2
:10BDC000ABF858B90024CCE64FF00008029847F8C9
:10BDD000048F013687427FF45DADA8E50224002E72
:10BDE00009F101093FF76CAE0025A6E6002002E547
:10BDF000002010E50123F5E6079A0EAE56F825302F
:10BE0000083ACDF8109002940792002B40F08E82F1
:10BE100006EB85042E4654F8045D013E083A002DD9
:10BE2000F9D007924FF07E50079900F0B1FC002E38
:10BE30000446C0F2AC804FEA860AC6EB867B0EAFA2
:10BE40004FEA8B095744C9F100034AA9386801EB4E
:10BE50000A08C3F3800BF4F759FE2146F4F7AAFE53
:10BE60004FF06E51C8F800002046F4F7A3FEA9F188
:10BE700004096FF0030ACA45054631D0BBF1000F33
:10BE80000BD057F8040CF4F741FE2946F4F792FE64
:10BE90006FF0070A48F8040C1AE057F80A00F4F7A4
:10BEA00035FE2946F4F786FE4FF06E5148F80A0039
:10BEB0002846F4F77FFEAAF1040405463859F4F742
:10BEC00025FE2946F4F776FEAAF1080A48F8040090
:10BED00028464FF06E51F4F76DFECA450546DCD199
:10BEE000701CDFF84C94DDF820A003900027059625
:10BEF000BAF1000FC0F20582002FC0F202820026C4
:10BF000000241AF0010F354620D0D8F80010D9F8D7
:10BF10000000F4F74FFE01462046F4F743FD0125EB
:10BF2000AA45044626DB0426BD420FDD22E0BB45C0
:10BF300020DC58F8021059F80200F4F73BFE0146E5
:10BF40002046F4F72FFDBD42044613DC58F80610D6
:10BF500059F80600F4F72EFE01462046F4F722FDBC
:10BF600005F1010B06F104020235DA45044602F13F
:10BF70000406DCDA5EABDDF80CC003EB87010137A9
:10BF8000674541F8A04CA8F10408B1D1059E689C12
:10BF9000032C16D8DFE814F085011F011F011B00D8
:10BFA00000230299002900F00B81379C369804F198
:10BFB00000420A9C00F1004503F1004325606260E5
:10BFC000A360049D05F007005FB0BDE8F08F002E70
:10BFD000E6DD06F1FF3836AF07EB88094D4655F828
:10BFE00004290DF1D40AD5F808B01046594601923B
:10BFF000F4F7D8FC804641460198F4F7D1FC01469D
:10C000005846F4F7CFFC5545C9F38003A860C5F83E
:10C01000048044D0BBB155F80429D5F808B01046C7
:10C0200059460192F4F7BEFC019980460846414604
:10C03000F4F7B6FC01465846F4F7B4FC5545C5F88C
:10C040000480A8602BD02C4654F80439D4F808B0EA
:10C05000184659460193F4F7A5FC804641460198DD
:10C06000F4F79EFC01465846F4F79CFCC4F80480A3
:10C07000A06055F804BC251FD5F8088058464146F5
:10C08000F4F790FC044621465846F4F789FC014633
:10C090004046F4F787FC55456C60A860D3D1012E6B
:10C0A0007FF77EAF4D4655F804B9C7EB090ED5F8BA
:10C0B00008A058465146AEF10409F4F773FC8046D7
:10C0C00041465846F4F76CFC01465046F4F76AFCCA
:10C0D000BD42C9F38009C5F80480A86043D0B9F116
:10C0E000000F15D055F804A9D5F8089050464946D8
:10C0F000F4F758FC804641465046F4F751FC01469F
:10C100004846F4F74FFCBD42C5F80480A8602AD029
:10C110002C4654F804A9D4F8089050464946F4F740
:10C1200041FC804641465046F4F73AFC01464846F9
:10C13000F4F738FCC4F80480A06055F8049C251F6F
:10C14000D5F8088048464146F4F72CFC04462146C1
:10C150004846F4F725FC01464046F4F723FCBD426F
:10C160006C60A860D4D1013607EB860708353E46DF
:10C170007A1B131F56F8041D0020C3F38007F4F741
:10C1800011FCAE4203463FF40CAF3FB156F8041D1C
:10C19000F4F708FCAE4203463FF403AF184656F8E6
:10C1A000041C341FF4F7FEFB083E54F8041CF4F79B
:10C1B000F9FBAE42F3D10299034600297FF4F5AEB4
:10C1C000DDF828C036993798CCF80010CCF8040078
:10C1D000CCF80830F5E60023002E29DB36AF751CBD
:10C1E00007EB85042546E21B55F8041DA2F1040E59
:10C1F0000020CEF38008F4F7D5FBBD42034617D0EC
:10C20000B8F1000F06D055F8041DF4F7CBFBBD4282
:10C2100003460DD0184655F8041C2C1FF4F7C2FB3A
:10C22000083D54F8041CF4F7BDFBBD42F3D10346AE
:10C230000299002967D003F10040DDF828C01946B3
:10C24000CCF800003698F4F7ABFB002E034621DD56
:10C2500036AF07EB8606F51B2A1F3799C2F3800716
:10C26000F4F7A0FB37ACB442034613D037B1616892
:10C27000F4F798FB38ACB44203460BD0184654F898
:10C28000041FF4F78FFB54F8041FF4F78BFBB44240
:10C29000F5D10346029909B103F100430A9C63609A
:10C2A0008FE6002E40DB36AF013607EB86000546F1
:10C2B000C21B55F8041D0020141FF4F773FBBD4288
:10C2C000C4F38006034615D036B155F8041DF4F7C3
:10C2D00069FBBD4203460DD0184655F8041C2C1FBF
:10C2E000F4F760FB083D54F8041CF4F75BFBBD4217
:10C2F000F3D10346029909B103F100430A9C23607C
:10C300005FE6002436E6184697E7DDF830E0900057
:10C3100003904FEA8E0AFFF70ABB2846F4F710FE97
:10C320000EAB43F826007DE50023E3E72E4679E5D2
:10C33000340001082DE9F84320F00043B3F1485FD1
:10C3400004460F46904603DAF4F7FAFD002859D068
:10C3500021462046F4F72EFC21460546F4F72AFC38
:10C360004CF6D311C2F62E7106462846F4F722FC8D
:10C3700042F63471C3F2D721F4F712FB2946F4F7E1
:10C3800019FC4EF61B71C3F23861F4F70BFB29461A
:10C39000F4F710FC40F60151C3F65011F4F700FB1E
:10C3A0002946F4F707FC48F68901C3F60841F4F77B
:10C3B000F9FA8146B8F1000F27D04FF07C5138468A
:10C3C000F4F7F8FB494680463046F4F7F3FB0146A4
:10C3D0004046F4F7E5FA2946F4F7ECFB3946F4F762
:10C3E000DFFA4AF6AB210546C3F62A613046F4F778
:10C3F000E1FB01462846F4F7D5FA01462046F4F75A
:10C40000CFFA04462046BDE8F88301462846F4F7F3
:10C41000D1FB4AF6AB21C3F62A61F4F7C1FA3146E3
:10C42000F4F7C8FB01462046F4F7BCFA0446204660
:10C43000BDE8F8830020704700210020C7F6F8719E
:10C44000704700BF2DE9F04120F00045B5F1A14F44
:10C45000044606460DDBB5F1FF4F00F39C80002833
:10C4600040F6DB7440F3D480C3F6C9742046BDE8BF
:10C47000F0814FF6FF73C3F6DF639D4200F3A280A5
:10C48000B5F1445FC0F28E804FF0FF372146204661
:10C49000F4F790FB01468046F4F78CFB46F6D71183
:10C4A000C3F685410546F4F785FB4DF65921C3F6E1
:10C4B0004B51F4F777FA2946F4F77CFB46F6353111
:10C4C000C3F68851F4F76EFA2946F4F773FB42F687
:10C4D0006E61C3F6BA51F4F765FA2946F4F76AFBC0
:10C4E00044F62511C3F61261F4F75CFA2946F4F715
:10C4F00061FB4AF6AB21C3F6AA61F4F753FA414651
:10C50000F4F758FB4AF221218046CBF61551284614
:10C51000F4F750FB4FF26B11C3F66E51F4F740FA8B
:10C520002946F4F747FB48F29571C3F69D51F4F79D
:10C5300037FA2946F4F73EFB48F63861C3F6E35173
:10C54000F4F72EFA2946F4F735FB4CF6CD41C3F645
:10C550004C61F4F725FA2946F4F72CFB7B1C0146C5
:10C56000404658D0F4F71EFA2146F4F723FB494B16
:10C5700053F82710F4F714FA2146F4F711FA01469C
:10C58000454850F82700F4F70BFA002E3DDB04462F
:10C590002046BDE8F0810146F4F704FA044620463F
:10C5A000BDE8F0814FF2CA21C7F24911F4F7FAF958
:10C5B0004FF07E51F4F7BAFC00283FF465AF2046F7
:10C5C000BDE8F08100F06AF84FF6FF71C3F697718D
:10C5D0008D4204464FF6FF7228DCC3F62F72954257
:10C5E00046DC0146F4F7DEF94FF07E51F4F7D8F956
:10C5F0004FF0804105462046F4F7D4F9014628461D
:10C60000F4F78CFB0027044640E700F100442DE7D7
:10C61000CBF6C9742AE7F4F7C5F92146F4F7CAFA4C
:10C6200001462046F4F7BCF904461FE7C4F21B029A
:10C63000954214DC4FF07F51F4F7B2F94FF07F517F
:10C6400005462046F4F7B6FA4FF07E51F4F7AAF902
:10C6500001462846F4F762FB0227044616E700204D
:10C660002146CBF68070F4F759FB032704460DE70B
:10C670004FF07E51F4F794F94FF07E510746204673
:10C68000F4F790F901463846F4F748FB01270446D1
:10C69000FCE600BF600001087000010820F00040C7
:10C6A000704700BFF8B520F00046F50D7F3D162D10
:10C6B000014604461BDC002D074620DB4FF6FF73C6
:10C6C000C0F27F0343FA05F606420ED04FF2CA21AC
:10C6D000C7F24911F4F766F90021F4F727FC18B105
:10C6E000002C1BDB27EA060421460846F8BDB6F1FC
:10C6F000FF4FFAD3F4F756F901460846F8BD4FF25A
:10C70000CA21C7F24911F4F74DF90021F4F70EFCE4
:10C710000028E9D0002C07DB0024E5E74FF40000F7
:10C7200040FA05F56719DDE70021CBF68071002E90
:10C7300018BF0C46D8E700BF08B902207047B0F117
:10C74000004FFAD0A0F500026FF001439A4201D8E1
:10C750000420704700F1FF419942F9D94FF6FE736A
:10C76000421EC0F27F039A4201D80320704700F1B5
:10C7700000414A1E9A42F8D9B0F1FF4F05D010F59A
:10C78000000F14BF0020012070470120704700BF38
:10C7900038B530F00044034602460D460FD0B4F1E0
:10C7A000FF4F0ED2B4F5000F11D3E40D6419FE2C27
:10C7B00033DC002C1BDD22F0FF4141EAC453184654
:10C7C00038BD0146F4F7EEF80346184638BD4FF081
:10C7D0009841F4F7EFF943F6B041CFF6FF718D427F
:10C7E000034612DBC0F3C7540246193CDEE714F1DE
:10C7F000160F21DA4CF25032954219460EDC44F203
:10C800006020C0F6A25000F023F844F26021C0F688
:10C81000A251F4F7CFF90346D1E719464FF2CA20E7
:10C82000C7F2491000F014F84FF2CA21C7F24911BB
:10C83000F4F7C0F90346C2E722F0FF4304F1190000
:10C8400043EAC0504FF04C51F4F7B4F90346B6E751
:10C8500001F0004120F00040084370472DE9F0410D
:10C86000274C84B025680746D5F84841002C41D0B4
:10C8700066681F2E1CDD234810B94FF0FF301FE003
:10C880004FF4C870039102920193AFF300800399B3
:10C890000446029A019B0028EFD0D5F84861002099
:10C8A00060602660C5F84841C4F88801C4F88C016E
:10C8B000656847B9A81C013544F820106560002060
:10C8C00004B0BDE8F081012000FA05F0D4F88861D9
:10C8D00004EB85080643022FC8F88820C4F8886155
:10C8E000C8F80831E6D1D4F88C3143EA0002C4F824
:10C8F0008C21DFE705F5A674C5F84841B8E700BF0D
:10C90000880101080000000000210A2201F028B877
:10C910002DE9F84FDDF828B081468A4698469AB14D
:10C9200093B11646002503E00FD0651CAE420BD92B
:10C930007419640808FB04A748463946D8470028FC
:10C94000F2DA2646AE42F3D800273846BDE8F88F23
:10C9500040F2D053C2F2000318687047114B124ADC
:10C9600070B5981A831018D0591E02EB83040D4637
:10C9700054F8042D01F00106904775B126B154F822
:10C98000040D8047013D08D054F8043D9847013D0F
:10C9900054F8041D8847013DF6D1BDE8704003F00E
:10C9A000FBBB00BFB0010108AC010108F8B5204F86
:10C9B000204C381B871017D07A1E2368012502F0FF
:10C9C00001069847AF420FD02EB154F8041F02253C
:10C9D0008847AF4208D0606880470235A268261DAC
:10C9E00090470834AF42F6D1134F144C03F0CEFBFE
:10C9F0003B1B9F1018D07D1E216805F00106012504
:10CA00008847AF4211D02EB154F8040F0225804759
:10CA1000AF420BD0626890470235A368261D984745
:10CA20000834AF42F6D1F8BDF8BDF8BDF8BD00BF7F
:10CA3000A4010108A4010108AC010108A401010836
:10CA40000F2A2DE9F00340F2A18041EA00039B0781
:10CA500040F09E800C68A2F1100504604B68AC4663
:10CA600043608C68BCF10F0F8460CC68C5F300157F
:10CA7000C46000F1100301F110042BD975B12568D1
:10CA8000ACF1100C1D6065685D60A5689D60E5688F
:10CA90001034DD601033BCF10F0F1BD9276804F18F
:10CAA00010061F60676803F110055F60A768ACF1AE
:10CAB000200C9F60E768DF6024691C61776806F1DD
:10CAC00010046F60B7682033AF60F668BCF10F0FD9
:10CAD000EE60E3D8A2F1100828F00F0302F00F0473
:10CAE00003F1100C032C00EB0C0301EB0C0851D9E3
:10CAF000211F4FEA9109444608EB890C54F8046B56
:10CB0000C8EB0C010CF1040C1D46644545F8046BA0
:10CB1000C1F3800112D029B154F8041B644545F8D3
:10CB2000041B0BD0274657F8041B2E4646F8041B5F
:10CB300064686C603C1D351D6445F3D109F1010C3E
:10CB40004FEA8C0902F0030208EB09014B44D2B111
:10CB50000D789A18DC4303F8015B1419934204F032
:10CB6000010410D02CB111F8014F03F8014B93428E
:10CB700009D04D781C4604F8015B8D7802315D7058
:10CB8000631C9342F5D1BDE8F00370470346DEE72E
:10CB90000346DDE741462246D9E700BFF0B48407EB
:10CBA000034600F08D80541E002A00F08780E507C0
:10CBB000CEB211D41A4602F8016B134615469207FD
:10CBC00010D0621E002C79D003F8016B14469A072E
:10CBD0001D4607D0013CEDE7034603F8016B9A07B9
:10CBE0001D46F7D1032C52D9CEB246EA06270F2CA8
:10CBF00047EA07432DD9A4F1100217460F2FC2F3BD
:10CC000000162B606B60AB60EB6005F1100216D96B
:10CC10003EB1103F136053609360D36010320F2F0A
:10CC20000DD9203F02F11006136053609360D3606A
:10CC3000136153619361D36120320F2FF1D8A4F1B6
:10CC4000100222F00F0204F00F041032032C1544DE
:10CC50001DD9271F3E462A46032E42F8043BC7F340
:10CC600080070DD927B1043E032E42F8043B07D9B3
:10CC7000174647F8043B083E53603A1D032EF7D889
:10CC8000231F23F00302131D04F00304ED18ACB1BD
:10CC9000C9B2EA432C1905F8011BA318A54203F0F9
:10CCA00001020BD01AB105F8011BA54206D02B4694
:10CCB00003F8011B69705D1CA542F8D1F0BC7047F8
:10CCC000054614468EE700BF830770B5064614D1AB
:10CCD0000368A3F1013222EA030010F0803F0CD177
:10CCE000331D1A4653F8044BA4F1013525EA040418
:10CCF00014F0803FF5D0104600E0304603782BB1A9
:10CD0000421C147810460132002CFAD100F080F851
:10CD1000304670BDC9B2F0B400294BD082070FD0A5
:10CD20000278002A71D0914242D0431C05E013F8EA
:10CD3000012B002A3BD091423AD09A071846F6D1EF
:10CD4000036841EA0127A3F1013222EA030212F04B
:10CD5000803F47EA07471CD17B40A3F1013222EA1A
:10CD6000030313F0803F14D1021D02E014F0803F52
:10CD70000FD1104652F8043BA3F1013687EA0304B1
:10CD800026EA0303A4F1013513F0803F25EA0404E9
:10CD9000ECD00278002A38D0914209D0431C01E03F
:10CDA000914205D0184613F8012B002AF8D11046FD
:10CDB000F0BC704783070BD00278002AF8D0431CE0
:10CDC00003E0017801330029F2D099071846F8D121
:10CDD0000168A1F1013323EA010212F0803F0AD178
:10CDE000031D184653F8041BA1F1013424EA010283
:10CDF00012F0803FF5D00378002BD9D0421C117877
:10CE0000104601320029FAD1D2E71046D0E700BF20
:10CE100080EA0102844612F0030F4FD111F0030F94
:10CE200032D14DF8044D11F0040F51F8043B0BD0F2
:10CE3000A3F101329A4312F0803F04BF4CF8043B47
:10CE400051F8043B16D100BF51F8044BA3F1013255
:10CE50009A4312F0803FA4F101320BD14CF8043B0D
:10CE6000A24312F0803F04BF51F8043B4CF8044B3E
:10CE7000EAD023460CF8013B13F0FF0F4FEA3323AF
:10CE8000F8D15DF8044B704711F0010F06D011F88E
:10CE9000012B0CF8012B002A08BF704711F0020F7C
:10CEA000BFD031F8022B12F0FF0F16BF2CF8022B67
:10CEB0008CF8002012F47F4FB3D1704711F8012B8A
:10CEC0000CF8012B002AF9D1704700BF20F00301B4
:10CED00010F00300C0F1000051F8043B00F1040C15
:10CEE0004FEACC0C6FF000021CBF22FA0CF2134385
:10CEF0004FF0010C4CEA0C2C4CEA0C4CA3EB0C024E
:10CF000022EA030212EACC1204BF51F8043B0430B7
:10CF1000F4D013F0FF0F1FBF013013F47F4F013027
:10CF200013F47F0F18BF0130704700BFF0B4002A20
:10CF300063D0344B04461B6814F8010B571E1D18B0
:10CF40006E7807F0010706F00305012D58D011F89F
:10CF5000015B5E19767806F00306012E08BF2035C6
:10CF6000401B4BD1002D49D0013A47D02FB314F8C4
:10CF7000010B1D186E7806F00305012D11F8015BF9
:10CF800008BF20305E19767806F00306012E08BF30
:10CF90002035401B32D18DB3013A0ED12EE011F86D
:10CFA000012B9E18767806F00306012E08BF20326A
:10CFB000801A23D112B36A1E20D014F8010B1D1859
:10CFC0006E7806F00305012D11F8015B08BF2030D3
:10CFD0005E19767806F00306012E08BF2035401B47
:10CFE0000CD15DB114F8010B551E1A18567806F0D5
:10CFF0000302012AD3D12030D1E71046F0BC70479C
:10D000002030A4E7A401002041EA00039B07F0B40C
:10D0100074D1032A72D90C4654F8045B161FA5F18B
:10D02000013727EA050717F0803F0346C6F3800C57
:10D0300031D10346032E324643F8045B2AD9BCF1B2
:10D04000000F0AD0214654F8045BA5F1013626EA08
:10D05000050616F0803F18D01DE0264656F8045B02
:10D060002146A5F1013727EA050717F0803F12D1C5
:10D0700043F8045B65683146A5F1013626EA0506EA
:10D08000043A0C1D16F0803F05D1043A032A43F8F8
:10D09000045BE2D821467AB30D78013A03F8015BCC
:10D0A0009DB112F0010F1C462AD1234622B311F87C
:10D0B000015F013A03F8015B3DB111F8015F013AEC
:10D0C00065705C1C2346002DEFD1AAB100219C188D
:10D0D000DA4303F8011BA218A34202F001020BD0AD
:10D0E0001AB103F8011BA34206D01A4602F8011B2D
:10D0F0005970531CA342F8D1F0BC70470346CAE7ED
:10D1000011F8015F1C4604F8015B013A2346002D2B
:10D11000CBD1DAE72DE9F00701273C4600254FF097
:10D12000FF3663198B4200EB060C0DD21CF804A0ED
:10D1300010F80380D0452ED201241D469F1B631991
:10D140008B4200EB060CF1D34FF0010A17605446F6
:10D1500000254FF0FF3C6319994200EB0C080ED9F3
:10D1600018F8048010F80390C1451AD901241D460F
:10D17000CCEB030A6319994200EB0C08F0D80CF1D0
:10D1800001000136B0423CBFBA463046C2F800A0AA
:10D19000BDE8F00770470BD001272E463C46ED193D
:10D1A000BFE709D04FF0010AAC4654465544D2E7D8
:10D1B000BC4205D00134B4E7544505D00134CAE778
:10D1C00027461D460124ACE7A2461D460124C2E7BE
:10D1D0002DE9F04FADF2244D15460646894610461E
:10D1E000194607AA1C46FFF795FF07AB82460DF2CA
:10D1F0001C411A1D5C6008338B425460F9D114B392
:10D2000001232F78611E08A8A34240F8271001EAE5
:10D21000030218D032B16A7802234F1EA34240F8AD
:10D22000227010D0B046A4465C1C15F803E0CE1A5C
:10D230002A5D02330F1B634540F82E6040F82270D0
:10D24000F2D146466446079928466918524600F0CE
:10D2500045FC002840F0B6800AF1FF3E05EB0E0CBD
:10D26000CDF808E0CAF1010E834604F1FF38CDF88D
:10D270000CC0CDF814E00746CDF810A04A46009542
:10D28000019408E027B1079FBB4201D20199CB1B53
:10D290009B4400272246019CB0185C440021A21A3E
:10D2A00000F07CFB002840F08780002C00F0848098
:10D2B000301910F8013C08A951F82330002BE1D1B6
:10D2C000049B9F4228BF3B46434527D2DDF8009090
:10D2D00006EB0B0119F80350CA5C09EB03009542F9
:10D2E00066D1DD43454415F0010F024613D00133EA
:10D2F000434513D24078CD5C013285420BD057E0D4
:10D3000012F8010FCD5C854252D1013312F8010FA2
:10D31000CD5C85424CD101334345F1D3DDF810900B
:10D32000029B4F4528BF4B4639D2DDF808C0DDF8D7
:10D33000009006EB0B0519F80C1015F80C00814253
:10D3400040F0C080DDF80CE009EB070ACAEB0E01E3
:10D35000C80772461ED5DDF8089009F1FF31DDF8E7
:10D360000C90685C19F801CC09F1FF32844516D1A4
:10D370000B460FE012F8019C15F800E04A1EF1453B
:10D380000DD10346013815F800C011F8011C6145A4
:10D3900005D10346581E524502F1FF31EAD101374B
:10D3A0009F4200F29180079F019ABB44D71B71E70F
:10D3B000DDF814E0F3446BE7002009B00DF5806D53
:10D3C000BDE8F08FCAEB0400504538BF5046CAF1A3
:10D3D0000102431C0AF1FF3C05EB0A0704F1FF3B85
:10D3E000019200944A460793B1464FF00008644604
:10D3F0003E46009909EB020008EB0107BA1A00212A
:10D4000000F0CCFA0028D7D1002FD5D009EB0700C7
:10D4100010F8013C08AA52F8230000284AD1DA4546
:10D4200009EB08002AD210F80A303178994218BF67
:10D43000534642D16FEA0A0303EB0B01C907324698
:10D44000534618D50AF101035B4517D2324612F84C
:10D45000011F10F803E08E450DD02EE012F8011FD9
:10D4600010F803C08C4528D1013312F8011F10F8C1
:10D4700003E08E4521D101335B45EFD3621C234687
:10D480009BD0295D025D914213D1E10709D5631E4E
:10D49000E95CC25C914204D00BE0E95CC25C914261
:10D4A00007D15A1E002B88D0A95C825C023B9142B6
:10D4B000F3D0079880443A469BE7DDF804C0E04487
:10D4C0009844F8E7049B6AE706EB0B0075E700BF9A
:10D4D0002DE9F04F037889B080460D46002B00F00F
:10D4E00065810A789AB184460131012602E011F87B
:10D4F000012B5AB1934214BF002606F001061CF816
:10D50000013F0C46002BF2D1207820B936B14046BD
:10D5100009B0BDE8F08F4FF00008F8E708F101000E
:10D520002978FFF7F7FB641B06460028F3D0012C8F
:10D5300000F0B580A044404594BFC0EB0807012728
:10D540001F2C06D939462A462346FFF741FE80465E
:10D55000DDE7214607AA2846FFF7DCFD079903907F
:10D5600069182846039A00F0B9FA002840F099801B
:10D57000DDF80CC0DDF80C900CF1FF3E05EB0E0160
:10D58000C9F1010C8346CDF808E080460491CDF83E
:10D5900014C03A46B146019508EB040609EB0200B7
:10D5A0000021B21A00F0FAF90028B4D1002EB2D04E
:10D5B000039B9B4528BF5B469C4227D9019D09EBF5
:10D5C000030010F80820E95CE81891425FD1DD43C0
:10D5D0002D1915F0010F024609EB080113D0013394
:10D5E0009C4213D94078CD5C013285420BD04EE08D
:10D5F00012F8010FCD5C854249D1013312F8010FB9
:10D60000CD5C854243D101339C42F1D8DDF80CE07A
:10D61000029ADE4540F2CD80019B09EB0805995C3A
:10D62000A85C814240F0C580DDF804A0049BDA4488
:10D63000CAEB0301C8071AD5029FDDF810C0791E96
:10D64000685C1CF8017C0CF1FF33874214D10A4658
:10D650000DE013F801EC2F5C4B1EBE450CD10246C9
:10D6600001382F5C11F8011CB94205D10246501E49
:10D67000534503F1FF31ECD10BF1010B934500F25F
:10D680009A80079A9044C2EB040B324684E7059DCA
:10D6900005EB080B0BEB03084FF0000BF5E780469A
:10D6A00035E7DDF80CA00399CAEB0403534538BFF6
:10D6B0005346CAF1010B581C06EB0A0205EB0A0897
:10D6C000CDF808B03B4607904FF00009019201F1F8
:10D6D000FF3B37468A4609EB0406F8180021F21A88
:10D6E00000F05CF900287FF416AF002E3FF413AF72
:10D6F000544598BF07EB09002CD9DDF804E098F8F1
:10D7000000001EF8093098424AD16FEA0A02111946
:10D71000C9074246534607EB090018D50AF1010331
:10D720009C4217D9424612F8011F10F803C08C45DD
:10D730000DD036E012F8011F10F803E08E4530D10D
:10D74000013312F8011F10F803C08C4529D10133B1
:10D750009C42EFD8BBF1FF3F5B463FF4F8AE15F8B3
:10D760000B1010F80B20914216D11BF0010F0AD0BC
:10D770000BF1FF33E95CC25C914204D00CE0E95C40
:10D78000C25C914208D15A1E002B3FF4E0AEA95C66
:10D79000825C023B9142F2D00798814433469AE77B
:10D7A0005346DDF808E0F1449944F7E70C460126BA
:10D7B000AAE6039A60E74E46C844A8E640F2D05372
:10D7C000C2F200031A6801235C3200F001B800BF06
:10D7D000F0B4002825D0074638463E780D4601377C
:10D7E00015F8014B3CB1A642FAD1002BF4D11760D9
:10D7F00007F8013C11E0C6B13D4600E01BB915F841
:10D80000016B0C46284614F8013B9E42F6D136B116
:10D81000002105F8011C1060781EF0BC70473046EE
:10D82000F9E710680028D6D1F7E716603046F4E72C
:10D830002DE9F00F494C82B0D4F800C001900F469A
:10D840003C4614F8015B0CEB05004678274606F0D1
:10D850000800C6B2002EF3D12D2D61D02B2D04BFB0
:10D86000244614F8015BB346002B41D1302D43D040
:10D870000A239A46BBF1000F0CBF6FF000474FF030
:10D880000047B7FBFAF90AFB1970009000208046A8
:10D890000CE0303DAB421BDD461C05D0C84539D8F5
:10D8A00035D00AFB0858012014F8015B0CEB050683
:10D8B000767806F00407FFB2002FEAD116F00306CF
:10D8C00006D0012E14BF57263726AD1BAB42E3DC32
:10D8D000431C2AD0BBF1000F01D0C8F10008002A78
:10D8E00031D0D0B94046116002B0BDE8F00F7047AA
:10D8F000102BBED1302DBCD12578782D25D0582DB8
:10D9000023D043BB4FF0080A30255346B2E70098B6
:10D910008542C6DD4FF0FF30C6E74046611EE2E7B4
:10D9200014F8015B4FF0010B9EE7BBF1000F01996A
:10D930000CBF6FF000404FF0004022230B60002A24
:10D94000D2D0611ECFE74046CEE74FF0100A65788F
:10D95000534602348EE79A4630258BE7A401002017
:10D9600070B440F2D054C2F2000406460D4620685E
:10D97000134631462A4670BCFFF75ABF024B13B11B
:10D98000024800F005B87047000000005DC90008BB
:10D990000146002002460346FEF760BF8307F0B44D
:10D9A000C9B200F09680531E002A00F094800278DD
:10D9B0008A420BD0421CD8071AD512F0030F10462A
:10D9C0001CD01478013B01328C4211D1F0BC70475D
:10D9D000002B7CD01278013B8A42F7D014F0030F61
:10D9E000204604F1010209D02478013B8C42EDD09D
:10D9F00012F0030F104602F10104E9D1032B3FD9C5
:10DA0000046841EA012545EA054585EA0407A7F1CE
:10DA1000013222EA07021E1F041D12F0803FC6F3E6
:10DA200080072DD1032E334629D967B126682046B9
:10DA300085EA0602A2F1013626EA0202043412F057
:10DA4000803F19D01CE020462468061D85EA0402A8
:10DA5000A2F1013424EA020212F0803F10D13468AE
:10DA6000043B85EA0402A2F1013424EA0202341DD7
:10DA700012F0803F304603D1043B032BE3D820460D
:10DA80005D1E23B303788B42A0D0431C0022E8071D
:10DA900014D51C781846012201338C4296D0954249
:10DAA000184603F1010402F102020ED01B788B42EA
:10DAB0008CD020462478431C8C4287D0954218464F
:10DAC00003F1010402F10202F0D100207EE71846C2
:10DAD0007CE7134692E7104678E700BF032AF0B4CC
:10DAE00031D941EA00039C072ED106680F68151F43
:10DAF000031D0C1DBE42C5F3800C24D1032D2A4604
:10DB00001FD9BCF1000F08D01E68256821461846B1
:10DB100004340433AE4211D015E0214618461C6887
:10DB20000B68051D0E1D9C420DD1314628462E68FE
:10DB30000D68043A031D0C1DAE4204D1043A032AB9
:10DB4000EBD8214618461AB303780C78A3420AD1C1
:10DB5000551E0022EB0714D510F8013F11F8014FB4
:10DB60000122A3420DD0181B10E010F8013F11F85C
:10DB7000014FA342F7D110F8013F11F8014FA34222
:10DB8000F1D1AA4202F10202EFD10020F0BC7047AD
:10DB90001046FBE71E1E6464646464640010014068
:10DBA00000101002000801400080100234080040FC
:10DBB000380800403C080040400800403404004061
:10DBC000380400403C04004040040040D0073200CC
:10DBD000320032003200320032003200C8006400ED
:10DBE0000000414554523132333400001D260008F4
:10DBF000A1260008612600083D26000879260008B5
:10DC0000FD26000829260008A73D0008CF3C000893
:10DC1000773D00082D3D0008E53C0008CD3C00089C
:10DC20000000803F00000000A8AAAA3F0000803F3B
:10DC30000000803F000080BFB0AA2ABF000080BF64
:10DC40000000803F0000803FB0AA2ABF000080BFD4
:10DC50000000803F00000000A8AAAA3F000080BF8B
:10DC60000000803F000080BFB0AA2ABF0000803FB4
:10DC70000000803F0000803FB0AA2ABF0000803F24
:10DC80000000803F00000000A8AAAA3F000000009A
:10DC90000000803F000080BFB0AA2ABF0000000043
:10DCA0000000803F0000803FB0AA2ABF00000000B3
:10DCB0000000803F000080BF0000803F000080BF68
:10DCC0000000803F000080BF000080BF0000803F58
:10DCD0000000803F0000803F0000803F0000803F48
:10DCE0000000803F0000803F000080BF000080BF38
:10DCF0000000803F00000000000000000000000065
:10DD00000000803F00000000000000000000000054
:10DD10000000803F000000000000803F0000803FC6
:10DD20000000803F000080BF000080BF00000000B6
:10DD30000000803F000000000000803F000080BF26
:10DD40000000803F0000803F000080BF0000008096
:10DD50000000803F000000000000803F000080BF06
:10DD60000000803F000080BF000000000000803FF6
:10DD70000000803F0000803F000000000000803F66
:10DD80000000803F00000000000080BF000080BF56
:10DD900000000000000000000301000080DC00081B
:10DDA0000400000050DD00080400000088DF0008C7
:10DDB0000201000028DF0008000100000000000050
:10DDC0000600000020DC000806000000C8DE000895
:10DDD00001010000000000000400000048DF00080E
:10DDE0000600000048E0000808000000A8E0000865
:10DDF0000800000048DE000808000000C8DF000836
:10DE0000010100000000000000010000000000000F
:10DE100000010000000000000400000010DD000808
:10DE200006000000B0DC0008000100000000000057
:10DE30000201000028E100080101000000000000CC
:10DE400000000000000000000000803FF704353FA4
:10DE5000F70435BF0000803F0000803FF70435BF66
:10DE6000F70435BF0000803F0000803FF70435BF56
:10DE7000F704353F0000803F0000803FF704353F46
:10DE8000F704353F0000803F0000803F00000000A5
:10DE9000000080BF000080BF0000803F000080BF06
:10DEA00000000000000080BF0000803F0000000074
:10DEB0000000803F000080BF0000803F0000803FE6
:10DEC00000000000000080BF0000803FD0B35DBFB5
:10DED0000000003F0000803F0000803FD0B35DBFE6
:10DEE000000000BF000080BF0000803FD0B35D3F56
:10DEF0000000003F0000803F0000803FD0B35D3F46
:10DF0000000000BF000080BF0000803F0000000054
:10DF1000000080BF0000803F0000803F0000000044
:10DF20000000803F000080BF0000803F0000803F75
:10DF300000000000000000000000803F000080BFE3
:10DF400000000000000000000000803F0000000012
:10DF50000000803F000080BF0000803F000080BFC5
:10DF6000000080BF000000000000803F00000000B3
:10DF70000000803F0000803F0000803F0000803FA5
:10DF8000000080BF000000000000803F000080BF54
:10DF90000000803F000080BF0000803F000080BF85
:10DFA000000080BF0000803F0000803F0000803FF5
:10DFB0000000803F0000803F0000803F0000803F65
:10DFC000000080BF000080BF0000803F0000803F55
:10DFD000000000BF0000803F0000803F000000BF45
:10DFE000000080BF0000803F0000803F000080BF35
:10DFF0000000003F0000803F0000803F0000003F25
:10E000000000803F0000803F0000803F0000003F94
:10E01000000080BF000080BF0000803F000080BF84
:10E02000000000BF000080BF0000803F000000BF74
:10E030000000803F000080BF0000803F0000803F64
:10E040000000003F000080BF0000803F000000BFD4
:10E05000D0B35D3F0000803F0000803F000000BF64
:10E06000D0B35DBF0000803F0000803F0000003F54
:10E07000D0B35D3F000080BF0000803F0000003F44
:10E08000D0B35DBF000080BF0000803F000080BFB4
:10E0900000000000000080BF0000803F0000803FC3
:10E0A000000000000000803F0000803F000080BFB3
:10E0B0000000803F000080BF0000803F000080BF64
:10E0C000000080BF0000803F0000803F0000803FD4
:10E0D0000000803F0000803F0000803F0000803F44
:10E0E000000080BF000080BF0000803F000080BFB4
:10E0F0000000803F0000803F0000803F000080BFA4
:10E10000000080BF000080BF0000803F0000803F13
:10E110000000803F000080BF0000803F0000803F83
:10E12000000080BF0000803F0000803F0000000032
:10E1300000000000000080BF0000803F00000000E1
:10E14000000000000000803F24505542582C34311C
:10E150002C312C303030332C303030312C313135C3
:10E160003230302C302A31450D0A0024504D544BAA
:10E170003235312C3131353230302A31460D0A00FA
:10E1800024505542582C34312C312C303030332C23
:10E19000303030312C35373630302C302A32440D87
:10E1A0000A0024504D544B3235312C35373630303F
:10E1B0002A32430D0A0024505542582C34312C3158
:10E1C0002C303030332C303030312C333834303048
:10E1D0002C302A32360D0A0024504D544B32353142
:10E1E0002C33383430302A32370D0A00245055424F
:10E1F000582C34312C312C303030332C30303031FD
:10E200002C31393230302C302A32330D0A00245070
:10E210004D544B3235312C31393230302A32320DB7
:10E220000A00B56206010300F00500FF19B5620699
:10E23000010300F00300FD15B56206010300F001C3
:10E2400000FB11B56206010300F00000FA0FB56291
:10E2500006010300F00200FC13B56206010300F0A2
:10E260000400FE17B562060103000102010E47B566
:10E2700062060103000103010F49B56206010300B4
:10E28000010601124FB562060103000112011E676B
:10E29000B5620616080003070300510800008A4112
:10E2A000B56206080600C80001000100DE6A000031
:10E2B0000000000000C2010048E100086BE1000816
:10E2C0000100000000E1000080E10008A2E1000878
:10E2D0000200000000960000B6E10008D8E1000846
:10E2E00003000000004B0000ECE100080EE2000813
:10E2F000040000008025000022EA000822EA00084D
:10E3000041455254313233340000000053F20008CA
:10E3100057F200085CF200086DF2000876F200087F
:10E3200081F200088CF2000897F2000875F10008ED
:10E33000A0F200086FF10008A9F20008B3F200088B
:10E34000BEF20008C4F2000800000000A5F10008B9
:10E35000A9F10008AFF10008B5F10008B8F1000814
:10E36000BFF10008C2F10008C7F10008D3F10008AE
:10E37000D6F10008DCF10008E3F10008EDF1000837
:10E38000F7F1000800F200080EF200081AF2000887
:10E3900021F2000827F2000834F200083FF20008DA
:10E3A0004CF2000800000000B7EF0008BBEF0008C7
:10E3B0007D810008E2EF0008E7EF00087986000899
:10E3C000FBEF000804F00008D17F000821F00008EE
:10E3D00026F00008C584000855F0000822EA00086D
:10E3E000997F00085AF0000862F00008AD7E00082E
:10E3F00076F0000885F000088D7E00089FF0000888
:10E4000022EA0008817C0008A4F00008A8F00008B7
:10E41000E57D0008F5EF0008C4F00008E97F00087A
:10E42000D7F00008DDF00008D5800008F8F00008FB
:10E4300000F10008898000080FF1000814F10008BD
:10E44000BD7D000833E9000824F10008718300084D
:10E4500052F1000846F10008AD7C000859F10008AF
:10E4600022EA0008757C000822EA000881F1000811
:10E4700089F1000891F1000899F10008A0F1000865
:10E4800000000000303132333435363738394142FC
:10E49000434445464748494A4B4C4D4E4F505152D4
:10E4A000535455565758595A004166726F333220AB
:10E4B000434C492076657273696F6E20322E32208C
:10E4C0004170722032322032303134202F203032ED
:10E4D0003A34363A343400417661696C61626C6575
:10E4E00020636F6D6D616E64733A0D0A00257309C8
:10E4F00025730D0A0053797374656D205570746926
:10E500006D653A202564207365636F6E64732C20FB
:10E51000566F6C746167653A202564202A20302E7E
:10E5200031562028256453206261747465727929FC
:10E530000D0A004350552025644D487A2C2064650F
:10E540007465637465642073656E736F72733A20CB
:10E55000002573200041434348573A202573002E7D
:10E560002563004379636C652054696D653A202505
:10E57000642C20493243204572726F72733A202511
:10E58000642C20636F6E6669672073697A653A2030
:10E5900025640D0A000D0A5265626F6F74696E671B
:10E5A0002E2E2E00536176696E672E2E2E004D752D
:10E5B000737420626520616E79206F7264657220C9
:10E5C0006F662041455452313233340D0A00437591
:10E5D0007272656E742061737369676E6D656E74B7
:10E5E0003A20004572726F723A20456E61626C6526
:10E5F00020616E6420706C756720696E20475053EF
:10E600002066697273740D0A00456E61626C696EF2
:10E61000672047505320706173737468726F756719
:10E62000682E2E2E0D0A00456E61626C65642066B0
:10E63000656174757265733A2000417661696C6139
:10E64000626C652066656174757265733A20004975
:10E650006E76616C69642066656174757265206EA2
:10E66000616D652E2E2E0D0A0044697361626C6522
:10E67000642000456E61626C656420000D0A4C6583
:10E680006176696E6720434C49206D6F64652E2E5C
:10E690002E0D0A00526573657474696E6720746F7D
:10E6A0002064656661756C74732E2E2E004375723E
:10E6B00072656E74206D697865723A2025730D0A53
:10E6C00000417661696C61626C65206D6978657284
:10E6D000733A2000496E76616C6964206D697865D3
:10E6E0007220747970652E2E2E0D0A004D697865A2
:10E6F000722073657420746F2025730D0A004375B2
:10E700007272656E742070726F66696C653A20254E
:10E71000640D0A0055736167653A0D0A6D6F746F79
:10E720007220696E646578205B76616C75655D202A
:10E730002D2073686F77205B6F72207365745D2086
:10E740006D6F746F722076616C75650D0A004E6F87
:10E750002073756368206D6F746F722C20757365FC
:10E760002061206E756D626572205B302C202564FF
:10E770005D0D0A004D6F746F72202564206973204F
:10E780007365742061742025640D0A00496E7661FA
:10E790006C6964206D6F746F722076616C75652C86
:10E7A00020313030302E2E323030300D0A0053659B
:10E7B0007474696E67206D6F746F722025642074A5
:10E7C0006F2025640D0A0061757820257520257558
:10E7D0000D0A00496E76616C696420466561747546
:10E7E000726520696E6465783A206D757374206275
:10E7F00065203C2025750D0A002025642025640035
:10E8000043757272656E742073657474696E677394
:10E810003A200D0A0025732073657420746F200060
:10E820004552523A2056616C756520617373696771
:10E830006E6D656E74206F7574206F662072616EE8
:10E8400067650D0A004552523A20556E6B6E6F7720
:10E850006E207661726961626C65206E616D650D16
:10E860000A0043757272656E7420436F6E66696745
:10E870003A20436F70792065766572797468696EA5
:10E88000672062656C6F7720686572652E2E2E0D8D
:10E890000A006D697865722025730D0A00636D6941
:10E8A0007820256400636D6978202564203020304D
:10E8B000203020300D0A0066656174757265202D68
:10E8C00025730D0A00666561747572652025730DE8
:10E8D0000A006D61702025730D0A00736574202590
:10E8E00073203D20004E4709004F4B0900437573CC
:10E8F000746F6D206D697865723A200D0A4D6F74E2
:10E900006F720954687209526F6C6C0950697463B4
:10E9100068095961770D0A002325643A09002573B7
:10E92000090053616E69747920636865636B3A0905
:10E93000007265736574006C6F6164004C6F616494
:10E940006564202573206D69782E2E2E0D0A0057E0
:10E95000726F6E67206E756D626572206F662061E2
:10E960007267756D656E74732C206E6565647320B7
:10E970006964782074687220726F6C6C207069749E
:10E980006368207961770D0A004D6F746F72206E95
:10E99000756D626572206D757374206265206265A5
:10E9A000747765656E203120616E642025640D0AE0
:10E9B000000D0A456E746572696E6720434C4920EC
:10E9C0004D6F64652C2074797065202765786974B3
:10E9D0002720746F2072657475726E2C206F722000
:10E9E0002768656C70270D0A000D0A2320000D1B97
:10E9F0005B4B001B5B324A1B5B313B31480045528D
:10EA0000523A20556E6B6E6F776E20636F6D6D613D
:10EA10006E642C20747279202768656C702700085A
:10EA20002008006C6F6F7074696D6500656D665FBE
:10EA300061766F6964616E6365006D69647263001D
:10EA40006D696E7468726F74746C65006D61787452
:10EA500068726F74746C65006D696E636F6D6D6163
:10EA60006E64006D696E636865636B006D617863E9
:10EA70006865636B006465616462616E6433645FE2
:10EA80006C6F77006465616462616E6433645F68B3
:10EA9000696768006E65757472616C3364006465E3
:10EAA000616462616E6433645F7468726F74746C05
:10EAB00065006D6F746F725F70776D5F7261746502
:10EAC00000736572766F5F70776D5F726174650059
:10EAD00072657461726465645F61726D00666C6119
:10EAE00070735F73706565640066697865647769E3
:10EAF0006E675F616C74686F6C645F6469720072EA
:10EB000065626F6F745F63686172616374657200E0
:10EB1000736F667473657269616C5F62617564724C
:10EB200061746500736F667473657269616C5F31DF
:10EB30005F696E76657274656400736F6674736581
:10EB40007269616C5F325F696E76657274656400CC
:10EB50006770735F74797065006770735F62617569
:10EB600064726174650073657269616C72785F7458
:10EB70007970650074656C656D657472795F70722B
:10EB80006F76696465720074656C656D6574727921
:10EB90005F706F72740074656C656D657472795F17
:10EBA00073776974636800766261747363616C651E
:10EBB00000766261746D617863656C6C766F6C74FD
:10EBC00061676500766261746D696E63656C6C7611
:10EBD0006F6C7461676500706F7765725F61646305
:10EBE0005F6368616E6E656C00616C69676E5F671C
:10EBF00079726F00616C69676E5F61636300616C5D
:10EC000069676E5F6D616700616C69676E5F626FF7
:10EC10006172645F726F6C6C00616C69676E5F62D9
:10EC20006F6172645F706974636800616C69676EBC
:10EC30005F626F6172645F796177007961775F63AA
:10EC40006F6E74726F6C5F646972656374696F6E06
:10EC5000006163635F6861726477617265006D6112
:10EC6000785F616E676C655F696E636C696E617415
:10EC7000696F6E006D6F726F6E5F74687265736836
:10EC80006F6C64006779726F5F6C70660067797291
:10EC90006F5F636D70665F666163746F7200677942
:10ECA000726F5F636D70666D5F666163746F720033
:10ECB0007069645F636F6E74726F6C6C65720079FB
:10ECC00061776465616462616E6400616C745F6841
:10ECD0006F6C645F7468726F74746C655F6E657579
:10ECE0007472616C00616C745F686F6C645F666104
:10ECF00073745F6368616E6765007468726F7474C3
:10ED00006C655F636F7272656374696F6E5F766165
:10ED10006C7565007468726F74746C655F636F7294
:10ED200072656374696F6E5F616E676C65007263B4
:10ED30005F726174650072635F6578706F007468FC
:10ED4000725F6D6964007468725F6578706F0072DD
:10ED50006F6C6C5F70697463685F72617465007971
:10ED600061777261746500747061726174650074BA
:10ED700070615F627265616B706F696E740066616D
:10ED8000696C736166655F64656C61790066616971
:10ED90006C736166655F6F66665F64656C61790060
:10EDA0006661696C736166655F7468726F74746CB8
:10EDB00065006661696C736166655F64657465634F
:10EDC000745F7468726573686F6C640072737369E2
:10EDD0005F6175785F6368616E6E656C00796177FD
:10EDE0005F646972656374696F6E007472695F75E0
:10EDF0006E61726D65645F736572766F0067696DD1
:10EE000062616C5F666C616773006163635F6C7005
:10EE1000665F666163746F720061636378795F64D3
:10EE200065616462616E64006163637A5F646561F9
:10EE30006462616E64006163635F756E61726D65CB
:10EE40006463616C006163635F7472696D5F7069B4
:10EE5000746368006163635F7472696D5F726F6C85
:10EE60006C006261726F5F7461625F73697A6500E2
:10EE70006261726F5F6E6F6973655F6C706600626E
:10EE800061726F5F63665F76656C006261726F5F6F
:10EE900063665F616C74006D61675F6465636C6974
:10EEA0006E6174696F6E006770735F706F735F700F
:10EEB000006770735F706F735F69006770735F7076
:10EEC0006F735F64006770735F706F73725F700061
:10EED0006770735F706F73725F69006770735F70E4
:10EEE0006F73725F64006770735F6E61765F70004E
:10EEF0006770735F6E61765F69006770735F6E61E4
:10EF0000765F64006770735F77705F7261646975C4
:10EF100073006E61765F636F6E74726F6C735F689F
:10EF2000656164696E67006E61765F7370656564C4
:10EF30005F6D696E006E61765F73706565645F6DAD
:10EF40006178006E61765F736C65775F726174657E
:10EF500000705F706974636800695F7069746368EA
:10EF600000705F726F6C6C00695F726F6C6C007028
:10EF70005F79617700695F79617700705F616C74B8
:10EF800000695F616C7400645F616C7400705F6C39
:10EF90006576656C00695F6C6576656C00645F6CB6
:10EFA0006576656C00705F76656C00695F76656C90
:10EFB00000645F76656C00617578006665617475E4
:10EFC00072655F6E616D6520617578666C61672042
:10EFD0006F7220626C616E6B20666F72206C697359
:10EFE0007400636D69780064657369676E2063758A
:10EFF00073746F6D206D6978657200646566617504
:10F000006C747300726573657420746F2064656638
:10F0100061756C747320616E64207265626F6F74C9
:10F020000064756D70007072696E7420636F6E6637
:10F030006967757261626C652073657474696E6767
:10F040007320696E2061207061737461626C652049
:10F05000666F726D006578697400666561747572BB
:10F0600065006C697374206F72202D76616C206F5F
:10F07000722076616C00677073706173737468726C
:10F080006F75676800706173737468726F75676815
:10F090002067707320746F2073657269616C0068FB
:10F0A000656C70006D6170006D617070696E6720D5
:10F0B0006F66207263206368616E6E656C206F728C
:10F0C000646572006D69786572206E616D65206F90
:10F0D00072206C697374006D6F746F720067657471
:10F0E0002F736574206D6F746F72206F75747075F7
:10F0F000742076616C75650070726F66696C65006E
:10F10000696E64657820283020746F20322900737E
:10F11000617665007361766520616E642072656258
:10F120006F6F74006E616D653D76616C7565206F03
:10F130007220626C616E6B206F72202A20666F7283
:10F14000206C6973740073686F77207379737465CA
:10F150006D207374617475730076657273696F6E78
:10F16000004759524F00414343004241524F005320
:10F170004F4E415200475053004750532B4D41478B
:10F18000004144584C333435004D505536303530FD
:10F19000004D4D413834357800424D413238300011
:10F1A0004E6F6E6500545249005155414450005114
:10F1B000554144580042490047494D42414C00598D
:10F1C00036004845583600464C59494E475F574926
:10F1D0004E47005934004845583658004F43544F65
:10F1E0005838004F43544F464C415450004F4354FD
:10F1F0004F464C41545800414952504C414E4500F5
:10F2000048454C495F3132305F4343504D004845DB
:10F210004C495F39305F44454700565441494C34AE
:10F220000048455836480050504D5F544F5F534595
:10F2300052564F004455414C434F50544552005391
:10F24000494E474C45434F50544552004355535443
:10F250004F4D0050504D005642415400494E464CCF
:10F26000494748545F4143435F43414C0053455233
:10F2700049414C5258004D4F544F525F53544F50D8
:10F2800000534552564F5F54494C5400534F465417
:10F2900053455249414C004C45445F52494E47004A
:10F2A0004641494C534146450054454C454D455413
:10F2B000525900504F5745524D4554455200564102
:10F2C00052494F003344000061F1000866F1000824
:10F2D0006AF100087DF100086FF1000875F100087F
:10F2E00079F100080000000023EA00080200000095
:10F2F000D810002000000000282300002CEA00089D
:10F3000000000000DA1000200000000001000000F2
:10F310003AEA000802000000DE110020B0040000FC
:10F32000A406000040EA0008020000009C11002032
:10F3300000000000D00700004CEA000802000000B6
:10F340009E11002000000000D007000058EA0008CD
:10F3500002000000A011002000000000D007000003
:10F3600063EA000802000000E01100200000000035
:10F37000D00700006CEA000802000000E211002043
:10F3800000000000D007000075EA0008020000003D
:10F39000A211002000000000D007000084EA00084D
:10F3A00002000000A411002000000000D0070000AF
:10F3B00094EA000802000000A611002000000000EE
:10F3C000D00700009EEA000802000000A8110020FB
:10F3D00000000000D0070000B2EA000802000000B0
:10F3E000AA11002032000000007D0000C1EA0008E0
:10F3F00002000000AC11002032000000F201000009
:10F40000D0EA000800000000E41100200000000025
:10F4100001000000DDEA000800000000E511002006
:10F420000000000064000000E9EA0008010000009C
:10F43000E6110020FFFFFFFF01000000FFEA0008C7
:10F4400000000000F6110020300000007E000000E7
:10F4500014EB000804000000EC110020B0040000D0
:10F4600000C2010010EB000804000000F0110020B1
:10F47000B0040000004B000024EB00080000000076
:10F48000F411002000000000010000003AEB000829
:10F4900000000000F5110020000000000100000045
:10F4A00050EB000800000000E81100200000000000
:10F4B0000400000059EB000801000000E9110020E1
:10F4C000000000000400000066EB000800000000DF
:10F4D000DC110020000000000300000074EB0008B5
:10F4E00000000000F81100200000000001000000F2
:10F4F00087EB000800000000F91100200000000068
:10F500000200000096EB000800000000FA11002045
:10F510000000000001000000A7EB00080000000050
:10F52000D01100200A000000C8000000B1EB000864
:10F5300000000000D11100200A000000320000008D
:10F54000C4EB000800000000D21100200A000000F7
:10F5500032000000D7EB000800000000D3110020AB
:10F560000000000009000000E9EB000800000000B6
:10F57000AE1100200000000008000000F4EB0008BD
:10F5800000000000AF110020000000000800000093
:10F59000FEEB000800000000B01100200000000099
:10F5A0000800000008EC000803000000B211002071
:10F5B0004CFFFFFF6801000019EC00080300000089
:10F5C000B41100204CFFFFFF680100002BEC000885
:10F5D00003000000B61100204CFFFFFF680100008F
:10F5E0003BEC000801000000B8110020FFFFFFFF06
:10F5F0000100000051EC000800000000B9110020DB
:10F6000000000000050000005EEC000802000000A1
:10F61000C2110020640000008403000074EC0008A4
:10F6200000000000C0110020000000008000000069
:10F6300084EC000802000000BA1100200000000065
:10F64000000100008DEC000802000000BC11002049
:10F6500064000000E80300009EEC000802000000C7
:10F66000BE11002064000000E8030000B0EC0008B8
:10F6700000000000681400200000000001000000ED
:10F680001FEE000800000000D4140020000000005D
:10F6900020000000BFEC000800000000D51400208E
:10F6A0000000000064000000CBEC00080000000037
:10F6B000D614002001000000FA000000E5EC00086C
:10F6C00000000000D714002000000000010000002E
:10F6D000FAEC000800000000DA140020000000002E
:10F6E0009600000014ED000802000000D81400206D
:10F6F00001000000840300002EED0008000000005F
:10F700008714002000000000FA00000036ED000819
:10F7100000000000881400200000000064000000C9
:10F720003EED0008000000008914002000000000E9
:10F730006400000046ED0008000000008A1400206C
:10F7400000000000640000004FED00080000000011
:10F750008B14002000000000640000005FED000832
:10F76000000000008C140020000000006400000075
:10F7700067ED0008000000008D140020000000006C
:10F78000640000006FED0008020000008E140020ED
:10F79000E8030000D00700007EED00080000000034
:10F7A0001C15002000000000C80000008DED0008BE
:10F7B000000000001D15002000000000C80000002F
:10F7C000A0ED0008020000001E150020E803000064
:10F7D000D0070000B2ED0008020000002015002054
:10F7E00064000000D0070000CCED0008010000001C
:10F7F000E71100200000000004000000DDED00081B
:10F800000100000022150020FFFFFFFF01000000A3
:10F81000EBED0008010000002315002000000000AF
:10F8200001000000FDED000800000000241500208C
:10F8300000000000FF0000000AEE000800000000C9
:10F840009614002000000000FA00000019EE0008E5
:10F850000000000098140020000000006400000078
:10F8600028EE0008000000009714002000000000AF
:10F870006400000036EE000800000000A81400201C
:10F88000000000000100000045EE00080300000039
:10F8900094140020D4FEFFFF2C01000054EE000859
:10F8A0000300000092140020D4FEFFFF2C01000092
:10F8B00062EE000800000000991400200000000023
:10F8C0003000000070EE0008050000009C140020CD
:10F8D00000000000010000007FEE000805000000AD
:10F8E000A014002000000000010000008BEE0008C2
:10F8F00005000000A414002000000000010000002A
:10F9000097EE00080300000090140020B0B9FFFF3C
:10F9100050460000A7EE0008000000006D14002013
:10F9200000000000C8000000B1EE00080000000068
:10F930007714002000000000C8000000BBEE0008A3
:10F94000000000008114002000000000C80000003A
:10F95000C5EE0008000000006E140020000000004A
:10F96000C8000000D0EE000800000000781400205D
:10F9700000000000C8000000DBEE000800000000EE
:10F980008214002000000000C8000000E6EE00081D
:10F99000000000006F14002000000000C8000000FC
:10F9A000F0EE0008000000007914002000000000C4
:10F9B000C8000000FAEE00080000000083140020D8
:10F9C00000000000C800000004EF00080200000072
:10F9D0002615002000000000D007000012EF0008EC
:10F9E000000000002A1500200000000001000000B7
:10F9F00027EF0008020000002C1500200A0000007C
:10FA0000D007000035EF0008020000002E1500208E
:10FA10000A000000D007000043EF000800000000CB
:10FA200029150020000000006400000051EF0008CC
:10FA3000000000006A14002000000000C800000060
:10FA400059EF0008000000007414002000000000BE
:10FA5000C800000023EC0008000000007E14002015
:10FA600000000000C800000061EF00080000000076
:10FA70006914002000000000C800000068EF0008C2
:10FA8000000000007314002000000000C800000007
:10FA900012EC0008000000007D14002000000000AF
:10FAA000C80000006FEF0008000000006B14002089
:10FAB00000000000C800000075EF00080000000012
:10FAC0007514002000000000C800000035EC00089C
:10FAD000000000007F14002000000000C8000000AB
:10FAE0007BEF0008000000006C1400200000000004
:10FAF000C800000081EF000800000000761400201C
:10FB000000000000C800000087EF000800000000AF
:10FB10008014002000000000C80000008DEF0008E5
:10FB2000000000007014002000000000C800000069
:10FB300095EF0008000000007A140020000000008B
:10FB4000C80000009DEF00080000000084140020A1
:10FB500000000000C8000000A5EF00080000000041
:10FB60007214002000000000C8000000ABEF000885
:10FB7000000000007C14002000000000C80000000D
:10FB8000B1EF000800000000861400200000000013
:10FB9000C8000000524F4C4C3B50495443483B591D
:10FBA00041573B414C543B506F733B506F73523B3A
:10FBB0004E6176523B4C4556454C3B4D41473B567A
:10FBC000454C3B0041524D3B00414E474C453B00AC
:10FBD000484F52495A4F4E3B004241524F3B00560C
:10FBE0004152494F3B004D41473B00484541444647
:10FBF0005245453B004845414441444A3B0043414E
:10FC00004D535441423B0043414D545249473B0000
:10FC100047505320484F4D453B0047505320484FD5
:10FC20004C443B0050415353544852553B004245CD
:10FC3000455045523B004C45444D41583B004C45D6
:10FC4000444C4F573B004C4C49474854533B0043AE
:10FC5000414C49423B00474F5645524E4F523B00A4
:10FC60004F53442053573B0054454C454D45545247
:10FC7000593B00000000004B000000CB61636F7334
:10FC800066000000000000007371727466000000DE
:10FC9000000FC93F000F494000CB9640000FC940FC
:10FCA0000053FB4000CB164100ED2F41000F4941AE
:10FCB0000031624100537B41003A8A4100CB9641BA
:10FCC000005CA34100EDAF41007EBC41000FC94183
:10FCD00000A0D5410031E24100C2EE410053FB419A
:10FCE00000F20342003A0A420083104200CB16425F
:10FCF00000141D42005C234200A5294200ED2F4262
:10FD000000363642007E3C4200C74242000F494264
:10FD1000A2000000F9000000830000006E00000057
:10FD20004E00000044000000150000002900000003
:10FD3000FC0000002700000057000000D100000078
:10FD4000F500000034000000DD000000C0000000ED
:10FD5000DB00000062000000950000009900000038
:10FD60003C00000043000000900000004100000043
:10FD7000FE0000005100000063000000AB00000026
:10FD8000DE000000BB000000C500000061000000B4
:10FD9000B7000000240000006E0000003A000000E0
:10FDA000420000004D000000D2000000E000000012
:10FDB00006000000490000002E000000EA000000DC
:10FDC00009000000D1000000920000001C000000AB
:10FDD000FE0000001D000000EB0000001C00000001
:10FDE000B100000029000000A70000003E00000054
:10FDF000E80000008200000035000000F50000006F
:10FE00002E000000BB000000440000008400000041
:10FE1000E90000009C0000007000000026000000C7
:10FE2000B40000005F0000007E0000004100000000
:10FE30003900000091000000D600000039000000E9
:10FE4000830000005300000039000000F4000000AF
:10FE50009C000000840000005F0000008B00000098
:10FE6000BD000000F9000000280000003B00000079
:10FE70001F000000F800000097000000FF000000D5
:10FE8000DE00000005000000980000000F000000E8
:10FE9000EF0000002F000000110000008B000000A8
:10FEA0005A0000000A0000006D0000001F00000062
:10FEB0006D000000360000007E000000CF00000052
:10FEC00027000000CB00000009000000B700000080
:10FED0004F000000460000003F00000066000000E8
:10FEE0009E0000005F000000EA0000002D000000FE
:10FEF0007500000027000000BA000000C7000000E5
:10FF0000EB000000E5000000F10000007B000000B5
:10FF10003D0000000700000039000000F70000006D
:10FF20008A0000005200000092000000EA00000079
:10FF30006B000000FB0000005F000000B10000004B
:10FF40001F0000008D0000005D00000008000000A0
:10FF500056000000030000003000000046000000D2
:10FF6000FC0000007B0000006B000000AB00000004
:10FF7000F0000000CF000000BC00000020000000E6
:10FF80009A000000F4000000360000001D00000090
:10FF9000A9000000E30000009100000061000000E3
:10FFA0005E000000E60000001B00000008000000EA
:10FFB0006500000099000000850000005F0000005F
:10FFC00014000000A00000006800000040000000D5
:10FFD0008D000000FF000000D8000000800000003D
:10FFE0004D000000730000002700000031000000F9
:10FFF000060000000600000015000000560000008A
:020000040801F1
:10000000CA00000073000000A8000000C900000042
:1000100060000000E20000007B000000C000000063
:100020008C0000006B0000000400000007000000CE
:10003000090000000000C93F0000F0390000DA3775
:100040000000A2330000842E0000502B0000C227C5
:100050000000D0220000C41F0000C61B000044178F
:100060006937AC3168212233B40F14336821A233CD
:100070003863ED3EDA0F493F5E987B3FDA0FC93FA8
:100080000020202020202020202028282828282068
:100090002020202020202020202020202020202060
:1000A00020881010101010101010101010101010C8
:1000B00010040404040404040404041010101010B8
:1000C0001010414141414141010101010101010182
:1000D00001010101010101010101010110101010D4
:1000E0001010424242424242020202020202020254
:1000F00002020202020202020202020210101010A8
:1001000020000000000000000000000000000000CF
:1001100000000000000000000000000000000000DF
:1001200000000000000000000000000000000000CF
:1001300000000000000000000000000000000000BF
:1001400000000000000000000000000000000000AF
:10015000000000000000000000000000000000009F
:10016000000000000000000000000000000000008F
:10017000000000000000000000000000000000007F
:100180000000000043000000A8010020F8B500BFF7
:10019000F8BC08BC9E467047F8B500BFF8BC08BC68
:0401A0009E467047C0
:0801A4007DD9000835010008B7
:0401AC001101000835
:1001B00000000040000002000000004004000400B5
:1001C0000000004008000800000000400C00100083
:1001D000000400400000020000040040040004008D
:1001E0000004004008000800000400400C0010005B
:1001F00003010001894300080000803F0000000067
:1002000000000000DC05DC05DC05DC05DC05DC05A8
:10021000DC05DC050000803F01000000000000005C
:10022000C4FB00080000000001000000C9FB00083A
:100230000100000002000000D0FB000802000000E6
:1002400003000000D9FB00080300000004000000C8
:10025000DFFB00080400000005000000E6FB0008CA
:100260000500000006000000EBFB0008060000008F
:1002700007000000F5FB0008070000000800000070
:10028000FEFB0008080000000900000007FC000851
:10029000090000000A00000010FC00080A0000002D
:1002A0000B0000001AFC00080B0000000C0000000E
:1002B00024FC00080C0000000D0000002EFC0008CB
:1002C0000D0000000E00000036FC00080E000000CB
:1002D0000F0000003EFC00080F00000010000000AE
:1002E00046FC000810000000110000004FFC000850
:1002F000110000001200000056FC0008120000006F
:100300001300000060FC000813000000140000004F
:1003100068FC000814000000150000000000000048
:10032000FF000000000000000000000001020304C4
:100330000607080900127A0000A24A04020406080F
:10034000000000000102030401020304060708097B
:10035000010000008000010800000000940400205B
:10036000FC040020640500200000000000000000E4
:10037000000000000000000000000000000000007D
:1003800000000000000000000000000084010108DF
:10039000000000000000000000000000000000005D
:1003A000000000000000000000000000000000004D
:1003B000000000000000000000000000000000003D
:1003C000000000000000000000000000000000002D
:1003D000000000000000000000000000000000001D
:1003E000000000000000000000000000000000000D
:1003F00000000000000000000000000000000000FD
:1004000001000000000000000E33CDAB34126DE699
:10041000ECDE05000B000000000000000000000002
:1004200000000000000000000000000000000000CC
:1004300000000000000000000000000000000000BC
:1004400000000000000000000000000000000000AC
:10045000000000000000000000000000000000009C
:04078000A8010020AC
:0400000508000000EF
:00000001FF
